:100000000C94FD4B0C941E4C0C946AD40C941E4C16
:100010000C941E4C0C941E4C0C941E4C0C941E4CB8
:100020000C941E4C0C941E4C0C941E4C0C9495D6A7
:100030000C941E4C0C941E4C0C940AB70C941E4C41
:100040000C941E4C0C941E4C0C941E4C0C941E4C88
:100050000C941E4C0C941E4C0C941E4C0C941E4C78
:100060000C941E4C0C9484D40C9413D40C941E4CFD
:100070000C94DDCD0C947FCD0C94BBCD0C941E4C18
:100080000C9435D50C941E4C0C941E4C0C941E4CA8
:100090000C941E4C0C941E4C0C941E4C0C941E4C38
:1000A0000C941E4C0C941E4C0C941E4C0C9489BE4B
:1000B0000C942DBF0C941E4C0C941E4C0C94FBB84D
:1000C0000C941E4C0C941E4C0C941E4C0C941E4C08
:1000D0000C941E4C0C941E4C0C941E4C0C941E4CF8
:1000E0000C944DA90C941E4C0C941E4C0C941E4C5C
:1000F0000C941E4C0C941E4C0C941E4C0C941E4CD8
:100100000C9460BE0C9404BF0C9437BE0C94DBBE00
:100110000C941E4C0C941E4C0C941E4C0C941E4CB7
:100120000C941E4C0C941E4C0C941E4C0C941E4CA7
:100130000C941E4C0C945FB80C941E4C0C941E4CEA
:100140000C941E4C0C941E4C0C941E4C0C941E4C87
:100150000C941E4C0C941E4C0C9443A90C941E4CF5
:100160000C941E4C0C941E4C0C941E4C0C941E4C67
:100170000C941E4C0C941E4C0C941E4C0C941E4C57
:100180000C941E4C0C941E4C0C941E4C0C941E4C47
:100190000C941E4C0C941E4C0C941E4C0C941E4C37
:1001A0000C94B2BE0C9456BF0C941E4C0C941E4C76
:1001B0000C94ADB80C941E4C0C941E4C0C941E4C1C
:1001C0000C941E4C0C941E4C0C941E4C0C941E4C07
:1001D0000C941E4C0C941E4C0C941E4C0C941E4CF7
:1001E0000C941E4C0C941E4C62756C757675807563
:1001F0008B75297B297B297B297B297B9175297B21
:10020000297B297B297B297B297B93759D75A77584
:10021000B175BB75297B297B297B297B297B297BB0
:10022000C575297B1B76297B297B297B297B297B2B
:10023000297B297B5A76297B1079297B297B297B8D
:10024000297B297B297B297B297B1079297B297BA9
:10025000297B87768C769676A076A276AC76B77672
:10026000297BC276297B297BFF76297B297B297B09
:10027000297B297B297B297B297B297B297B297B5E
:10028000297B297B297B297B0977297B297B297B72
:10029000297B297B297B297B297B297B13771D7768
:1002A000277770777A77937793779D77A777B1776A
:1002B000BB77C577CA77D477DE77277B277B277B09
:1002C000277B277B277B277B277B277B277B277B1E
:1002D000277B277B277B277B277B277B277B277B0E
:1002E000277B9D77277B277B277B277B277B277B8C
:1002F000277B277B277B277B277B277B277B277BEE
:10030000277B277B277BE877F277FC770678277BAC
:10031000277B277B277B277B277B277B277B937765
:10032000B47A757A797A817A5D7A617A697A6D7A46
:100330008D7AA07AA87AAC7AB07A0C7B857A8178AB
:100340009278A378297B297B1B785375297BB47815
:10035000C578D67810798477F878297B2C78297B32
:10036000E7783D781078297B297B297B4E785F7868
:100370007078D0BDD8BDE0BDE8BDF0BDF8BD00BE11
:1003800008BEFBC058C060C068C070C078C080C0E4
:1003900088C090C098C0A0C0A8C0B0C0B8C0C0C03D
:1003A000E0C0E0C0E0C0E0C0E0C0E0C0E0C0E0C04D
:1003B000E0C0E0C0E0C0E0C0E0C0E0C0E0C0E0C03D
:1003C000E0C0E0C0E0C0E0C0E0C0E0C0E0C0E0C02D
:1003D000E0C0E0C0E0C0E0C0E0C0E0C0E0C0E0C01D
:1003E000E0C0E0C0E0C0C8C0D0C0E0C0E0C0E0C035
:1003F000E0C0E0C0E0C0E0C0E0C0E0C0E0C0E0C0FD
:10040000E0C0E0C0E0C0E0C0E0C0E0C0E0C0E0C0EC
:10041000E0C0E0C0E0C0E0C0E0C0E0C0E0C0E0C0DC
:10042000E0C0E0C0E0C0E0C0E0C0E0C0E0C0E0C0CC
:10043000E0C0E0C0E0C0E0C0E0C0E0C0E0C0E0C0BC
:10044000E0C0E0C0E0C0E0C0D8C0084AD73B3BCE27
:10045000016E84BCBFFDC12F3D6C74319ABD5683C3
:100460003DDA3D00C77F11BED9E4BB4C3E916BAA7B
:10047000AABE000000803F05A84CCDB2D44EB938CA
:1004800036A9020C50B9918688083CA6AAAA2ABEB1
:10049000000000803F07634236B79BD8A71A39682F
:1004A0005618AEBAAB558C1D3CB7CC5763BD6DED3D
:1004B000FD753EF6177231BF000000803F08000056
:1004C00000BE922449123EABAAAA2ABECDCCCC4C87
:1004D0003E00000080BEABAAAAAA3E00000000BFFA
:1004E000000000803F0000000000084178D3BB43BB
:1004F00087D1133D190E3CC3BD4282AD2B3E68EC43
:100500008276BED98FE1A93E4C80EFFFBE01C4FFC9
:100510007F3F0000000000000C9475B00C94857AB9
:100520000C944F5B0C9446C00C94697A0C94615BFC
:100530000C941D680C94D2C40C94A6AA0C94D0BD43
:100540000C94617A0C940F5F0C948CBD0C9492AA5D
:100550000C9409600C94DF6B0C94E75E0C94675B61
:100560000C9470C00C949ACC0C94EB5E0C944E716D
:100570000C945F780C94D55F0C949F6C0C94636220
:100580000C94344C0C94A0C00C94EEBC0C9428C079
:100590000C94E0BD0C942A4C0C9469AB0C94785BE1
:1005A0000C940B5E0C941B5F0C94FF5B0C94204C22
:1005B0000C94F8780C94F2770C94C0C00C94B7614A
:1005C0000C94B2AA0C9480C00C94F2820C943C85DA
:1005D0000C9471B00C94DB610C941B760C94D8676E
:1005E0000C94335E0C94FF5E0C94CA770C942DCC63
:1005F0000C94256D0C945D680C940B5F0C94A467AF
:100600000C94F55F0C94555B0C9496870C94975B57
:100610000C94297B0C9496760C944DB00C9486D057
:100620000C943D780C94726F0C94A3BD0C9469B03B
:100630000C9489D10C9490C00C94F15F0C944A5F97
:100640000C94B85B0C94914F0C949ECA0C94075F69
:100650000C94AFC50C94985C0C94F8BD0C949377F3
:100660000C94255E0C94425B0C94175F0C94ED5F28
:100670000C94CBBB0C946C750C94145D0C94835B44
:100680000C9406780C9422630C9499580C945B5B40
:100690000C940C7B0C941F5F0C94E7780C94A07660
:1006A0000C94AC7A0C94B8C00C94AC760C94A775EE
:1006B0000C946F670C94D8C00C94F0BD0C94E15F5F
:1006C0000C94A7BD0C9453750C94D6780C949BBDD8
:1006D0000C94A9950C947A6F0C94DD7C0C94D15BEE
:1006E0000C94695F0C94A25B0C94FC720C941377CD
:1006F0000C942B5F0C9461830C94734C0C946DB030
:100700000C94DF5E0C94B47C0C946E5C0C949EAAEA
:100710000C9458C00C94D4770C94A7770C94A0B187
:100720000C94D8BD0C9431B00C9404D20C94847702
:100730000C94BB770C94546C0C94E0C00C944E78E1
:100740000C94FC770C948C760C9487760C94C3BC38
:100750000C94CDAE0C94B7760C9467670C9483BD63
:100760000C94015D0C94FBC00C949FBD0C94B9C417
:100770000C94B6AA0C94B46C0C9442C00C94C9AE00
:100780000C94605E0C9473670C9498C00C94F35EA8
:100790000C948D7A0C949AAA0C943A5E0C94C578B9
:1007A0000C94A8C00C94FF760C94C4660C947FBD86
:1007B0000C94AEAA0C94F95F0C948E7D0C946B672C
:1007C0000C94D15F0C94415E0C945A760C94817811
:1007D0000C94E7640C94A87A0C94844C0C94B0C0EC
:1007E0000C94797A0C94A8660C9428BD0C949361AF
:1007F0000C941B780C94E3CA0C94817A0C94A27626
:100800000C94C2760C9439610C94E57C0C9400BE77
:100810000C94757A0C9462750C944C720C943B6237
:100820000C9465830C948DAE0C9411600C94BB7584
:100830000C94FB620C94DA5D0C9420CF0C94637DD5
:100840000C945B630C9452D10C94F2D00C9486BB44
:100850000C940D600C943D620C94FB5E0C94B47887
:100860000C94256C0C94B47A0C9410780C94EEC40F
:100870000C9468C00C94C9B10C9460C00C94A07A1C
:100880000C94B1770C9492780C94D0C00C94277788
:100890000C9491750C94D97C0C94BAC40C941ACD18
:1008A0000C947F5E0C9402620C94D2620C946B7B6D
:1008B0000C94C8C00C94C5770C9410BC0C94707840
:1008C0000C94617C0C94D7BC0C9488620C94375CBB
:1008D0000C94DB5E0C948F610C9408BE0C94126730
:1008E0000C94E8770C94E35E0C948FAE0C941D602E
:1008F0000C9480750C945C6B0C94EF5E0C9491AE30
:100900000C9428600C946D7A0C94E8BD0C94BE672E
:100910000C942CCD0C94035F0C9450BD0C94636725
:100920000C94AD620C94235F0C948C5B0C94107946
:100930000C94AD5B0C94BA720C9478C00C949375C3
:100940000C949D770C948B750C94FD5F0C94825DD8
:100950000C94277B0C94B97C0C94B3D30C94E97C55
:100960000C946D5B0C947A770C941D770C94F2CFF9
:100970000C94B97D0C94DE770C9468D20C94135FC0
:100980000C9496AA0C94A3780C9469830C94AAAA4C
:100990000C9487BD0C9488C00C9476750C949D685B
:1009A0000C940BC50C9400530C9431720C94097781
:1009B0000C9405600C94DD5F0C948C5F0C94F75ED6
:1009C0000C94065E0C94275F0C94E55F0C942C78D5
:1009D0000C9401600C94B07A0C946D5F0C94C57506
:1009E0000C94B1750C94F2670C94E85B0C94A2AA79
:1009F0000C941CB00C94726C0C949D750C94E95F73
:100A00000C94D95F0C94E17C0C94C7AE0C94D15C2F
:100A10000C947B7B0C94247D0C9470770C942C5E4E
:100A20000C945D7A0C94BBCC0C9422C05B2573258E
:100A3000735D20257320257320706F736974696F4F
:100A40006E2531382E336625730A005B25732573B6
:100A50005D202573202573206F66667365742532CB
:100A6000302E336625730A005B257325735D2025C0
:100A700073207A65726F206261636B6F66662531E1
:100A8000392E336625730A005B257325735D202597
:100A900073206C61746368206261636B6F666625A6
:100AA00031382E336625730A005B257325735D206C
:100AB0002573206C617463682076656C6F6369745C
:100AC000792531332E306625732F6D696E0A005BF0
:100AD000257325735D20257320736561726368201B
:100AE00076656C6F636974792531322E30662573B3
:100AF0002F6D696E0A005B257325735D20257320B9
:100B0000737769746368206D617825313764205B81
:100B1000303D6F66662C313D686F6D696E672C32B3
:100B20003D6C696D69742C333D6C696D69742B681B
:100B30006F6D696E675D0A005B257325735D202507
:100B40007320737769746368206D696E253137642B
:100B5000205B303D6F66662C313D686F6D696E6756
:100B60002C323D6C696D69742C333D6C696D697410
:100B70002B686F6D696E675D0A005B257325735D79
:100B8000202573207261646975732076616C7565C8
:100B90002532302E346625730A005B257325735D7C
:100BA000202573206A756E6374696F6E20646576A4
:100BB000696174696F6E2531342E3466257320287F
:100BC0006C61726765722069732066617374657207
:100BD000290A005B257325735D202573206A6572E1
:100BE0006B20686F6D696E672531362E3066257310
:100BF0002F6D696E5E33202A2031206D696C6C691F
:100C00006F6E0A005B257325735D202573206A656E
:100C1000726B206D6178696D756D2531352E30668A
:100C200025732F6D696E5E33202A2031206D696C2B
:100C30006C696F6E0A005B257325735D2025732038
:100C400074726176656C206D696E696D756D2531A4
:100C5000372E336625730A005B257325735D2025C7
:100C6000732074726176656C206D6178696D756D45
:100C70002531372E336625730A005B257325735D96
:100C80002025732076656C6F63697479206D6178B7
:100C9000696D756D2531312E306625732F6D696E46
:100CA0000A005B257325735D2025732066656564E6
:100CB00072617465206D6178696D756D2531312EB5
:100CC000306625732F6D696E0A005B257325735D91
:100CD0002025732061786973206D6F646525313834
:100CE000642025730A005B6D615D20206D696E20B4
:100CF000617263207365676D656E742531382E33BC
:100D00006625730A005B736C5D2020736F66742028
:100D10006C696D697420656E61626C652531326441
:100D20000A005B63745D202063686F7264616C20ED
:100D3000746F6C6572616E63652531372E3466257C
:100D4000730A005B6A615D20206A756E6374696F67
:100D50006E20616363656C65726174696F6E2538BE
:100D60002E306625730A005B6764695D20646566E2
:100D700061756C742067636F646520646973746166
:100D80006E6365206D6F6465253264205B303D477E
:100D900039302C313D4739315D0A005B6770615D48
:100DA0002064656661756C742067636F646520708C
:100DB00061746820636F6E74726F6C253364205B9E
:100DC000303D4736312C313D4736312E312C323DC6
:100DD0004736345D0A005B67636F5D20646566615A
:100DE000756C742067636F646520636F6F72642035
:100DF00073797374656D253364205B312D3620283B
:100E00004735342D473539295D0A005B67756E5DBE
:100E10002064656661756C742067636F6465207516
:100E20006E697473206D6F6465253564205B303D99
:100E30004732302C313D4732315D0A005B67706CC0
:100E40005D2064656661756C742067636F646520FE
:100E5000706C616E6525313064205B303D47313701
:100E60002C313D4731382C323D4731395D0A002560
:100E70006320776F726B206F66667365743A2531F5
:100E8000322E336625730A002563206D616368691D
:100E90006E6520706F736E3A2531312E336625737F
:100EA0000A00256320706F736974696F6E3A25318B
:100EB000352E336625730A00546F6F6C206E756D86
:100EC0006265722020202020202020202025640A16
:100ED00000466565642072617465206D6F64653AD3
:100EE00020202020202025730A0044697374616E3D
:100EF0006365206D6F64653A202020202020202526
:100F0000730A0050617468204D6F64653A20202098
:100F1000202020202020202025730A00506C616EA4
:100F2000653A202020202020202020202020202062
:100F30002025730A004D6F74696F6E206D6F6465B4
:100F40003A20202020202020202025730A00436FF3
:100F50006F7264696E6174652073797374656D3A3C
:100F600020202025730A00556E6974733A202020D2
:100F700020202020202020202020202025730A004F
:100F8000486F6D696E672073746174653A20202024
:100F9000202020202025730A0046656564686F6C58
:100FA000642073746174653A20202020202025730A
:100FB0000A004D6F74696F6E2073746174653A2016
:100FC0002020202020202025730A004379636C65AF
:100FD0002073746174653A20202020202020202076
:100FE00025730A00526177206D616368696E652020
:100FF00073746174653A20202025730A004D616383
:1010000068696E652073746174653A202020202021
:10101000202025730A004C696E65206E756D62652F
:10102000723A2531302E30660A00466565642072BA
:101030006174653A2531362E336625732F6D696EDE
:101040000A0056656C6F636974793A2531372E331F
:101050006625732F6D696E0A00B0107F105F104710
:101060003935202D20756E6974732D7065722D725F
:1010700065766F6C7574696F6E206D6F646500477F
:101080003934202D20756E6974732D7065722D6D45
:10109000696E757465206D6F64652028692E652EF4
:1010A000206665656472617465206D6F64652900F2
:1010B000473933202D20696E766572736520746917
:1010C0006D65206D6F646500EC10CC1047393120E0
:1010D0002D20696E6372656D656E74616C20646944
:1010E0007374616E6365206D6F64650047393020ED
:1010F0002D206162736F6C7574652064697374610F
:101100006E6365206D6F6465003D1125110F1147F9
:101110003634202D20636F6E74696E756F75732081
:101120006D6F6465004736312E31202D2065786162
:1011300063742073746F70206D6F6465004736317F
:10114000202D2065786163742070617468206D6F54
:10115000646500771168115911473139202D2059E4
:101160005A20706C616E6500473138202D20585A26
:1011700020706C616E6500473137202D2058592052
:10118000706C616E65000312F111D811B7119011E6
:10119000473830202D2063616E63656C206D6F745D
:1011A000696F6E206D6F646520286E6F6E652061BB
:1011B00063746976652900473320202D20636F759D
:1011C0006E74657220636C6F636B77697365206101
:1011D0007263206665656400473220202D20636CB1
:1011E0006F636B7769736520617263206665656400
:1011F00000473120202D206C696E65617220666584
:10120000656400473020202D206C696E6561722076
:10121000747261766572736520287365656B290049
:10122000CA12B01296127C12621248122E12473560
:1012300039202D20636F6F7264696E61746520734D
:10124000797374656D203600473538202D20636F23
:101250006F7264696E6174652073797374656D2053
:101260003500473537202D20636F6F7264696E61DA
:1012700074652073797374656D20340047353620AA
:101280002D20636F6F7264696E617465207379736A
:1012900074656D203300473535202D20636F6F72E4
:1012A00064696E6174652073797374656D203200B2
:1012B000473534202D20636F6F7264696E617465E9
:1012C0002073797374656D203100473533202D20EC
:1012D0006D616368696E6520636F6F7264696E61CA
:1012E00074652073797374656D00FD12F712F01246
:1012F000486F6D696E6700486F6D6564004E6F746E
:1013000020486F6D65640031132C13271321131CC3
:10131000131313456E6420486F6C6400486F6C644F
:1013200000446563656C00506C616E0053796E63B8
:10133000004F666600441340133B13486F6C640013
:1013400052756E0053746F70006E1364135E135702
:101350001353134A6F6700486F6D696E67005072D0
:101360006F6265004D616368696E696E67004F6604
:101370006600A4139E13981393138F13891380137D
:1013800053687574646F776E004379636C650045CC
:101390006E640053746F7000416C61726D00526531
:1013A00061647900496E697469616C697A696E6714
:1013B0000007140114FB13F613F213EE13E913E301
:1013C00013DD13D613D213C91353687574646F7782
:1013D0006E004A6F6700486F6D696E6700437963FE
:1013E0006C650050726F626500486F6C64005275E6
:1013F0006E00456E640053746F7000416C61726DD5
:1014000000526561647900496E697469616C697A3A
:10141000696E67002E141814473231202D206D6933
:101420006C6C696D65746572206D6F646500473220
:1014300030202D20696E63686573206D6F646500D0
:1014400068145D14511448145B7261646975735DAE
:10145000005B696E686962697465645D005B7374E2
:10146000616E646172645D005B64697361626C6586
:10147000645D0082147E1479142064656700206D19
:101480006D0020696E002A2A2A204E4F5449434598
:10149000202A2A2A20526573657474696E67206257
:1014A000617564207261746520746F202573005B20
:1014B000626175645D2055534220626175642072DB
:1014C00061746525313564205B313D393630302C0F
:1014D000323D31393230302C333D33383430302CDA
:1014E000343D35373630302C353D313135323030C2
:1014F0002C363D3233303430305D0A005B72786D0B
:101500005D2073657269616C205258206D6F64654F
:1015100025313564205B303D73747265616D696E91
:10152000675F6D6F64652C313D7061636B65745FDF
:101530006D6F64655D0A005B65785D2020656E6196
:10154000626C6520666C6F7720636F6E74726F6C6F
:1015500025313064205B303D6F66662C313D584F3D
:101560004E2F584F46462C323D5254532F4354531E
:101570005D0A005B65655D2020656E61626C6520BB
:101580006563686F25313864205B303D6F66662C7B
:10159000313D6F6E5D0A005B65635D20206578708C
:1015A000616E64204C4620746F2043524C46206F7D
:1015B0006E205458253664205B303D6F66662C31B2
:1015C0003D6F6E5D0A00F915F415EE15E815E2158C
:1015D000DB15D41532333034303000313135323010
:1015E0003000353736303000333834303000313960
:1015F0003230300039363030003000737973006695
:1016000062000000000702D97C02623B62A83AF641
:1016100088DC43737973006676000000000703DD01
:101620007C02623B62AC3AEC51783F73797300689C
:1016300070000000000700E17C02622263B43A00FF
:1016400000803F737973006876000000000700E5B2
:101650007C0262B97CB83A0000004173797300697A
:1016600064000000000400E97C617C3B62A43A0055
:10167000000000000000006E00000000000100DB20
:101680005ED15BD2629B3200000000000000006C63
:10169000696E6500000100DB5EE85BD2629B320090
:1016A0000000000000000076656C000000000241B0
:1016B0005EFF5B3B62A43A00000000000000006691
:1016C00065656400000002605E375C3B62A43A001E
:1016D000000000000000007374617400000000DF6F
:1016E0005E425B3B62A43A00000000000000006D17
:1016F00061637300000000E35E4F5B3B62A43A004D
:10170000000000000000006379637300000000E740
:101710005E555B3B62A43A00000000000000006DD3
:101720006F747300000000EB5E5B5B3B62A43A00E9
:1017300000000000000000686F6C6400000000EF13
:101740005E615B3B62A43A0000000000000000758F
:101750006E697400000000F75E6D5B3B62A43A00A6
:1017600000000000000000636F6F7200000000FBCB
:101770005E785B3B62A43A00000000000000006D50
:101780006F6D6F00000000FF5E835B3B62A43A0058
:1017900000000000000000706C616E00000000039B
:1017A0005F8C5B3B62A43A00000000000000007008
:1017B00061746800000000075F975B3B62A43A0019
:1017C0000000000000000064697374000000000B5A
:1017D0005FA25B3B62A43A000000000000000066CC
:1017E000726D6F000000000F5FAD5B3B62A43A00BA
:1017F00000000000000000746F6F6C000000001318
:101800005FB85B3B62A43A000000006D706F006D32
:10181000706F78000000031D60985C3B62A43A0082
:101820000000006D706F006D706F79000000031D87
:1018300060985C3B62A43A000000006D706F006D20
:10184000706F7A000000031D60985C3B62A43A0050
:101850000000006D706F006D706F61000000031D6F
:1018600060985C3B62A43A000000006D706F006DF0
:10187000706F62000000031D60985C3B62A43A0038
:101880000000006D706F006D706F63000000031D3D
:1018900060985C3B62A43A00000000706F730070B7
:1018A0006F73780000000311606E5C3B62A43A0025
:1018B000000000706F7300706F73790000000311F7
:1018C000606E5C3B62A43A00000000706F730070B1
:1018D0006F737A0000000311606E5C3B62A43A00F3
:1018E000000000706F7300706F73610000000311DF
:1018F000606E5C3B62A43A00000000706F73007081
:101900006F73620000000311606E5C3B62A43A00DA
:10191000000000706F7300706F73630000000311AC
:10192000606E5C3B62A43A000000006F6673006F5B
:10193000667378000000032860D15C3B62A43A0023
:101940000000006F6673006F667379000000032863
:1019500060D15C3B62A43A000000006F6673006FC8
:1019600066737A000000032860D15C3B62A43A00F1
:101970000000006F6673006F66736100000003284B
:1019800060D15C3B62A43A000000006F6673006F98
:10199000667362000000032860D15C3B62A43A00D9
:1019A0000000006F6673006F667363000000032819
:1019B00060D15C3B62A43A00000000686F6D006873
:1019C0006F6D6500000000F35E675B0B5EA43A007C
:1019D000000000686F6D00686F6D780000000011F6
:1019E0006093613B62703200000000686F6D0068B8
:1019F0006F6D7900000000116093613B62713200ED
:101A0000000000686F6D00686F6D7A0000000011C3
:101A10006093613B62723200000000686F6D006885
:101A20006F6D6100000000116093613B62733200D2
:101A3000000000686F6D00686F6D620000000011AB
:101A40006093613B62743200000000686F6D006853
:101A50006F6D6300000000116093613B627532009E
:101A6000000000707262007072626500000000B9D0
:101A7000C493613B627632000000007072620070B5
:101A800072627800000003B9C402623B62773200E0
:101A9000000000707262007072627900000003B989
:101AA000C402623B627B3200000000707262007010
:101AB00072627A00000003B9C402623B627F3200A6
:101AC000000000707262007072626100000003B971
:101AD000C402623B628332000000007072620070D8
:101AE00072626200000003B9C402623B6287320086
:101AF000000000707262007072626300000003B93F
:101B0000C402623B628B32000000006A6F67006AA9
:101B10006F677800000000B9C48F61255E953200C0
:101B20000000006A6F67006A6F677900000000B903
:101B3000C48F612C5E9532000000006A6F67006AF6
:101B40006F677A00000000B9C48F61335E95320080
:101B50000000006A6F67006A6F676100000000B9EB
:101B6000C48F613A5E953200000000707772007099
:101B700077723100000000A7BDD7BC3B62A43A00D9
:101B8000000000707772007077723200000000A7CA
:101B9000BDD7BC3B62A43A000000007077720070B1
:101BA00077723300000000A7BDD7BC3B62A43A00A7
:101BB000000000707772007077723400000000A798
:101BC000BDD7BC3B62A43A000000003100000031E8
:101BD0006D61000000030083BD93613D62D1580038
:101BE0000000003100000031736100000003038732
:101BF000BD026286BBDC586666E63F3100000031FC
:101C000074720000000B048CBD0262CBBBE0580074
:101C100000204231000000316D6900000003009B8C
:101C2000BD936110BCD2580000004131000000316A
:101C3000706F00000003009FBD93616362D658007F
:101C40000000003100000031706D0000000300A3AF
:101C5000BD9361C3BCD75800000040320000003281
:101C60006D61000000030083BD93613D62F0580088
:101C700000803F32000000327361000000030387E0
:101C8000BD026286BBFB586666E63F32000000324A
:101C900074720000000B048CBD0262CBBBFF5800C5
:101CA00000204232000000326D6900000003009BFA
:101CB000BD936110BCF158000000413200000032B9
:101CC000706F00000003009FBD93616362F55800D0
:101CD0000000003200000032706D0000000300A31D
:101CE000BD9361C3BCF658000000403300000033D0
:101CF0006D61000000030083BD93613D620F5900D8
:101D000000803F330000003373610000000303874D
:101D1000BD026286BB1A596666E63F330000003397
:101D200074720000000B048CBD0262CBBB1E590014
:101D300000204233000000336D6900000003009B67
:101D4000BD936110BC105900000041330000003306
:101D5000706F00000003009FBD936163621459001F
:101D600000803F3300000033706D0000000300A3CB
:101D7000BD9361C3BC15590000004034000000341D
:101D80006D61000000030083BD93613D622E590028
:101D9000000040340000003473610000000303873A
:101DA000BD026286BB39596666E63F3400000034E6
:101DB00074720000000B048CBD0262CBBB3D596005
:101DC00076074034000000346D6900000003009B7A
:101DD000BD936110BC2F59000080403400000034D6
:101DE000706F00000003009FBD9361636233590070
:101DF0000000003400000034706D0000000300A3F8
:101E0000BD9361C3BC3459000000407800000078E5
:101E1000616D00000003008C5F015D145D2C3100DA
:101E200000803F7800000078766D0000000B00D540
:101E30005F0262126731310050434778000000783A
:101E400066720000000B00D15F026212672D310044
:101E50005043477800000078746E0000000B03DDEB
:101E60005F026212673931000000007800000078DC
:101E7000746D0000000B03D95F02621267353100F8
:101E800000D24378000000786A6D0000000B00E18A
:101E90005F0262825D3D3100401C467800000078A0
:101EA0006A680000000B00E55F0262DA5D41310004
:101EB000409C4678000000786A640000000B04E94A
:101EC0005F0262126749310AD7233C78000000782C
:101ED000736E0000000300F15F936128C050300072
:101EE00000803F780000007873780000000300F560
:101EF0005F936128C0513000000000780000007836
:101F000073760000000B00F95F0262126751310026
:101F1000803B4578000000786C760000000B00FDE7
:101F20005F0262126755310000C8427800000078F5
:101F30006C620000000B03016002621267593100FD
:101F400000204178000000787A620000000B030551
:101F500060026212675D3100004040790000007944
:101F6000616D00000003008C5F015D145D61310054
:101F700000803F7900000079766D0000000B00D5ED
:101F80005F026212676631005043477900000079B2
:101F900066720000000B00D15F02621267623100BE
:101FA0005043477900000079746E0000000B03DD98
:101FB0005F026212676E3100000000790000007954
:101FC000746D0000000B03D95F026212676A310072
:101FD00000D24379000000796A6D0000000B00E137
:101FE0005F0262825D723100401C46790000007918
:101FF0006A680000000B00E55F0262DA5D7631007E
:10200000409C4679000000796A640000000B04E9F6
:102010005F026212677E310AD7233C7900000079A3
:10202000736E0000000300F15F936128C05230001E
:1020300000803F790000007973780000000300F50C
:102040005F936128C05330000000007900000079E0
:1020500073760000000B00F95F02621267863100A0
:10206000803B4579000000796C760000000B00FD94
:102070005F026212678A310000C84279000000796D
:102080006C620000000B030160026212678E310077
:1020900000204179000000797A620000000B0305FE
:1020A00060026212679231000040407A0000007ABC
:1020B000616D00000003008C5F015D145D963100CE
:1020C00000803F7A0000007A766D0000000B00D59A
:1020D0005F026212679B31000096447A0000007A2A
:1020E00066720000000B00D15F0262126797310038
:1020F0000096447A0000007A746E0000000B03DD45
:102100005F02621267A331000000007A0000007ACB
:10211000746D0000000B03D95F026212679F3100EB
:1021200000C8427A0000007A6A6D0000000B00E1EE
:102130005F0262825DA7310000C8427A0000007A27
:102140006A680000000B00E55F0262DA5DAB3100F7
:1021500000FA437A0000007A6A640000000B04E988
:102160005F02621267B3310AD7233C7A0000007A1B
:10217000736E0000000300F15F936128C0543000CB
:102180000000007A0000007A73780000000300F578
:102190005F936128C055300000803F7A0000007ACC
:1021A00073760000000B00F95F02621267BB31001A
:1021B0000096447A0000007A6C760000000B00FD67
:1021C0005F02621267BF310000C8427A0000007AE5
:1021D0006C620000000B03016002621267C33100F1
:1021E0000020417A0000007A7A620000000B0305AB
:1021F0006002621267C73100004040610000006168
:10220000616D00000003008C5F015D145DCB310047
:1022100000803F6100000061766D0000000300D582
:102220005F02622263D03100606A47610000006192
:1022300066720000000300D15F02622263CC3100AD
:10224000803B476100000061746E0000000303DD05
:102250005F02621267D8310000C84361000000616C
:10226000746D0000000303D95F02622263D4310061
:102270000080BF61000000616A6D0000000300E1A2
:102280005F0262825DDC310080BB4661000000615C
:102290006A680000000300E55F0262DA5DE0310079
:1022A00080BB4661000000616A640000000304E92D
:1022B0005F02622263E831CDCCCC3D610000006159
:1022C00072610000000B03ED5F02622263EC3100DB
:1022D00000803F6100000061736E0000000300F1A8
:1022E0005F936128C056300000803F6100000061AC
:1022F00073780000000300F55F936128C057300039
:10230000000000610000006173760000000300F926
:102310005F02622263F0310080BB45610000006112
:102320006C760000000300FD5F02622263F431005E
:10233000007A4461000000616C6200000003030148
:102340006002622263F83100000040610000006119
:102350007A620000000303056002622263FC310020
:102360000000406200000062616D00000003008C0C
:102370005F015D145D003200000000620000006239
:10238000766D0000000300D55F0262226305320013
:10239000006145620000006266720000000300D127
:1023A0005F02622263013200006145620000006248
:1023B000746E0000000303DD5F026212670D3200DD
:1023C0000080BF6200000062746D0000000303D94A
:1023D0005F026222630932000080BF620000006277
:1023E0006A6D0000000300E15F0262825D1132004D
:1023F00000A04162000000626A640000000300E97E
:102400005F026222631D320AD7233C620000006231
:1024100072610000000B03ED5F0262226321320053
:1024200000803F6300000063616D00000003008CCA
:102430005F015D145D353200000000630000006341
:10244000766D0000000300D55F026222633A32001D
:10245000006145630000006366720000000300D164
:102460005F02622263363200006145630000006350
:10247000746E0000000303DD5F02621267423200E7
:102480000080BF6300000063746D0000000303D987
:102490005F026222633E32000080BF63000000637F
:1024A0006A6D0000000300E15F0262825D46320057
:1024B00000A04163000000636A640000000300E9BB
:1024C0005F0262226352320AD7233C63000000633A
:1024D00072610000000B03ED5F026222635632005E
:1024E00000803F703100007031667271000300920D
:1024F000AA02622263AD570000C84270310000702A
:102500003163736C00030096AA02622263B1570024
:10251000007A447031000070316373680003009AE0
:10252000AA02622263B5570000FA447031000070BD
:102530003163706C0003039EAA02622263B95700E4
:1025400000003E703100007031637068000303A228
:10255000AA02622263BD57CDCC4C3E7031000070A0
:102560003177736C000300A6AA02622263C1570090
:10257000007A44703100007031777368000300AA5C
:10258000AA02622263C5570000FA4470310000704D
:102590003177706C000303AEAA02622263C9570050
:1025A00000003E703100007031777068000303B2A4
:1025B000AA02622263CD57CDCC4C3E703100007030
:1025C00031706F66000303B6AA02622263D157CD51
:1025D000CCCC3D673534006735347800000B0309F7
:1025E00060026212679C30000000006735340067AB
:1025F00035347900000B03096002621267A03000D5
:10260000000000673534006735347A00000B030999
:102610006002621267A43000000000673534006772
:1026200035346100000B03096002621267A83000B4
:10263000000000673534006735346200000B030981
:102640006002621267AC300000000067353400673A
:1026500035346300000B03096002621267B030007A
:10266000000000673535006735357800000B030939
:102670006002621267B4300000524367353500676C
:1026800035357900000B03096002621267B830002B
:10269000005243673535006735357A00000B030972
:1026A0006002621267BC30000000006735350067C9
:1026B00035356100000B03096002621267C030000B
:1026C000000000673535006735356200000B0309EF
:1026D0006002621267C43000000000673535006791
:1026E00035356300000B03096002621267C83000D1
:1026F000000000673536006735367800000B0309A7
:102700006002621267CC30000052436735360067C2
:1027100035367900000B03096002621267D0300081
:1027200000A041673536006735367A00000B030993
:102730006002621267D430000020C167353600673E
:1027400035366100000B03096002621267D8300061
:10275000000000673536006735366200000B03095C
:102760006002621267DC30000000006735360067E7
:1027700035366300000B03096002621267E0300027
:10278000000000673537006735377800000B030914
:102790006002621267E430000000006735370067AE
:1027A00035377900000B03096002621267E83000D8
:1027B000000000673537006735377A00000B0309E2
:1027C0006002621267EC3000000000673537006776
:1027D00035376100000B03096002621267F03000B8
:1027E000000000673537006735376200000B0309CA
:1027F0006002621267F4300000000067353700673E
:1028000035376300000B03096002621267F830007D
:10281000000000673538006735387800000B030981
:102820006002621267FC3000000000673538006704
:1028300035387900000B030960026212670031002D
:10284000000000673538006735387A00000B03094F
:1028500060026212670431000000006735380067CB
:1028600035386100000B030960026212670831000D
:10287000000000673538006735386200000B030937
:1028800060026212670C3100000000673538006793
:1028900035386300000B03096002621267103100D3
:1028A000000000673539006735397800000B0309EF
:1028B000600262126714310000000067353900675A
:1028C00035397900000B0309600262126718310084
:1028D000000000673539006735397A00000B0309BD
:1028E00060026212671C3100000000673539006722
:1028F00035396100000B0309600262126720310064
:10290000000000673539006735396200000B0309A4
:1029100060026212672431000000006735390067E9
:1029200035396300000B0309600262126728310029
:10293000000000673932006739327800000103096E
:102940006002623B620C33000000006739320067AE
:1029500039327900000103096002623B62103300E2
:10296000000000673932006739327A00000103093C
:102970006002623B62143300000000673932006776
:1029800039326100000103096002623B62183300C2
:102990000000006739320067393262000001030924
:1029A0006002623B621C330000000067393200673E
:1029B00039326300000103096002623B6220330088
:1029C0000000006732380067323878000001030DDC
:1029D0006002623B62243300000000673238006707
:1029E000323879000001030D6002623B6228330037
:1029F000000000673238006732387A000001030DAA
:102A00006002623B622C33000000006732380067CE
:102A1000323861000001030D6002623B6230330016
:102A20000000006732380067323862000001030D91
:102A30006002623B62343300000000673238006796
:102A4000323863000001030D6002623B62383300DC
:102A50000000006733300067333078000001030D59
:102A60006002623B623C3300000000673330006765
:102A7000333079000001030D6002623B6240330095
:102A8000000000673330006733307A000001030D27
:102A90006002623B6244330000000067333000672D
:102AA000333061000001030D6002623B6248330075
:102AB0000000006733300067333062000001030D0F
:102AC0006002623B624C33000000006733300067F5
:102AD000333063000001030D6002623B625033003B
:102AE0000000006A6964006A69646100000000B95E
:102AF000C4DB61FB62CB3A000000006A6964006AD3
:102B000069646200000000B9C4DB61FB62CF3A0077
:102B10000000006A6964006A69646300000000B92B
:102B2000C4DB61FB62D33A000000006A6964006A9A
:102B300069646400000000B9C4DB61FB62D73A003D
:102B4000000000737973006A61000000000F002B21
:102B50005F026212676A300024F44973797300637C
:102B600074000000000F044A5F026212676E300AB0
:102B7000D7233C73797300736C0000000007006971
:102B80005F93613D627230000000007379730073DF
:102B90007400000000070042C0936122C04530006D
:102BA00000803F737973006D740000000007027F9E
:102BB000BD0262EEBCCD5800000040000000006D78
:102BC00065000000000000BAC450BD50BDA43A002A
:102BD000000000000000006D64000000000000BA6A
:102BE000C428BD28BDA43A000000007379730065B5
:102BF0006A000000000700618393616362BC3A00D1
:102C000000803F737973006A76000000000700655A
:102C1000839361F282613D00008040737973006AA2
:102C200073000000000700698393616362633D00E5
:102C300000803F737973007476000000000700AFD6
:102C4000C593616362405A0000803F7379730071DD
:102C50007600000000070075B09361AD6206580071
:102C6000000000737973007376000000000700CD48
:102C7000AE9361886213580000803F7379730073CC
:102C800069000000000700C9AEB76191AE1458009A
:102C9000007A4373797300656300000000070063E6
:102CA0006793611D68D22900000000737973006585
:102CB00065000000000700676793619D68D32900E5
:102CC0000000007379730065780000000007006B56
:102CD0006793615D68D4290000803F737973007247
:102CE000786D00000007006F6793616362D529006B
:102CF00000803F73797300626175640000040073A3
:102D0000679361C466D0290000A0400000000073F2
:102D100072000000000000C7AE8DAE8FAEA43A0076
:102D20000000000000000071720000000000006957
:102D3000B01CB03B62A43A0000000000000000712B
:102D4000690000000000006DB031B03B62A43A00A1
:102D500000000000000000716F0000000000007122
:102D6000B04DB03B62A43A000000000000000065D6
:102D700072000000000000B9C469AB3B62A43A00D5
:102D8000000000000000007166000000000000B9B3
:102D9000C48F61065EA43A000000000000000072CB
:102DA00078000000000000EEC4A8663B62A43A0070
:102DB000000000000000006D73670000000000BA12
:102DC000C48F613B62A43A00000000000000006371
:102DD0006C656172000000B9C400530053A43A004E
:102DE000000000000000007465737400000000B96A
:102DF000C4637D46C0A43A000000000000000064E7
:102E000065666100000000B9C48E7D3961A43A0096
:102E100000000000000000626F6F7400000000B945
:102E2000C4B97DB47CA43A00000000000000006832
:102E3000656C7000000000B9C4247D3B62A43A00B8
:102E4000000000000000006800000000000000B961
:102E5000C4247D3B62A43A000000007379730067CC
:102E6000706C0000000700175F936188628030007B
:102E70000000007379730067756E00000007001B87
:102E80005F9361636281300000803F7379730067F4
:102E9000636F00000007001F5F93613D627F300099
:102EA00000803F73797300677061000000070023A2
:102EB0005F9361886282300000004073797300671D
:102EC00064690000000700275F936163628330003C
:102ED000000000000000006763000000000000B96F
:102EE000C46B7B7B7BA43A00000000000000006DF7
:102EF00061000000000B046D5F026212677730CD45
:102F0000CCCC3D000000006664000000000300D24D
:102F1000C493616362623D000000007564610075E6
:102F200064613000000300EEC4DB61FB62603A00C4
:102F3000000000756461007564613100000300EEFB
:102F4000C4DB61FB62643A000000007564610075D7
:102F500064613200000300EEC4DB61FB62683A008A
:102F6000000000756461007564613300000300EEC9
:102F7000C4DB61FB626C3A0000000075646200759E
:102F800064623000000300EEC4DB61FB62703A0053
:102F9000000000756462007564623100000300EE99
:102FA000C4DB61FB62743A00000000756462007566
:102FB00064623200000300EEC4DB61FB62783A0019
:102FC000000000756462007564623300000300EE67
:102FD000C4DB61FB627C3A0000000075646300752D
:102FE00064633000000300EEC4DB61FB62803A00E2
:102FF000000000756463007564633100000300EE37
:10300000C4DB61FB62843A000000007564630075F4
:1030100064633200000300EEC4DB61FB62883A00A7
:10302000000000756463007564633300000300EE04
:10303000C4DB61FB628C3A000000007564640075BB
:1030400064643000000300EEC4DB61FB62903A0070
:10305000000000756464007564643100000300EED4
:10306000C4DB61FB62943A00000000756464007583
:1030700064643200000300EEC4DB61FB62983A0036
:10308000000000756464007564643300000300EEA2
:10309000C4DB61FB629C3A000000005F7465005F66
:1030A000746578000000020BC502623B627855002F
:1030B0000000005F7465005F746579000000020B1A
:1030C000C502623B627C55000000005F7465005FD2
:1030D00074657A000000020BC502623B62805500F5
:1030E0000000005F7465005F746561000000020B02
:1030F000C502623B628455000000005F7465005F9A
:10310000746562000000020BC502623B62885500D4
:103110000000005F7465005F746563000000020BCF
:10312000C502623B628C55000000005F7472005F54
:10313000747278000000020BC502623B629D56006B
:103140000000005F7472005F747279000000020B6F
:10315000C502623B62A156000000005F7472005F0E
:1031600074727A000000020BC502623B62A5560031
:103170000000005F7472005F747261000000020B57
:10318000C502623B62A956000000005F7472005FD6
:10319000747262000000020BC502623B62AD560011
:1031A0000000005F7472005F747263000000020B25
:1031B000C502623B62B156000000005F7473005F9D
:1031C000747331000000020BC502623B62085600B6
:1031D0000000005F7073005F707331000000020B2D
:1031E000C502623B621856000000005F6373005F17
:1031F000637331000000020BC502623B6228560077
:103200000000005F6573005F657331000000020B12
:10321000C502623B623856000000005F7873005FB1
:10322000787331000000020BC502623B62685900EE
:103230000000005F6665005F666531000000020BFC
:10324000C502623B624856000000005F7473005F75
:10325000747332000000020BC502623B620C560020
:103260000000005F7073005F707332000000020B9B
:10327000C502623B621C56000000005F6373005F82
:10328000637332000000020BC502623B622C5600E1
:103290000000005F6573005F657332000000020B81
:1032A000C502623B623C56000000005F7873005F1D
:1032B000787332000000020BC502623B6280590045
:1032C0000000005F6665005F666532000000020B6B
:1032D000C502623B624C56000000005F7473005FE1
:1032E000747333000000020BC502623B621056008B
:1032F0000000005F7073005F707333000000020B0A
:10330000C502623B622056000000005F6373005FED
:10331000637333000000020BC502623B623056004B
:103320000000005F6573005F657333000000020BEF
:10333000C502623B624056000000005F7873005F88
:10334000787333000000020BC502623B629859009B
:103350000000005F6665005F666533000000020BD9
:10336000C502623B625056000000005F7473005F4C
:10337000747334000000020BC502623B62145600F5
:103380000000005F7073005F707334000000020B78
:10339000C502623B622456000000005F6373005F59
:1033A000637334000000020BC502623B62345600B6
:1033B0000000005F6573005F657334000000020B5E
:1033C000C502623B624456000000005F7873005FF4
:1033D000787334000000020BC502623B62B05900F2
:1033E0000000005F6665005F666534000000020B48
:1033F000C502623B62545600000000000000005FFE
:1034000064616D00000000B9C47F5E7F5EA43A0075
:10341000000000000000007365303000000200B9B9
:10342000C4B761D2621F58000000000000000073A2
:1034300065303100000200B9C4B761D26221580082
:10344000000000000000007365303200000200B987
:10345000C4B761D26223580000000000000000736E
:1034600065303300000200B9C4B761D2622558004C
:10347000000000000000007365303400000200B955
:10348000C4B761D26227580000000000000000733A
:1034900065303500000200B9C4B761D26229580016
:1034A000000000000000007365303600000200B923
:1034B000C4B761D2622B5800000000000000007306
:1034C00065303700000200B9C4B761D2622D5800E0
:1034D000000000000000007365303800000200B9F1
:1034E000C4B761D2622F58000000000000000073D2
:1034F00065303900000200B9C4B761D262315800AA
:10350000000000000000007365313000000200B9C7
:10351000C4B761D26233580000000000000000739D
:1035200065313100000200B9C4B761D2623558007C
:10353000000000000000007365313200000200B995
:10354000C4B761D262375800000000000000007369
:1035500065313300000200B9C4B761D26239580046
:10356000000000000000007365313400000200B963
:10357000C4B761D2623B5800000000000000007335
:1035800065313500000200B9C4B761D2623D580010
:10359000000000000000007365313600000200B931
:1035A000C4B761D2623F5800000000000000007301
:1035B00065313700000200B9C4B761D262415800DA
:1035C000000000000000007365313800000200B9FF
:1035D000C4B761D2624358000000000000000073CD
:1035E00065313900000200B9C4B761D262455800A4
:1035F000000000000000007365323000000200B9D6
:10360000C4B761D262475800000000000000007398
:1036100065323100000200B9C4B761D26249580076
:10362000000000000000007365323200000200B9A3
:10363000C4B761D2624B5800000000000000007364
:1036400065323300000200B9C4B761D2624D580040
:10365000000000000000007365323400000200B971
:10366000C4B761D2624F5800000000000000007330
:1036700065323500000200B9C4B761D2625158000A
:10368000000000000000007365323600000200B93F
:10369000C4B761D2625358000000000000000073FC
:1036A00065323700000200B9C4B761D262555800D4
:1036B000000000000000007365323800000200B90D
:1036C000C4B761D2625758000000000000000073C8
:1036D00065323900000200B9C4B761D2625958009E
:1036E000000000000000007379730000000000B9C2
:1036F000C4E7645B63A43A000000000000000070AF
:1037000031000000000000B9C4E7645B63A43A0024
:10371000000000000000003100000000000000B9BF
:10372000C4E7645B63A43A000000000000000032BC
:1037300000000000000000B9C4E7645B63A43A0025
:10374000000000000000003300000000000000B98D
:10375000C4E7645B63A43A0000000000000000348A
:1037600000000000000000B9C4E7645B63A43A00F5
:10377000000000000000007800000000000000B918
:10378000C4E7645B63A43A00000000000000007915
:1037900000000000000000B9C4E7645B63A43A00C5
:1037A000000000000000007A00000000000000B9E6
:1037B000C4E7645B63A43A000000000000000061FD
:1037C00000000000000000B9C4E7645B63A43A0095
:1037D000000000000000006200000000000000B9CE
:1037E000C4E7645B63A43A000000000000000063CB
:1037F00000000000000000B9C4E7645B63A43A0065
:10380000000000000000006735340000000000B92F
:10381000C4E7645B63A43A00000000000000006796
:1038200035350000000000B9C4E7645B63A43A00CA
:10383000000000000000006735360000000000B9FD
:10384000C4E7645B63A43A00000000000000006766
:1038500035370000000000B9C4E7645B63A43A0098
:10386000000000000000006735380000000000B9CB
:10387000C4E7645B63A43A00000000000000006736
:1038800035390000000000B9C4E7645B63A43A0066
:10389000000000000000006739320000000000B99D
:1038A000C4E7645B63A43A00000000000000006706
:1038B00032380000000000B9C4E7645B63A43A003A
:1038C000000000000000006733300000000000B975
:1038D000C4E7645B63A43A00000000000000006DD0
:1038E000706F0000000000B9C4E7645B63A43A0095
:1038F00000000000000000706F730000000000B9BD
:10390000C4E7645B63A43A00000000000000006F9D
:1039100066730000000000B9C4E7645B63A43A006A
:1039200000000000000000686F6D0000000000B99A
:10393000C4E7645B63A43A0000000000000000706C
:1039400072620000000000B9C4E7645B63A43A003F
:10395000000000000000007077720000000000B955
:10396000C4E7645B63A43A00000000000000006A42
:103970006F670000000000B9C4E7645B63A43A000D
:10398000000000000000006A69640000000000B947
:10399000C4E7645B63A43A00000000000000007507
:1039A00064610000000000B9C4E7645B63A43A00EE
:1039B000000000000000007564620000000000B913
:1039C000C4E7645B63A43A000000000000000075D7
:1039D00064630000000000B9C4E7645B63A43A00BC
:1039E000000000000000007564640000000000B9E1
:1039F000C4E7645B63A43A00000000000000005FBD
:103A000074650000000000B9C4E7645B63A43A0079
:103A1000000000000000005F74720000000000B9A8
:103A2000C4E7645B63A43A00000000000000005F8C
:103A300074730000000000B9C4E7645B63A43A003B
:103A4000000000000000005F70730000000000B97B
:103A5000C4E7645B63A43A00000000000000005F5C
:103A600063730000000000B9C4E7645B63A43A001C
:103A7000000000000000005F65730000000000B956
:103A8000C4E7645B63A43A00000000000000005F2C
:103A900078730000000000B9C4E7645B63A43A00D7
:103AA000000000000000005F66650000000000B933
:103AB000C4E7645B63A43A00000000000000006DEE
:103AC00000000000000000B9C4D8673B62A43A00BF
:103AD000000000000000007100000000000000B9BC
:103AE000C4BE673B62A43A00000000000000006F03
:103AF00000000000000000B9C4A4673B62A43A00C3
:103B0000000000000000002400000000000000B9D8
:103B1000C4F2673B62A43A00000000486F6D696E12
:103B200067206572726F72202D202563206178698D
:103B3000732073657474696E6773206D6973636F46
:103B40006E666967757265640050726F62696E6750
:103B5000206572726F72202D202563206178697351
:103B60002063616E6E6F74206D6F76652064757270
:103B7000696E672070726F62696E67005B69645D71
:103B8000202054696E7947204944253330730A0058
:103B90005B68765D2020686172647761726520766B
:103BA000657273696F6E2531362E32660A005B6866
:103BB000705D2020686172647761726520706C614D
:103BC00074666F726D2531352E32660A005B66763B
:103BD0005D20206669726D7761726520766572730B
:103BE000696F6E2531362E32660A005B66625D2093
:103BF000206669726D77617265206275696C6425F3
:103C000031382E32660A00456E7465722024626F68
:103C10006F743D3120746F20656E74657220746816
:103C20006520626F6F74206C6F616465722E0A008C
:103C30000A0A0A2323232054696E794720424F4FF2
:103C400054204C4F414445522048656C702023233A
:103C5000230A00456E7465722024646566613D31F7
:103C600020746F20726573657420746865207379A1
:103C70007374656D20746F20746865206661637469
:103C80006F72792064656661756C742076616C75FD
:103C900065732E0A546869732077696C6C206F769F
:103CA0006572777269746520616E79206368616EF0
:103CB00067657320796F752068617665206D616432
:103CC000652E0A000A0A0A2323232054696E7947C5
:103CD00020524553544F52452044454641554C547B
:103CE000532048656C70202323230A00496E766FA9
:103CF0006B652073656C662074657374206279202F
:103D0000656E746572696E672024746573743D4EC8
:103D1000207768657265204E206973206F6E65207C
:103D20006F663A0A202024746573743D3120207335
:103D30006D6F6B6520746573740A2020247465733D
:103D4000743D322020686F6D696E672074657374EE
:103D500020202028796F75206D7573742074726926
:103D60007020686F6D696E6720737769746368652A
:103D700073290A202024746573743D3320207371E5
:103D8000756172652074657374202020286120732A
:103D90006572696573206F662073717561726573F2
:103DA000290A202024746573743D342020617263D5
:103DB000207465737420202020202028736F6D6587
:103DC000206C6172676520636972636C6573290A90
:103DD000202024746573743D3520206477656C6CF5
:103DE000207465737420202020286D6F7665732001
:103DF0007370616365642062792031207365636F3D
:103E00006E64206477656C6C73290A2020247465C5
:103E100073743D36202066656564686F6C64207439
:103E20006573742028656E746572202120616E644C
:103E3000207E20746F20686F6C6420616E64207235
:103E40006573746172742C20726573706563746934
:103E500076656C79290A202024746573743D3720B7
:103E6000204D20636F64657320746573742020286F
:103E70004D20636F64657320696E7465726D696E41
:103E8000676C65642077697468206D6F7665732947
:103E90000A202024746573743D3820204A534F4E05
:103EA00020746573742020202020286D6F74696F42
:103EB0006E20746573742072756E207573696E67F9
:103EC000204A534F4E20636F6D6D616E6473290AF3
:103ED000202024746573743D392020696E766572E4
:103EE00073652074696D6520746573740A202024DD
:103EF000746573743D313020726F74617279206D16
:103F00006F74696F6E20746573740A202024746561
:103F100073743D313120736D616C6C206D6F76650B
:103F20007320746573740A202024746573743D31A2
:103F30003220736C6F77206D6F76657320746573B4
:103F4000740A202024746573743D313320636F6FCD
:103F50007264696E6174652073797374656D206F26
:103F60006666736574207465737420284739322C33
:103F7000204735342D473539290A0A54657374733F
:103F800020617373756D6520612063656E74657261
:103F90006564205859206F726967696E20616E648C
:103FA000206174206C656173742038306D6D2063FE
:103FB0006C656172616E636520696E20616C6C2056
:103FC000646972656374696F6E730A5465737473A0
:103FD00020617373756D65205A2068617320617468
:103FE000206C656173742034306D6D20706F73695F
:103FF000697469766520636C656172616E63650AD8
:104000005465737473207374617274207769746873
:104010002061204730205830205930205A30206D00
:104020006F76650A486F6D696E67206973207468E2
:104030006520657863657074696F6E2E204E6F2001
:10404000696E697469616C20706F736974696F6EF1
:10405000206F7220636C656172616E6365206973A5
:1040600020617373756D65640A000A0A0A232323AD
:104070002054696E79472053454C4620544553548B
:104080002048656C70202323230A00456163682063
:104090002420636F6D6D616E642061626F766520B0
:1040A000616C736F20646973706C617973207468DC
:1040B0006520746F6B656E20666F72206561636842
:1040C0002073657474696E6720696E205B205D20C3
:1040D000627261636B6574730A546F2076696577E9
:1040E0002073657474696E677320656E74657220E1
:1040F0006120746F6B656E3A0A0A2020243C746F4D
:104100006B656E3E0A0A466F72206578616D706C51
:1041100065202479667220746F20646973706C6105
:1041200079207468652059206D6178206665656422
:1041300020726174650A0A546F2075706461746539
:104140002073657474696E677320656E7465722080
:10415000746F6B656E20657175616C732076616C30
:1041600075653A0A0A2020243C746F6B656E3E3DEB
:104170003C76616C75653E0A0A466F72206578610F
:104180006D706C6520247966723D38303020746F14
:1041900020736574207468652059206D61782066ED
:1041A000656564207261746520746F20383030203A
:1041B0006D6D2F6D696E7574650A466F7220636F41
:1041C0006E66696775726174696F6E20646574618B
:1041D000696C73207365653A2068747470733A2F44
:1041E0002F6769746875622E636F6D2F73796E74B3
:1041F0006865746F732F54696E79472F77696B699F
:104200002F54696E79472D436F6E666967757261C9
:1042100074696F6E0A00546865736520636F6D6D15
:10422000616E6473206172652061637469766520D4
:10423000666F7220636F6E66696775726174696F0D
:104240006E3A0A2020247379732053686F772073A5
:10425000797374656D202867656E6572616C2920BD
:1042600073657474696E67730A20202431202020DE
:1042700053686F77206D6F746F722031207365748F
:1042800074696E677320286F722077686174657631
:104290006572206D6F746F7220796F752077616E13
:1042A0007420312C322C332C34290A2020247820FD
:1042B000202053686F7720582061786973207365D8
:1042C0007474696E677320286F72207768617465F3
:1042D000766572206178697320796F752077616ED9
:1042E0007420782C792C7A2C612C622C63290A207A
:1042F00020246D20202053686F7720616C6C206D26
:104300006F746F722073657474696E67730A20200E
:10431000247120202053686F7720616C6C206178B5
:1043200069732073657474696E67730A2020246F43
:1043300020202053686F7720616C6C206F66667355
:1043400065742073657474696E67730A2020242471
:1043500020202053686F7720616C6C207365747423
:10436000696E67730A2020246820202053686F77C5
:1043700020746869732068656C702073637265656A
:104380006E0A0A000A0A0A2323232054696E794719
:1043900020434F4E46494755524154494F4E2048BD
:1043A000656C70202323230A000A466F722064651F
:1043B0007461696C65642054696E794720696E6622
:1043C0006F207365653A2068747470733A2F2F6795
:1043D00069746875622E636F6D2F73796E7468658A
:1043E000746F732F54696E79472F77696B692F0A41
:1043F000466F7220746865206C6174657374206602
:1044000069726D77617265207365653A20687474AE
:1044100070733A2F2F6769746875622E636F6D2F02
:1044200073796E746865746F732F54696E79470A77
:10443000506C65617365206C6F6720616E792069CF
:10444000737375657320617420687474703A2F2FCC
:104450007777772E73796E746865746F732E636FD8
:104460006D2F666F72756D730A486176652066758B
:104470006E0A000A4E6F74653A2054696E794720BF
:1044800067656E657261746573206175746F6D61C7
:1044900074696320737461747573207265706F72D0
:1044A00074732062792064656661756C740A54685F
:1044B00069732063616E2062652064697361626C58
:1044C000656420627920656E746572696E67202468
:1044D00073763D300A536565207468652077696B93
:1044E000692062656C6F7720666F72206D6F7265F0
:1044F0002064657461696C732E0A00546865736585
:1045000020636F6D6D616E647320617265206163FD
:10451000746976652066726F6D2074686520636FBC
:104520006D6D616E64206C696E653A0A205E78205C
:10453000202020202020202020202020526573656C
:10454000742028636F6E74726F6C207829202D2080
:10455000736F6674776172652072657365740A2083
:10456000203F202020202020202020202020204DFF
:10457000616368696E6520706F736974696F6E201E
:10458000616E642067636F6465206D6F64656C2085
:1045900073746174650A20202420202020202020AC
:1045A00020202020202053686F7720616E642073C4
:1045B000657420636F6E66696775726174696F6E8A
:1045C0002073657474696E67730A2020212020208F
:1045D0002020202020202020202046656564686F50
:1045E0006C64202D2073746F70206D6F74696F6E12
:1045F00020776974686F7574206C6F73696E6720BB
:10460000706F736974696F6E0A20207E20202020ED
:104610002020202020202020204379636C65205317
:1046200074617274202D20726573746172742066D7
:10463000726F6D2066656564686F6C640A2020681F
:104640002020202020202020202020202053686FA0
:104650007720746869732068656C70207363726575
:10466000656E0A2020246820202020202020202081
:1046700020202053686F7720636F6E6669677572BC
:104680006174696F6E2068656C7020736372656514
:104690006E0A20202474657374202020202020209E
:1046A00020204C6973742073656C662D7465737477
:1046B000730A202024746573743D4E20202020202E
:1046C000202052756E2073656C662D74657374209E
:1046D0004E0A202024686F6D653D31202020202067
:1046E000202052756E206120686F6D696E672063AF
:1046F00079636C650A202024646566613D31202061
:104700002020202020526573746F726520616C6CCC
:104710002073657474696E677320746F20226661FC
:1047200063746F7279222064656661756C74730AB4
:10473000000A0A0A2323232054696E79472048651A
:104740006C70202323230A005B6A735D20206A7348
:104750006F6E2073657269616C697A652073747914
:104760006C65253964205B303D72656C61786564E9
:104770002C313D7374726963745D0A005B6A765D07
:1047800020206A736F6E20766572626F7369747928
:1047900025313564205B303D73696C656E742C3156
:1047A0003D666F6F7465722C323D6D657373616722
:1047B00065732C333D636F6E666967732C343D6C93
:1047C000696E656E756D2C353D766572626F7365C9
:1047D0005D0A005B656A5D2020656E61626C652024
:1047E0006A736F6E206D6F646525313364205B30B2
:1047F0003D746578742C313D4A534F4E5D0A000C70
:10480000590659FF58FA58F158E658DB58CF58C3A3
:1048100058B5589E588F5882587658625855584007
:10482000582C582958265817580258ED57DE57CE9D
:1048300057BC57A55788576B5752573C572B57199A
:10484000570C57FA56E056DD56DA56D756D456D19D
:1048500056CE56CB56C856C556C256BF56BC56B98C
:1048600056B656B356B056AD56AA56A756A456A13C
:10487000569E569B569856955692568F568C5689EC
:10488000568656835680567D567A5677567456719C
:10489000566E566B566856655662565F565C56594C
:1048A000565656535650564D564A564756445641FC
:1048B000563E561A56FA55E055C655AC5588556BB6
:1048C0005553553D552355FF54E254D054B0549997
:1048D0005480545E54455427540B54F353E153C34E
:1048E00053AE53AA53A653A2539E539A5396539230
:1048F000538E538A53865382537E537A5376537220
:10490000536E5354533A5327530B53F952E252C147
:1049100052B0529052705256523C522552F251C5EA
:1049200051A55183515D5136511A51FB50E150C789
:1049300050A2507950615036500A50D44F9F4F8D3D
:104940004F7B4F6C4F594F404F1E4F0C4FFA4EE864
:104950004ED64EC44EB24EA04E8E4E7C4E6A4E582F
:104960004E464E344E224E1E4E1A4E164E124E0ECD
:104970004E0A4E064E024EFE4DFA4DF64DF24DEEEB
:104980004DEA4DE64DE24DDE4DDA4DD64DD24DBEEF
:104990004DA04D844D594D344D0F4D0B4D074D03DA
:1049A0004DFF4CFB4CF74CF34CEF4CEB4CE74CE31E
:1049B0004CDF4CDB4CD74CC34CA74C8B4C6F4C534F
:1049C0004C374C1B4CFF4BE34BC74BAB4B8F4B73E4
:1049D0004B6F4B6B4B674B634B5F4B5B4B574B4387
:1049E0004B1B4BF44ACE4AA14A7B4A4E4A4A4A469E
:1049F0004A424A2F4A0E4AF9494A6F6767696E6709
:104A0000206379636C65206661696C65640050722F
:104A10006F626520656E64706F696E7420697320C3
:104A20007374617274696E6720706F696E74005080
:104A3000726F6265206379636C65206661696C657D
:104A40006400323439003234380032343700486F71
:104A50006D696E67204572726F72202D20486F6DF0
:104A6000696E67207377697463686573206D697315
:104A7000636F6E6669677572656400486F6D696E15
:104A800067204572726F72202D204E6567617469D0
:104A90007665206C61746368206261636B6F666623
:104AA00000486F6D696E67204572726F72202D200D
:104AB00054726176656C206D696E2026206D617878
:104AC00020617265207468652073616D6500486FB0
:104AD0006D696E67204572726F72202D204C617473
:104AE00063682076656C6F63697479206973207AD6
:104AF00065726F00486F6D696E67204572726F72E4
:104B0000202D205365617263682076656C6F636940
:104B10007479206973207A65726F00486F6D696ED1
:104B200067204572726F72202D20426164206F727F
:104B3000206E6F20617869732073706563696669A0
:104B4000656400486F6D696E67206379636C6520EA
:104B50006661696C65640032333900323338003283
:104B600033370032333600323335003233340032DB
:104B7000333300536F6674206C696D6974206578F7
:104B8000636565646564202D2043206D6178005362
:104B90006F6674206C696D697420657863656564FF
:104BA0006564202D2043206D696E00536F6674206C
:104BB0006C696D6974206578636565646564202D32
:104BC0002042206D617800536F6674206C696D69B6
:104BD00074206578636565646564202D2042206DCE
:104BE000696E00536F6674206C696D697420657816
:104BF000636565646564202D2041206D61780053F4
:104C00006F6674206C696D6974206578636565648E
:104C10006564202D2041206D696E00536F667420FD
:104C20006C696D6974206578636565646564202DC1
:104C3000205A206D617800536F6674206C696D692D
:104C400074206578636565646564202D205A206D45
:104C5000696E00536F6674206C696D6974206578A5
:104C6000636565646564202D2059206D617800536B
:104C70006F6674206C696D6974206578636565641E
:104C80006564202D2059206D696E00536F66742075
:104C90006C696D6974206578636565646564202D51
:104CA0002058206D617800536F6674206C696D69BF
:104CB00074206578636565646564202D2058206DD7
:104CC000696E00536F6674206C696D697420657835
:104CD0006365656465640032313900323138003211
:104CE0003137003231360032313500323134003262
:104CF0003133003231320032313100323130003262
:104D0000303900323038003230370032303600541B
:104D1000726170657A6F696420706C616E6E657225
:104D2000206661696C656420746F20636F6E7665C0
:104D3000726765004C696D69742073776974636884
:104D400020686974202D2053687574646F776E2015
:104D50006F63637572726564004D616368696E6547
:104D600020697320616C61726D6564202D20436F32
:104D70006D6D616E64206E6F742070726F63657309
:104D8000736564004D6F7665206C6573732074687D
:104D9000616E206D696E696D756D2074696D650059
:104DA0004D6F7665206C657373207468616E206D3D
:104DB000696E696D756D206C656E67746800476516
:104DC0006E657269632054696E7947206572726FEF
:104DD0007200313939003139380031393700313911
:104DE0003600313935003139340031393300313949
:104DF0003200313931003139300031383900313841
:104E00003800313837003138360031383500313824
:104E10003400313833003138320031383100313824
:104E200030005420776F726420697320696E766158
:104E30006C6964005420776F7264206973206D6917
:104E40007373696E67005220776F726420697320F4
:104E5000696E76616C6964005220776F72642069B4
:104E600073206D697373696E67005120776F726488
:104E700020697320696E76616C6964005120776FD8
:104E80007264206973206D697373696E67004C20CA
:104E9000776F726420697320696E76616C69640053
:104EA0004C20776F7264206973206D697373696E2B
:104EB00067004820776F726420697320696E76619D
:104EC0006C6964004820776F7264206973206D6993
:104ED0007373696E67004520776F72642069732071
:104EE000696E76616C6964004520776F7264206931
:104EF00073206D697373696E67004420776F726405
:104F000020697320696E76616C6964004420776F54
:104F10007264206973206D697373696E6700502035
:104F2000776F7264206973206E6F742061207661E0
:104F30006C696420746F6F6C206E756D62657200B1
:104F40005020776F7264206973206E6F7420616ED9
:104F500020696E7465676572005020776F726420F7
:104F60006973206E65676174697665005020776F9C
:104F70007264206973207A65726F005020776F72B7
:104F80006420697320696E76616C696400502077D3
:104F90006F7264206973206D697373696E67004175
:104FA00072632073706563696669636174696F6EAB
:104FB000206572726F72202D20656E64706F696E4D
:104FC00074206973207374617274696E6720706FE6
:104FD000696E74004172632073706563696669630A
:104FE0006174696F6E206572726F72202D2072611C
:104FF0006469757320617263206F7574206F662019
:10500000746F6C6572616E636500417263207370CA
:105010006563696669636174696F6E206572726F3A
:1050200072202D206D697373696E67206F666673D9
:105030006574287329004172632073706563696623
:1050400069636174696F6E206572726F72202D20C2
:105050006D697373696E6720617869732865732958
:105060000041726320737065636966696361746986
:105070006F6E206572726F72005370696E646C653A
:10508000206D757374206265207475726E696E6729
:1050900020666F72207468697320636F6D6D616E36
:1050A00064005370696E646C65206D757374206262
:1050B00065206F666620666F72207468697320636E
:1050C0006F6D6D616E64005370696E646C65205322
:1050D00020776F726420697320696E76616C6964F1
:1050E000005370696E646C65205320776F72642082
:1050F0006973206D697373696E67005370696E64BC
:105100006C652073706565642065786365656465AA
:1051100064206D6178696D756D005370696E646CA3
:10512000652073706565642062656C6F77206D69BA
:105130006E696D756D0050726F6772616D6D65643B
:1051400020706F696E742073616D652061732063D8
:10515000757272656E7420706F696E740043757439
:1051600074657220636F6D70656E736174696F6EC4
:105170002063616E6E6F7420626520656E61626C83
:105180006564005265717565737465642076656C3D
:105190006F636974792065786365656473206C69F1
:1051A0006D697473004730206F72204731206D7530
:1051B00073742062652061637469766520666F721E
:1051C0002047353300526F746172792061786573BE
:1051D0002063616E6E6F7420626520757365642054
:1051E00077697468207468697320636F6D6D616E90
:1051F0006400496E76657273652074696D65206D13
:105200006F64652063616E6E6F74206265207573D4
:1052100065642077697468207468697320636F6DB2
:105220006D616E64004665656472617465206E6FC1
:1052300074207370656369666965640053656C65A5
:105240006374656420706C616E6520697320696E9B
:1052500076616C69640053656C6563746564207085
:105260006C616E65206973206D697373696E670088
:10527000417869732074617267657420706F736917
:1052800074696F6E20697320696E76616C69640061
:10529000417869732074617267657420706F7369F7
:1052A00074696F6E206973206D697373696E67002E
:1052B000417869732069732064697361626C656405
:1052C000004178697320697320696E76616C696446
:1052D00020666F72207468697320636F6D6D616EF4
:1052E0006400417869732063616E6E6F742062653B
:1052F0002070726573656E74004178697320776FF2
:105300007264206D697373696E670047636F6465CB
:10531000206D6F64616C2067726F75702076696FA5
:105320006C6174696F6E004D20636F646520756EEB
:10533000737570706F727465640047636F64652085
:10534000636F6D6D616E6420756E737570706F72D2
:105350007465640047656E657269632047636F64B6
:105360006520696E707574206572726F72003132DB
:1053700039003132380031323700313236003132C3
:1053800035003132340031323300313232003132C3
:1053900031003132300031313900313138003131B2
:1053A00037003131360031313500313134004A5364
:1053B0004F4E20737472696E6720746F6F206C6F2C
:1053C0006E67004A534F4E20696E70757420686195
:1053D0007320746F6F206D616E79207061697273D4
:1053E000004A534F4E2073796E7461782065727253
:1053F0006F7200496E7075742076616C75652072ED
:10540000616E6765206572726F7200496E707574A7
:105410002065786365656473206D6178696D756D6D
:105420002076616C756500496E707574206C6573CB
:1054300073207468616E206D696E696D756D20767C
:10544000616C756500496E7075742065786365657B
:105450006473206D6178206C656E67746800436FBB
:105460006D6D616E64206E6F74206163636570742E
:10547000656420617420746869732074696D6500C7
:10548000506172616D657465722063616E6E6F74D8
:10549000206265207265616400506172616D65749F
:1054A000657220697320726561642D6F6E6C79007E
:1054B000556E737570706F72746564206E756D6271
:1054C0006572206F72204A534F4E207479706500C8
:1054D000426164206E756D62657220666F726D61E7
:1054E0007400496E76616C6964206F72206D616C26
:1054F000666F726D656420636F6D6D616E640055DB
:105500006E7265636F676E697A656420636F6D6D37
:10551000616E64206F7220636F6E666967206E61D2
:105520006D650047656E65726963206173736572AE
:1055300074696F6E206661696C757265004D656D8A
:105540006F7279206661756C74206465746563742C
:10555000656400537461636B206F766572666C6F6F
:105560007720646574656374656400436F6E74725C
:105570006F6C6C657220617373657274696F6E20F5
:105580006661696C7572650043616E6F6E69636117
:105590006C206D616368696E6520617373657274F8
:1055A000696F6E206661696C75726500506C616E22
:1055B0006E657220617373657274696F6E206661C7
:1055C000696C7572650053746570706572206173E3
:1055D00073657274696F6E206661696C75726500BF
:1055E000456E636F64657220617373657274696F71
:1055F0006E206661696C75726500494F2073756233
:105600002D73797374656D20617373657274696F3E
:105610006E206661696C75726500436F6E666967BE
:10562000207375622D73797374656D206173736572
:105630007274696F6E206661696C757265003839C5
:105640000038380038370038360038350038340034
:1056500038330038320038310038300037390037FD
:1056600038003737003736003735003734003733E6
:105670000037320037310037300036390036380015
:1056800036370036360036350036340036330036CD
:1056900032003631003630003539003538003537C4
:1056A00000353600353500353400353300353200ED
:1056B00035310035300034390034380034370034A7
:1056C00036003435003434003433003432003431A1
:1056D00000343000333900333800333700333600BC
:1056E00042616420737461747573207265706F72A7
:1056F000742073657474696E6700506572736973A2
:1057000074656E6365206572726F7200466C6F61BE
:1057100074206973204E414E00466C6F617420699D
:105720007320696E66696E697465004D6F766520D9
:1057300074696D65206973204E414E004D6F76652A
:105740002074696D6520697320696E66696E69747D
:10575000650047656E65726963206578636570747E
:10576000696F6E207265706F7274004661696C6556
:105770006420746F2067657420706C616E6E657252
:10578000206275666665720053797374656D206179
:105790006C61726D202D207368757474696E67205A
:1057A000646F776E00496E697469616C697A6174BF
:1057B000696F6E206661696C75726500526561641F
:1057C0002D6F6E6C79206164647265737300496E2D
:1057D00076616C6964204164647265737300446926
:1057E00076696465206279207A65726F00466C6F15
:1057F0006174696E6720706F696E74206572726F74
:105800007200496E7465726E616C2072616E6765BC
:10581000206572726F7200496E7465726E616C20E1
:105820006572726F720031390031380046756E63EF
:1058300074696F6E206973207374756262656400A9
:10584000456E746572696E6720626F6F74206C6F4D
:105850006164657200496E697469616C697A696E28
:1058600067004275666665722066756C6C202D2037
:10587000666174616C004275666665722066756C5F
:105880006C0042756666657220656D707479004EB5
:105890006F207375636820646576696365004D6188
:1058A000782066696C652073697A65206578636520
:1058B000656465640046696C65206E6F74206F7066
:1058C000656E00456E64206F662066696C650045F4
:1058D0006E64206F66206C696E650048617264209A
:1058E0007265736574005465726D696E6174656488
:1058F00000436F6D706C657465004E6F6F7000458E
:10590000616761696E004572726F72004F4B005B98
:105910007031706F665D2070776D2070686173659F
:10592000206F66662020202531352E3366205B30BF
:105930002E2E315D0A005B70317770685D207077C4
:105940006D20636377207068617365206869253115
:10595000352E3366205B302E2E315D0A005B7031B0
:1059600077706C5D2070776D20636377207068615D
:105970007365206C6F2531352E3366205B302E2EFB
:10598000315D0A005B70317773685D2070776D2040
:105990006363772073706565642068692531352EEF
:1059A00030662052504D0A005B703177736C5D2079
:1059B00070776D20636377207370656564206C6F0A
:1059C0002531352E30662052504D0A005B70316310
:1059D00070685D2070776D206377207068617365F3
:1059E000206869202531352E3366205B302E2E311C
:1059F0005D0A005B703163706C5D2070776D2063B1
:105A000077207068617365206C6F202531352E33E7
:105A100066205B302E2E315D0A005B703163736847
:105A20005D2070776D2063772073706565642068F2
:105A300069202531352E30662052504D0A005B70AA
:105A40003163736C5D2070776D20637720737065B0
:105A50006564206C6F202531352E30662052504D04
:105A60000A005B70316672715D2070776D2066721E
:105A7000657175656E63792020202531352E30667D
:105A800020487A0A0053595354454D205245414409
:105A900059004C6F6164696E6720636F6E66696759
:105AA000732066726F6D20454550524F4D00496E10
:105AB000697469616C697A696E6720636F6E666983
:105AC000677320746F2053686170656F6B6F32204D
:105AD0003530306D6D2070726F66696C65007B22A9
:105AE0006572223A7B226662223A25302E32662C7B
:105AF000227374223A25642C226D7367223A222580
:105B000073227D7D0A007B65723A7B66623A25309E
:105B10002E32662C73743A25642C6D73673A2225F5
:105B200073227D7D0A005B71765D2020717565753D
:105B300065207265706F727420766572626F73692A
:105B40007479253764205B303D6F66662C313D7378
:105B5000696E676C652C323D747269706C655D0AA4
:105B600000716F3A25640A0071693A25640A007170
:105B7000723A25640A005B73765D20207374617449
:105B80007573207265706F727420766572626F73C0
:105B9000697479253664205B303D6F66662C313D33
:105BA00066696C74657265642C323D766572626FED
:105BB00073655D0A005B73695D20207374617475A1
:105BC0007320696E74657276616C2531342E30668F
:105BD000206D730A004D6F746F7220256320706F03
:105BE00077657220656E61626C65642073746174A0
:105BF000653A25322E30660A005B257325735D20D9
:105C00006D257320706F776572206D616E616765B9
:105C10006D656E7425313064205B303D646973615D
:105C2000626C65642C313D616C77617973206F6EB5
:105C30002C323D696E206379636C652C333D776847
:105C4000656E206D6F76696E675D0A005B25732552
:105C5000735D206D257320706F6C61726974792596
:105C6000313864205B303D6E6F726D616C2C313D5C
:105C7000726576657273655D0A005B257325735DD9
:105C8000206D2573206D6963726F73746570732561
:105C9000313664205B312C322C342C385D0A005BA9
:105CA000257325735D206D25732074726176656C94
:105CB00020706572207265766F6C7574696F6E25E1
:105CC00031302E346625730A005B257325735D2001
:105CD0006D2573207374657020616E676C65253265
:105CE000302E336625730A005B257325735D206DA6
:105CF0002573206D617020746F2061786973253180
:105D00003564205B303D582C313D592C323D5A2EA4
:105D10002E2E5D0A005B6D745D20206D6F746F72B6
:105D20002069646C652074696D656F757425313404
:105D30002E3266205365630A00485D445D3F5D2056
:105D400064656700206D6D0020696E005B73745D93
:105D50002020737769746368207479706525313801
:105D600064205B303D4E4F2C313D4E435D0A005464
:105D700065737420232564206E6F7420666F756EC2
:105D8000640A004E362047393220583735205930C2
:105D9000205A300A4E3720463530302E300A4E38E1
:105DA00020473159302E3239315A2D322E3139387F
:105DB0000A4E39205837342E37363759302E303581
:105DC000385A2D322E3335350A4E3130205837347B
:105DD0002E373039592D302E3030305A2D322E3367
:105DE00037310A4E3131205837342E3532395A2D59
:105DF000322E3236340A4E3132205837342E363372
:105E00003459302E3130355A2D322E3331390A4E35
:105E10003133205837342E38343359302E3331341F
:105E20005A2D322E3138330A4E3134205837352E20
:105E300030303059302E3437315A2D322E313236FF
:105E40000A4E31352059302E3635305A2D322E310A
:105E500030300A4E3136205837342E3738335930E7
:105E60002E3433345A2D322E3133310A4E3137200D
:105E70005837342E35363659302E3231375A2D3286
:105E80002E3234340A4E3138205837342E333530E0
:105E9000592D302E3030305A2D322E3138320A4EB4
:105EA0003139205837342E3137305A2D322E313493
:105EB000340A4E3230205837342E34323959302E8D
:105EC0003235395A2D322E3136350A4E323120587C
:105ED00037342E35333359302E3336335A2D322E54
:105EE0003139310A4E3232205837342E363839594A
:105EF000302E3531395A2D322E3131340A4E32336B
:105F0000205837342E38343459302E3637345A2D01
:105F1000322E3039360A4E3234205837352E303052
:105F20003059302E3833305A2D322E3131340A4E1A
:105F300032352059312E3031305A2D322E31343411
:105F40000A4E3236205837342E37383759302E37EC
:105F500039375A2D322E3039380A4E3237205837D9
:105F6000342E36323859302E3633385A2D322E31BF
:105F700030380A4E3238205837342E3436395930BA
:105F80002E3437385A2D322E3135370A4E323920D9
:105F90005837342E33303959302E3331395A2D3267
:105FA0002E3131300A4E3330205837342E303434CD
:105FB00059302E3035335A2D322E3130380A4E3387
:105FC00031205837332E39393059302E3030305A4D
:105FD0002D322E3037370A4E3332205837332E3891
:105FE00031315A2D312E3934370A4E333320583758
:105FF000332E39373359302E3136325A2D322E3036
:1060000037390A4E3334205837342E32343359302E
:106010002E3433325A2D322E3038340A4E33352056
:106020005837342E34353959302E3634395A2D32CA
:106030002E3135370A4E3336205837342E36373620
:1060400059302E3836355A2D322E3130390A4E33EA
:1060500037205837342E38333859312E3032375AAA
:106060002D322E3131310A4E3338205837352E300B
:10607000303059312E3138395A2D322E3136300ADE
:106080004E33392059312E3336395A2D322E31398B
:10609000340A4E3430205837342E38343259312EA9
:1060A0003231315A2D322E3133340A4E34312058A8
:1060B00037342E36383459312E3035335A2D322E6E
:1060C0003132300A4E3432205837342E343231597E
:1060D000302E3739305A2D322E3137360A4E34337E
:1060E000205837342E33313659302E3638345A2D25
:1060F000322E3133370A4E3434205837342E31356E
:106100003859302E3532365A2D322E3037370A4E26
:106110003435205837332E39343759302E33313611
:106120005A2D322E3036370A4E3436205837332E19
:1061300038393459302E3236335A2D322E303436E7
:106140000A4E3437205837332E37333759302E31F3
:1061500030355A2D312E3931380A4E3438205837DF
:10616000332E36333159302E3030305A2D312E38CF
:1061700037320A4E3439205837332E3435325A2DBF
:10618000312E3831350A4E3530205837332E3636D9
:106190003559302E3231345A2D312E3931340A4EA0
:1061A0003531205837332E38323559302E33373485
:1061B0005A2D322E3032380A4E3532205837332E8F
:1061C00038373959302E3432375A2D322E3037364F
:1061D0000A4E3533205837342E30393259302E3666
:1061E00034315A2D322E3039340A4E353420583756
:1061F000342E33303659302E3835345A2D322E3134
:1062000039320A4E3535205837342E353139593127
:106210002E3036385A2D322E3134310A4E35362052
:106220005837342E37333359312E3238315A2D32D4
:106230002E3134330A4E3537205837342E38343027
:1062400059312E3338385A2D322E3137340A4E35E3
:1062500038205837342E38393359312E3434325AA5
:106260002D322E3136390A4E3539205837352E30F9
:10627000303059312E3534385A2D322E3132310AE0
:106280004E36302059312E3732385A2D322E303793
:10629000360A4E3631205837342E38343359312EA1
:1062A0003537315A2D322E3133300A4E363220589E
:1062B00037342E37333859312E3436365A2D322E64
:1062C0003139350A4E3633205837342E3437365963
:1062D000312E3230345A2D322E3134370A4E363484
:1062E000205837342E32313559302E3934335A2D27
:1062F000322E3230320A4E3635205837332E39306E
:106300003059302E3632385A2D322E3130310A4E35
:106310003636205837332E38343859302E35373604
:106320005A2D322E3039360A4E3637205837332E12
:1063300035383659302E3331345A2D312E393133E8
:106340000A4E3638205837332E33373759302E31EE
:1063500030355A2D312E3830380A4E3639205837DC
:10636000332E32373259302E3030305A2D312E37CD
:1063700038370A4E3730205837332E3138325A2DBD
:10638000312E3738370A4E3731205837332E3039CF
:10639000325A2D312E3735300A4E373220583733A6
:1063A0002E34313059302E3331385A2D312E383683
:1063B000380A4E3733205837332E37383159302E7C
:1063C0003638395A2D322E3038360A4E3734205866
:1063D00037342E30393959312E3030375A2D322E4C
:1063E0003232340A4E3735205837342E3230355950
:1063F000312E3131335A2D322E3231310A4E373669
:10640000205837342E33363459312E3237325A2D04
:10641000322E3137360A4E3737205837342E36323F
:106420003959312E3533375A2D322E3139310A4E02
:106430003738205837342E36383259312E353930E6
:106440005A2D322E3137370A4E3739205837342EED
:1064500038393459312E3830325A2D322E303636C2
:106460000A4E3830205837352E30303059312E39D9
:1064700030385A2D322E3034360A4E3831205932C7
:106480002E3038375A2D322E3035310A4E383220E0
:106490005837342E38333959312E3932375A2D3254
:1064A0002E3036320A4E3833205837342E363739AC
:1064B00059312E3736365A2D322E3133360A4E3870
:1064C00034205837342E36323559312E3731335A3D
:1064D0002D322E3137300A4E3835205837342E358C
:1064E000373259312E3635395A2D322E3138300A5D
:1064F0004E3836205837342E33353859312E34340F
:10650000355A2D322E3135370A4E38372058373428
:106510002E31393759312E3238345A2D322E313905
:10652000350A4E3838205837342E30393059312E0C
:106530003137375A2D322E3234350A4E38392058F9
:1065400037332E39383359312E3037305A2D322ED9
:106550003232350A4E3930205837332E38323359DB
:10656000302E3931305A2D322E3133380A4E3931EE
:10657000205837332E33393459302E3438325A2D8F
:10658000312E3931370A4E3932205837332E3138CF
:106590003059302E3236385A2D312E3832350A4E97
:1065A0003933205837322E39363659302E3035347B
:1065B0005A2D312E3731310A4E3934205837322E88
:1065C000393133592D302E3030305A2D312E363965
:1065D000330A4E3935205837322E3733335A2D315E
:1065E0002E3634360A4E3936205837322E3939375E
:1065F00059302E3236345A2D312E3735330A4E3932
:1066000037205837332E32363059302E3532375AFC
:106610002D312E3930320A4E3938205837332E3644
:10662000323959302E3839365A2D322E3037370A12
:106630004E3939205837332E38343059312E3130D5
:10664000375A2D322E3232340A4E313030205837FC
:10665000332E38393359312E3136305A2D322E32CD
:1066600034350A4E3130312058373559305A300AD6
:10667000004E312054314D360A4E32204731370A10
:106680004E33204732310A4E382046313830300AF6
:106690004E392047310A4E313030204739322058A8
:1066A0002D32352E313737592D33342E30373220B5
:1066B0005A2D312E303030202854454D502C205248
:1066C000454D4F5645204C41544552290A4E3334CE
:1066D0003320582D32352E353935592D33342E335C
:1066E00034390A4E33343420582D32352E37303178
:1066F000592D33342E3433360A4E33343520582D49
:1067000032352E373931592D33342E3532300A4E49
:1067100033343620582D32352E383634592D333413
:106720002E3630310A4E33343720582D32352E393B
:106730003230592D33342E3637390A4E333438201F
:10674000582D32352E393630592D33342E373534D5
:106750000A4E33343920582D32352E393832592DDE
:1067600033342E3832360A4E33353020582D3235F8
:106770002E393837592D33342E3839350A4E3335C2
:106780003120582D32352E393736592D33342E39A4
:1067900036310A4E33353220582D32352E393438C1
:1067A000592D33352E3032330A4E33353320582DA0
:1067B00032352E393033592D33352E3038320A4E9A
:1067C00033353420582D32352E383431592D333568
:1067D0002E3133380A4E33353520582D32352E3789
:1067E0003633592D33352E3139300A4E3335362074
:1067F000582D32352E363639592D33352E32333920
:106800000A4E33353720582D32352E353539592D2E
:1068100033352E3238340A4E33353820582D323540
:106820002E343333592D33352E3332350A4E33352A
:106830003920582D32352E323931592D33352E33FA
:1068400036330A4E33363020582D32352E3133341C
:10685000592D33352E3339370A4E33363120582DE2
:1068600032342E393633592D33352E3432380A4EE0
:1068700033363220582D32342E373737592D3335B1
:106880002E3435350A4E33363320582D32342E35DA
:106890003737592D33352E3437370A4E33363420B7
:1068A000582D32342E333637592D33352E34393670
:1068B0000A4E33363520582D32342E313434592D8A
:1068C00033352E3531310A4E33363620582D32339A
:1068D0002E393039592D33352E3532320A4E333672
:1068E0003720582D32332E363631592D33352E354B
:1068F00032390A4E33363820582D32332E34303365
:10690000592D33352E3533320A4E33363920582D32
:1069100032332E313333592D33352E3533320A4E3F
:1069200033373020582D32322E383533592D333508
:106930002E3532370A2F4E32353138204730583015
:106940002E333237592D33332E3532315A2D312EE5
:106950003030300A4E32353139204D3330004E312F
:10696000204732300A4E3520473430204731370A2D
:106970004E3130205431204D30360A284E313520EA
:10698000473930204730205830205930205A30299C
:106990000A4E3230205335303030204D3033200A0B
:1069A0004E32352058302E3036342059302E333286
:1069B00036205A300A4E34302047303120463136A6
:1069C0002E300A4E35302058302E30363420593093
:1069D0002E3332360A4E35352058302E30363020A0
:1069E00059302E3239330A4E36302058302E303757
:1069F000372059302E3236370A4E36352058302E51
:106A00003131312059302E3235370A4E3730205847
:106A1000302E3134392059302E3235320A4E373546
:106A20002058302E3138382059302E3235350A4E24
:106A300038302058302E3232372059302E32363806
:106A40000A4E38352058302E3235372059302E3204
:106A500037310A4E39302058302E333335205930F3
:106A60002E3236350A4E39352058302E3431322008
:106A700059302E3237310A4E3130302058302E34D2
:106A800037342059302E3238370A4E3130352058BD
:106A9000302E3439312059302E3238390A4E3131C6
:106AA000302058302E3531372059302E3237330AC6
:106AB0004E3131352058302E3534342059302E3275
:106AC00036330A4E3132302058302E353830205986
:106AD000302E3236310A4E3132352058302E35398B
:106AE000352059302E3236330A4E3133302058306B
:106AF0002E3632312059302E3237340A4E3133356A
:106B00002058302E3635392059302E3330360A4E43
:106B10003134302058302E3637332059302E33332D
:106B2000350A4E3134352058302E36373920593019
:106B30002E3336310A4E3135302058302E36373824
:106B40002059302E3338390A4E3135352058302E01
:106B50003637302059302E3432300A4E313630201C
:106B600058302E3637302059302E3434360A4E31D4
:106B700036352058302E3638302059302E343734C0
:106B80000A4E3137302058302E3730342059302ECD
:106B90003439370A4E3137352058302E37333220CA
:106BA00059302E3531350A4E3138302058302E3795
:106BB00039342059302E3533350A4E313835205886
:106BC000302E3837322059302E3536370A4E31398B
:106BD000302058302E3935302059302E3630340A96
:106BE0004E3139352058312E3033312059302E3640
:106BF00034370A4E3230302058312E313439205952
:106C0000302E3732320A4E3230352058312E333062
:106C1000382059302E3835340A4E32313020583130
:106C20002E3433302059302E3938340A4E32313533
:106C30002058312E3434372059302E3938360A4E08
:106C40003232302058312E3632382059302E3832F8
:106C5000320A4E3232352058312E373332205930F5
:106C60002E3731340A4E3233302058322E303039FC
:106C70002059302E3338310A4E3233352058322ED7
:106C80003131362059302E3236360A4E32343020E9
:106C900058322E3232382059302E3135370A4E32A2
:106CA00034352058322E3238302059302E3132339C
:106CB0000A4E3235302058322E3333322059302E9E
:106CC0003039340A4E3235352058322E34323320A2
:106CD00059302E3037300A4E3236302058322E346A
:106CE00038392059302E3036350A4E323635205854
:106CF000322E3535372059302E3036360A4E32375F
:106D0000302058322E3632372059302E3038340A5F
:106D10004E3237352058322E3639332059302E3105
:106D200030390A4E3238302058322E37333020591D
:106D3000302E3133330A4E3238352058322E383027
:106D4000352059302E3139300A4E32393020583200
:106D50002E3832392059302E3231360A4E323935FA
:106D60002058322E3838302059302E3239310A4EE0
:106D70003330302058322E3838342059302E3330CA
:106D8000300A4E3330352058322E383938205930B9
:106D90002E3333320A4E3331302058322E393035CB
:106DA0002059302E3336370A4E3331352058322EA3
:106DB0003931302059302E3430370A4E33323020BA
:106DC00058322E3930382059302E3434360A4E336A
:106DD00032352058322E3930312059302E34393561
:106DE0000A4E3333302058322E3839372059302E5E
:106DF0003439350A4E3333352058322E3839302065
:106E000059302E3532340A4E3334302058322E3831
:106E100034322059302E3630340A4E33343520582F
:106E2000322E3831342059302E3636350A4E33352D
:106E3000302058322E3739342059302E3735300A29
:106E40004E3335352058322E3739312059302E38CF
:106E500033380A4E3336302058322E3831392059E3
:106E6000302E3937360A4E3336352058322E3833E5
:106E7000372059312E3034340A4E333730205832CF
:106E80002E3836322059312E3131320A4E333735D1
:106E90002058322E3837372059312E3134350A4EAA
:106EA0003338302058322E3931322059312E323198
:106EB000370A4E3338352058322E39313720593180
:106EC0002E3232360A4E3339302058322E3935318F
:106ED0002059312E3238310A4E3339352058322E6E
:106EE0003937302059312E3239350A4E343030207E
:106EF00058322E3939362059312E3239350A4E342E
:106F000030352058332E3031332059312E32373539
:106F10000A4E3431302058332E3032342059312E3D
:106F20003235340A4E3431352058332E3037302044
:106F300059312E3135310A4E3432302058332E300B
:106F400037372059312E3133340A4E3432352058F8
:106F5000332E3132352059312E3033390A4E343305
:106F6000302058332E3133382059312E3031390A00
:106F70004E3433352058332E3230352059302E39A7
:106F800030380A4E3434302058332E3238322059BB
:106F9000302E3739370A4E3434352058332E3336B5
:106FA000312059302E3639310A4E3435302058339D
:106FB0002E3432362059302E3539320A4E3435359A
:106FC0002058332E3435362059302E3534330A4E7E
:106FD0003436302058332E3437392059302E343956
:106FE000330A4E3436352058332E34393420593054
:106FF0002E3437320A4E3437302058332E35303560
:107000002059302E3434360A4E3437352058332E3A
:107010003531382059302E3431370A4E343830204B
:1070200058332E3533302059302E3339310A4E340F
:1070300038352058332E3536342059302E33303001
:107040000A4E3439302058332E3537372059302EF8
:107050003235330A4E3439352058332E3536382000
:1070600059302E3231320A4E3530302058332E35D9
:1070700034342059302E3137360A4E3530352058C9
:10708000332E3534312059302E3134360A4E3531D5
:10709000302058332E3535332059302E3131390ACE
:1070A0004E3531352058332E3537362059302E3174
:1070B00030360A4E3532302058332E353937205984
:1070C000302E3130320A4E3532352058332E36319B
:1070D000382059302E3130390A4E3533302058336C
:1070E0002E3633392059302E3132390A4E35333568
:1070F0002058332E3635302059302E3135390A4E4E
:107100003534302058332E3636332059302E31372F
:10711000380A4E3534352058332E3637382059301A
:107120002E3139320A4E3535302058332E36393922
:107130002059302E3139370A4E3535352058332E07
:107140003732332059302E3139360A4E3536302019
:1071500058332E3736342059302E3137390A4E35D0
:1071600036352058332E3830352059302E313635CB
:107170000A4E3537302058332E3838342059302EC7
:107180003135390A4E3537352058332E39343920C8
:1071900059302E3136350A4E3538302058332E3995
:1071A00036362059302E3137350A4E35383520588D
:1071B000332E3937382059302E3139340A4E35398B
:1071C000302058332E3937382059302E3232330A96
:1071D0004E3539352058332E3936302059302E323D
:1071E00034350A4E3630302058332E383334205957
:1071F000302E3331310A4E3630352058332E373663
:10720000322059302E3334350A4E3631302058333F
:107210002E3732362059302E3338390A4E36313532
:107220002058332E3730332059302E3435380A4E1B
:107230003632302058332E3638322059302E3533FE
:10724000300A4E3632352058332E363739205930F1
:107250002E3533340A4E3633302058332E363236FC
:107260002059302E3638310A4E3633352058332ED9
:107270003536382059302E3832380A4E36343020E0
:1072800058332E3434342059312E3038300A4E36AB
:1072900034352058332E3430352059312E3136379D
:1072A0000A4E3635302058332E3430342059312EA2
:1072B0003136370A4E3635352058332E333837209D
:1072C00059312E3230380A4E3636302058332E336C
:1072D00038342059312E3230380A4E36363520585F
:1072E000332E3336352059312E3236350A4E363765
:1072F000302058332E3335352059312E3238350A67
:107300004E3637352058332E3334382059312E330A
:1073100030380A4E3638302058332E333333205924
:10732000312E3335300A4E3638352058332E33322D
:10733000312059312E3339310A4E36393020583305
:107340002E3331312059312E3432380A4E36393508
:107350002058332E3333392059312E3432330A4EEC
:107360003730302058332E3434302059312E3430D9
:10737000360A4E3730352058332E353130205931CA
:107380002E3430380A4E3731302058332E353835C8
:107390002059312E3432310A4E3731352058332EB0
:1073A0003631312059312E3433390A4E37323020BC
:1073B00058332E3631312059312E3434310A4E377C
:1073C00032352058332E3631352059312E34343170
:1073D0000A4E3733302058332E3633362059312E6B
:1073E0003438380A4E3733352058332E363334206C
:1073F00059312E3531370A4E3734302058332E3636
:1074000032322059312E3534330A4E373435205834
:10741000332E3630352059312E3536330A4E373536
:10742000302058332E3537362059312E3537350A2E
:107430004E3735352058332E3534342059312E35DA
:1074400038310A4E3736302058332E3437392059E8
:10745000312E3539320A4E3736352058332E3435F1
:10746000312059312E3539380A4E373730205833CC
:107470002E3338372059312E3632360A4E373735CB
:107480002058332E3339302059312E3633360A4EB8
:107490003738302058332E3533322059312E36309C
:1074A000320A4E3738352058332E36303120593194
:1074B0002E3539370A4E3739302058332E36363884
:1074C0002059312E3539380A4E3739352058332E68
:1074D0003738322059312E3631320A4E383030208A
:1074E00058332E3739342059312E3631380A4E3838
:1074F00030352058332E3836382059312E36333631
:107500000A4E3831302058332E3931382059312E37
:107510003635350A4E3831352058332E393435203A
:1075200059312E3636370A4E3832302058332E39FC
:1075300036342059312E3638350A4E3832352058F7
:10754000332E3936372059312E3638350A4E3833F6
:10755000302058332E3937342059312E3639390AF4
:107560004E3833352058332E3938342059312E37A0
:1075700032350A4E3834302058332E3938342059B9
:10758000312E3735380A4E3834352058332E3937B6
:10759000302059312E3739300A4E383530205833A3
:1075A0002E3934352059312E3831370A4E38353599
:1075B0002058332E3931382059312E3832360A4E80
:1075C0003836302058332E3839312059312E383260
:1075D000370A4E3836352058332E38343220593158
:1075E0002E3830390A4E3837302058332E37393854
:1075F0002059312E3738340A4E3837352058332E3B
:107600003734362059312E3737320A4E3838302049
:1076100058332E3639382059312E3736340A4E3801
:1076200038352058332E3633352059312E373636FB
:107630000A4E3839302058332E3535332059312E03
:107640003738350A4E3839352058332E34373820FC
:1076500059312E3832300A4E3930302058332E34DA
:1076600030392059312E3836340A4E3930352058C9
:10767000332E3334352059312E3931380A4E3931D1
:10768000302058332E3236342059322E3032330ADD
:107690004E3931352058332E3234382059322E307D
:1076A00035310A4E3932302058332E323430205999
:1076B000322E3038310A4E3932352058332E33319C
:1076C000362059322E3038360A4E3933302058336E
:1076D0002E3339302059322E3130340A4E39333579
:1076E0002058332E3431342059322E3132310A4E63
:1076F0003934302058332E3433312059322E31353D
:10770000330A4E3934352058332E3433332059322E
:107710002E3138300A4E3935302058332E34323736
:107720002059322E3230350A4E3935352058332E15
:107730003431332059322E3232340A4E3936302029
:1077400058332E3339322059322E3234320A4E39E0
:1077500036352058332E3333352059322E323434D7
:107760000A4E3937302058332E3237382059322ECE
:107770003233360A4E3937352058332E32353620DB
:1077800059322E3234320A4E3938302058332E32A4
:1077900033392059322E3235310A4E393835205896
:1077A000332E3231312059322E3238300A4E3939A7
:1077B000302058332E3137342059322E3335360AA3
:1077C0004E3939352058332E3135392059322E3340
:1077D00039370A4E313030302058332E3135302091
:1077E00059322E3433380A4E313030352058332E4A
:1077F0003134302059322E3438310A4E3130313064
:107800002058332E3133322059322E3531300A4E42
:10781000313031352058332E3131382059322E3520
:1078200034330A4E313032302058332E303939203B
:1078300059322E3537360A4E313032352058332EF4
:107840003035312059322E3633310A4E3130333013
:107850002058332E3030332059322E3636360A4EE9
:10786000313033352058322E3935372059322E36C3
:1078700038350A4E313034302058322E39303720E6
:1078800059322E3639390A4E313034352058322E9D
:107890003836302059322E3731310A4E31303530BA
:1078A0002058322E3831392059322E3732370A4E8D
:1078B000313035352058322E3736382059322E3770
:1078C00034350A4E313036302058322E373136209A
:1078D00059322E3735370A4E313036352058322E50
:1078E0003637352059322E3735370A4E313037305A
:1078F0002058322E3537392059322E3733310A4E3F
:10790000313037352058322E3537302059322E3726
:1079100032330A4E313038302058322E3535392046
:1079200059322E3732300A4E313038352058322E07
:107930003533302059322E3730310A4E313039301C
:107940002058322E3530312059322E3639330A4EF6
:10795000313039352058322E3437312059322E36D5
:1079600038330A4E313130302058322E34343320FF
:1079700059322E3636380A4E313130352058322EB3
:107980003339362059322E3633340A4E31313130C4
:107990002058322E3335342059322E3539310A4EA3
:1079A000313131352058322E3335322059322E358F
:1079B00039310A4E313132302058322E33323520AF
:1079C00059322E3534330A4E313132352058322E69
:1079D0003331352059322E3532310A4E3131333080
:1079E0002058322E3330372059322E3439380A4E4F
:1079F000313133352058322E3239362059322E3437
:107A000036340A4E313134302058322E3239332058
:107A100059322E3432370A4E313134352058322E15
:107A20003239352059322E3336360A4E313135301F
:107A30002058322E3332312059322E3330330A4E11
:107A4000313135352058322E3335382059322E32E7
:107A500034370A4E313136302058322E3431392005
:107A600059322E3230330A4E313136352058322ECB
:107A70003431392059322E3137390A4E31313730CD
:107A80002058322E3430352059322E3135380A4EB6
:107A9000313137352058322E3336322059322E319B
:107AA00032330A4E313138302058322E33353420BB
:107AB00059322E3130340A4E313138352058322E79
:107AC0003335342059322E3039310A4E3131393084
:107AD0002058322E3338302059322E3036350A4E67
:107AE000313139352058322E3431302059322E3050
:107AF00035310A4E313230302058322E3431302078
:107B000059322E3034370A4E313230352058322E29
:107B10003430352059322E3032380A4E313231303D
:107B20002058322E3430382059322E3031300A4E1F
:107B3000313231352058322E3431362059312E39F8
:107B400039350A4E313232302058322E3433332018
:107B500059312E3938320A4E313232352058322ED0
:107B60003433382059312E3936330A4E31323330DE
:107B70002058322E3434372059312E3934380A4EB9
:107B8000313233352058322E3436312059312E39A6
:107B900033380A4E313234302058322E34383020C7
:107BA00059312E3933310A4E313234352058322E84
:107BB0003437382059312E3839390A4E3132353080
:107BC0002058322E3438372059312E3837350A4E66
:107BD000313235352058322E3530342059312E3857
:107BE00035340A4E313236302058322E3532372075
:107BF00059312E3834380A4E313236352058322E2B
:107C00003534392059312E3834390A4E3132373033
:107C10002058322E3537372059312E3836310A4E1A
:107C2000313237352058322E3630342059312E3803
:107C300036360A4E313238302058322E3633312023
:107C400059312E3835340A4E313238352058322EDB
:107C50003634302059312E3832370A4E31323930ED
:107C60002058322E3634302059312E3739320A4ED0
:107C7000313239352058322E3632392059312E37AB
:107C800035390A4E313330302058322E36313220D9
:107C900059312E3732370A4E313330352058322E93
:107CA0003537362059312E3639340A4E313331309A
:107CB0002058322E3533362059312E3636320A4E80
:107CC000313331352058322E3437302059312E3669
:107CD00031360A4E313332302058322E333435208B
:107CE00059312E3535310A4E313332352058322E46
:107CF0003330372059312E3532310A4E313333305B
:107D00002058322E3236302059312E3438320A4E35
:107D1000313333352058322E3234332059312E341A
:107D200037370A4E313334302058322E3232382031
:107D300059312E3436390A4E313334352058322EEB
:107D40003232322059312E3434380A4E3133353004
:107D50002058322E3232382059312E3432350A4EE4
:107D6000313335352058322E3235342059312E34C6
:107D700030350A4E313336302058322E32363820E4
:107D800059312E3337330A4E313336352058322E9F
:107D90003237392059312E3334320A4E31333730AD
:107DA0002058322E3330382059312E3238370A4E8F
:107DB000313337352058322E3334302059312E327A
:107DC00035340A4E313338302058322E3430372093
:107DD00059312E3230310A4E313338352058322E57
:107DE0003434312059312E3135360A4E3133393061
:107DF0002058322E3435342059312E3133310A4E49
:107E0000313339352058322E3436302059312E3125
:107E100030360A4E313430302058322E3436342049
:107E200059312E3130320A4E313430352058322E0D
:107E30003437312059312E3033360A4E3134313017
:107E40002058322E3436362059302E3937310A4EEA
:107E5000313431352058322E3435312059302E38D6
:107E600039370A4E313432302058322E34313520F1
:107E700059302E3739310A4E313432352058322EAE
:107E80003430332059302E3736370A4E31343330C0
:107E90002058322E3338382059302E3736350A4E96
:107EA000313433352058322E3330362059302E3885
:107EB00034310A4E313434302058322E32323220AE
:107EC00059302E3931310A4E313434352058322E62
:107ED0003131342059302E3939350A4E313435306C
:107EE0002058322E3030322059312E3037360A4E5B
:107EF000313435352058312E3930352059312E3135
:107F000033390A4E313436302058312E373534204B
:107F100059312E3232330A4E313436352058312E13
:107F20003633372059312E3237380A4E3134373014
:107F30002058312E3538322059312E3330310A4E07
:107F4000313437352058312E3535382059312E33DC
:107F500031350A4E313438302058312E3436302005
:107F600059312E3335320A4E313438352058312EBE
:107F70003339392059312E3336300A4E31343930C5
:107F80002058312E3333382059312E3335340A4EB0
:107F9000313439352058312E3238372059312E338B
:107FA00032390A4E313530302058312E32343820B3
:107FB00059312E3239340A4E313530352058312E70
:107FC0003231372059312E3235340A4E3135313085
:107FD0002058312E3231342059312E3235320A4E6A
:107FE000313531352058312E3137322059312E314B
:107FF00039350A4E313532302058312E3132382061
:1080000059312E3133390A4E313532352058312E1F
:108010003131302059312E3131370A4E313533303C
:108020002058302E3935382059302E3934310A4E07
:10803000313533352058302E3839312059302E38EB
:1080400037330A4E313534302058302E383235200F
:1080500059302E3830380A4E313534352058302ECC
:108060003735352059302E3734370A4E31353530D3
:108070002058302E3631392059302E3633330A4EBF
:10808000313535352058302E3437372059302E359C
:1080900032360A4E313536302058302E34373720BC
:1080A00059302E3532340A4E313536352058302E7F
:1080B0003431312059302E3437360A4E313537308D
:1080C0002058302E3333312059302E3435340A4E77
:1080D000313537352058302E3237382059302E344C
:1080E00032370A4E313538302058302E3233312075
:1080F00059302E3339370A4E313538352058302E25
:108100003138332059302E3337390A4E3135393032
:108110002058302E3133352059302E3336350A4E23
:10812000313539352058302E3037362059302E33FE
:1081300034310A4E31363035204730302046333026
:108140002E300A4E31363130204D3035200A4E3136
:1081500036313520473930205830205930205A30B8
:108160000A4E31363135204D33300A28456E6420B1
:108170006F6620434E432050726F6772616D290015
:10818000284D53472A2A2A2A204D6963726F737437
:1081900065702054657374205B76315D202A2A2A2D
:1081A0002A290A47303020473137204732312047CB
:1081B00034302047343920473830204739300A6777
:1081C00030783079307A300A7B22316D69223A3149
:1081D0007D0A7B22326D69223A317D0A7B22336D22
:1081E00069223A317D0A7B22346D69223A317D0A57
:1081F0006730207831300A7B22316D69223A327D36
:108200000A78300A7B22316D69223A347D0A78314E
:10821000300A7B22316D69223A387D0A78300A674C
:1082200030207931300A7B22326D69223A327D0A60
:1082300079300A7B22326D69223A347D0A793130F5
:108240000A7B22326D69223A387D0A79300A67301A
:10825000207A31300A7B22336D69223A327D0A7AE4
:10826000300A7B22336D69223A347D0A7A31300A32
:108270007B22336D69223A387D0A7A300A673020D2
:108280006131300A7B22346D69223A327D0A6130D5
:108290000A7B22346D69223A347D0A6131300A7BCF
:1082A00022346D69223A387D0A61300A6D32002825
:1082B0004D53472A2A2A2A20436F6F7264696E61E0
:1082C0007465206F666673657473207465737420BB
:1082D0005B76315D202A2A2A2A290A6730306731E5
:1082E000376732316734306734396738306739304F
:1082F0000A6735340A673932783079307A300A665D
:108300003630300A284D53472A2A2A2A20746573AA
:108310007420473932206F6666736574732A2A2A7F
:108320002A290A286D73675374657020313A204DED
:108330006F76652066726F6D20302C3020746F2050
:1083400033302C30206D6D20696E20706F7369742E
:10835000697665205820646972656374696F6E2957
:108360000A286D73675374657020323A2052657322
:108370006574206F726967696E20746F20302E30CB
:10838000207573696E6720473932290A286D736733
:108390005374657020333A204D6F766520746F20DA
:1083A00032302C302E2053686F756C64206D6F76E0
:1083B00065203230206D6D20696E20706F73697496
:1083C000697665205820646972656374696F6E20F0
:1083D000616E6420737461747573207265706F725E
:1083E000742073686F756C64207374617274206696
:1083F000726F6D20302C30290A286D7367537465B5
:108400007020343A204D6F766520746F20302E3006
:1084100020202053686F756C64206D6F7665203264
:1084200030206D6D20696E206E65676174697665B8
:10843000205820646972656374696F6E20616E6490
:1084400020737461747573207265706F7274207319
:10845000686F756C642073746172742066726F6DDE
:108460002032302C30290A67317833300A673932AC
:1084700078300A67317832300A6731783079300ADB
:108480002473720A67393278300A673470302E35B7
:108490000A284D53472A2A2A2A20746573742047D4
:1084A0003535206F6666736574732A2A2A2A290A6D
:1084B000286D73675374657020313A2053657420BA
:1084C000436F6F7264696E6174652073797374654C
:1084D0006D2032205B6735355D20746F206F6666D6
:1084E000736574206F662035302C3530290A286D6D
:1084F00073675374657020323A2053656C656374FA
:108500002047353520636F6F7264696E6174652032
:1085100073797374656D290A286D73675374657078
:1085200020333A204D6F766520746F20302C302E2A
:1085300020486561642073686F756C64206D6F7688
:108540006520646961676F6E616C6C7920696E206B
:108550002B5820616E64202B5920616E6420737447
:1085600061747573207265706F72742073686F75B3
:108570006C642073746172742066726F6D20302C8D
:1085800030290A6731304C327032783530793530E5
:108590000A6735350A6730783079300A67347030C9
:1085A0002E350A284D53472A2A2A2A2074657374C7
:1085B00020473533206162736F6C757465206F7668
:1085C00065727269646573202A2A2A2A290A286D2D
:1085D00073675374657020313A2052756E206120A4
:1085E00073717561726520696E2047353520737926
:1085F0007374656D290A286D736753746570203232
:108600003A2052756E206120737175617265207712
:108610002F473533206F76657272696465290A6762
:1086200030783079300A673078323079300A673004
:108630007832307932300A673078307932300A67F0
:1086400030783079300A673470302E350A67353328
:108650006730783079300A6735336730783230796F
:10866000300A67353367307832307932300A67350F
:1086700033673078307932300A6735336730783095
:1086800079300A6730783079300A673470302E35A7
:108690000A284D53472A2A2A2A20746573742052C7
:1086A000657475726E20746F20686F6D65202A2A5C
:1086B0002A2A290A286D73675374657020313A207D
:1086C00052657475726E20746F20686F6D652075C9
:1086D00073696E6720473238290A286D73675374AF
:1086E000657020323A20526573657420746F20479C
:1086F000353420636F6F72642073797374656D29EC
:108700000A6732380A6735340A6D333000284D5312
:10871000472A2A2A2A20546573742061636375727C
:10872000616379206F6620736C6F77206D6F76655B
:1087300073205B76315D202A2A2A2A290A6735357B
:108740000A6730783079300A673470302E350A671E
:108750003470302E350A67317831306632320A672C
:1087600035340A6730783079300A6D333000284D5F
:1087700053472A2A2A2A2054657374207665727911
:108780002073686F7274206D6F766573205B76312D
:108790005D202A2A2A2A290A6730783079300A6728
:1087A0003470302E350A673178302E3166313030F2
:1087B000300A78300A78302E310A78300A78302E34
:1087C000310A78300A78302E310A78300A78302E23
:1087D000310A78300A78302E310A78300A78302E13
:1087E000310A78300A78302E310A78300A78302E03
:1087F000310A78300A78302E310A78300A78302EF3
:10880000310A78300A78302E310A78300A78302EE2
:10881000310A78300A78302E310A78300A78302ED2
:10882000310A673470302E350A78300A78302E30AD
:10883000310A78300A78302E30310A78300A7830B0
:108840002E30310A78300A78302E30310A78300AEA
:1088500078302E30310A78300A78302E30310A786C
:10886000300A78302E30310A78300A78302E3031A4
:108870000A78300A78302E30310A78300A78302E73
:1088800030310A78300A78302E30310A78300A7860
:10889000302E30310A78300A78302E30310A783074
:1088A0000A78302E30310A6730783079300A6D32EC
:1088B00000284D53472A2A2A2A20526F7461727960
:1088C0002041786973204D6F74696F6E2054657311
:1088D00074205B76315D202A2A2A2A290A673030E3
:1088E000673137673231673430673439673830671A
:1088F00039300A6730783079307A306130623063ED
:10890000300A6735350A6730783079300A66333691
:108910003030300A6730613336300A623336300A1D
:10892000633336300A61300A62300A63300A6731D5
:1089300061313434300A62313434300A63313434D2
:10894000300A61300A62300A63300A6731613134BB
:10895000343062373230633336300A783079307AE7
:10896000306130623063300A6731783630613134DB
:10897000343062373230633336300A783079307AC7
:10898000306130623063300A6731783630793530A3
:10899000613134343062373230633336300A783004
:1089A00079307A306130623063300A67317836303E
:1089B0007935307832356131343430623732306372
:1089C0003336300A783079307A3061306230633053
:1089D0000A6735340A6730783079300A6D333000F1
:1089E000284D53472A2A2A2A20496E7665727365D4
:1089F0002054696D65204D6F74696F6E20546573E6
:108A000074205B76315D202A2A2A2A290A673030B1
:108A100067313767323167343067343967383067E8
:108A200039300A6735350A6730783079300A673966
:108A3000330A66302E30310A67317831300A7931A5
:108A4000300A7A31300A6131300A78300A79300AD6
:108A50007A300A61300A67317831307931307A2DD5
:108A600031306131300A6730783079307A306130B6
:108A70000A66302E310A6732783130792D31307AFA
:108A80002D32306931300A6730783079307A300AE7
:108A90006733783130792D31307A2D323069313089
:108AA0000A6730783079307A300A67327832307934
:108AB000307A2D32306931300A6730783079307A47
:108AC000300A673378323079306931300A6730786C
:108AD0003079307A300A6732783079307A2D333015
:108AE0006931300A6733783079307A306931300A49
:108AF0006730783079307A300A6732783079306987
:108B00003230202843572033363020646567726541
:108B10006573290A67337830793069323020284309
:108B20004357203336302064656772656573290AC0
:108B30006739340A6735340A6730783079300A6D1E
:108B40003330007B226763223A2267303067313747
:108B500067323167343067343967383067393022EB
:108B60007D0A7B226763223A22673535227D0A7BA4
:108B7000226763223A22673078307930227D0A7B7F
:108B8000226763223A2266353030227D0A7B2267D3
:108B900063223A22284D53477371756172657329B8
:108BA000227D0A7B226763223A22673078323022A4
:108BB0007D0A7B226763223A22793230227D0A7B4A
:108BC000226763223A227830227D0A7B2267632261
:108BD0003A227930227D0A7B226763223A2267316A
:108BE000783130227D0A7B226763223A2279313044
:108BF000227D0A7B226763223A227830227D0A7B1B
:108C0000226763223A227930227D0A7B226763221F
:108C10003A22284D5347636972636C657329227D3C
:108C20000A7B226763223A226732783130792D310C
:108C300030693130227D0A7B226763223A22673015
:108C400078307930227D0A7B226763223A226733AB
:108C5000783130792D3130693130227D0A7B2267BD
:108C600063223A22673078307930227D0A7B22678E
:108C700063223A2267327832307930693130227D8E
:108C80000A7B226763223A22673078307930227D6E
:108C90000A7B226763223A2267337832307930695F
:108CA0003130227D0A7B226763223A226730783096
:108CB0007930227D0A7B226763223A22673278303C
:108CC0007930693130227D0A7B226763223A22673C
:108CD0003378307930693130227D0A7B2267632214
:108CE0003A22673534227D0A7B226763223A226763
:108CF0003078307930227D0A7B226763223A226DF8
:108D00003330227D00284D53472A2A2A2A204D63DA
:108D10006F6465732074657374205B76315D202AFF
:108D20002A2A2A290A6735350A6730783079300AC5
:108D30006D330A673470310A6D350A673470310A51
:108D40006D340A673470310A6D350A673470310A40
:108D50006D370A673470310A6D390A673470310A29
:108D60006D380A673470310A6D390A663530300A59
:108D700067307832300A7932300A6D330A78300A37
:108D80006D340A79300A6D350A67317831300A6DF1
:108D9000370A7931300A6D380A78300A6D390A7924
:108DA000300A6732783130792D31306931300A6DCF
:108DB000330A6730783079300A6D340A6733783196
:108DC00030792D31306931300A6D350A67307830AD
:108DD00079300A6D370A673278323079306931304C
:108DE0000A6D380A6730783079300A6D390A67338E
:108DF00078323079306931300A6730783079300A2A
:108E00006732783079306931300A673378307930B9
:108E10006931300A6735340A6730783079300A6D45
:108E2000333000284D53472A2A2A2A204665656494
:108E3000686F6C642054657374205B76315D202A02
:108E40002A2A2A290A284D53472A2A2A2A204D61EC
:108E50006E75616C6C7920656E746572202120617D
:108E60006E64207E20647572696E67206D6F766512
:108E70006D656E7420746F2074657374202A2A2ABD
:108E80002A290A6735350A6730783079300A67341D
:108E900070330A6730306731376732316734306793
:108EA00034396738306739300A663630300A67300F
:108EB000783130307637362E3736350A783079309B
:108EC0000A6735340A6730783079300A6D333000FC
:108ED000284D53472A2A2A2A204477656C6C20544F
:108EE000657374205B76315D202A2A2A2A290A6755
:108EF00030306731376732316739300A6735350AC4
:108F00006730783079300A663530300A673078312A
:108F1000300A673470310A67307832300A6734704B
:108F2000310A67307831300A673470310A67307837
:108F300030300A673470310A79350A6735340A6788
:108F400030783079300A6D330A673470310A67300F
:108F50007831307931300A6D350A673470310A67FB
:108F6000307832307932300A6D340A673470310A21
:108F700067307833307933300A6D380A67347031AE
:108F80000A67307834307934300A6D390A673470C2
:108F9000310A67307835307935300A673078307982
:108FA000300A6D3330002F286D73672A2A2A2A2051
:108FB0004172632054657374205B76315D202A2AE8
:108FC0002A2A290A4E31206730306731376732311B
:108FD0006734306734396738306739300A4E31309A
:108FE000206730783079300A4E32302066353030A4
:108FF0000A4E3330206732783130792D3130693183
:109000003020284357203237302064656772656509
:1090100073290A4E3430206730783079300A4E3563
:1090200030206733783130792D3130693130202864
:109030004343572039302064656772656573290A98
:109040004E3630206730783079300A4E383020671D
:109050003278323079306931302028435720313826
:10906000302064656772656573290A4E3730206762
:1090700030783079300A4E383020673378323079A2
:10908000306931302028434357203138302064651F
:109090006772656573290A4E3930206730783079F8
:1090A000300A4E39392046313230300A4E313030B4
:1090B00020673278307930693230202843572033A6
:1090C00036302064656772656573290A4E31313028
:1090D0002067327830793069323020284357203386
:1090E000363020616761696E290A4E313230206660
:1090F00037303020284368616E6765206665656497
:109100002072617465207768696C6520696E2047FC
:1091100032206D6F74696F6E206D6F6465290A4E21
:10912000313330206732783079306932302028434B
:109130005720333630203372642074696D65290AF4
:109140004E3134302067327830793069323020281F
:10915000435720333630203474682074696D652994
:109160000A4E31353020663530300A4E31363020E7
:109170006733783079307A3430693230202843438D
:1091800057203336302064656772656573207769D0
:109190007468206C696E6561722074726176656CAA
:1091A000290A4E313730206733783079307A306988
:1091B00032302028434357203336302061676169BD
:1091C0006E290A4E313830206637303020286D73D2
:1091D000672A2A2A2A4368616E6765206665656486
:1091E0002072617465207768696C6520696E20471C
:1091F00033206D6F74696F6E206D6F64652A2A2A43
:109200002A290A4E31393020673378307930693273
:109210003020284343572033363020337264207483
:10922000696D65290A4E32303020673378307930E5
:109230006932302028434357203336302034746855
:109240002074696D65290A4E32313020286D7367AC
:109250002A2A2A2A473138204576616C20746573A2
:10926000742A2A2A2A290A4E3232302047312058BD
:1092700033302E373037205A35302E3732372046AC
:109280003530300A4E3233302047313820473032C3
:10929000205836372E373338205A32332E3631376E
:1092A0002052323520463235300A4E323430206773
:1092B00038300A4E323530206730783079307A30A5
:1092C0000A4E323630206D333000284D53472A2A5B
:1092D0002A2A2053717561726573204D6F74696F0E
:1092E0006E2054657374205B76315D202A2A2A2A09
:1092F000290A673030673137673231673430673475
:10930000396738306739300A6730783079300A6722
:10931000307832302028747261766572736520610E
:109320002032306D6D2073717561726520696E2019
:109330005820616E642059290A7932300A78300A3F
:1093400079300A67317831306635303020286472E0
:10935000617720612031306D6D20737175617265A8
:1093600020696E205820616E642059206174204667
:10937000353030290A7931300A78300A79300A6775
:10938000307A32302028747261766572736520619C
:109390002032306D6D2073717561726520696E20A9
:1093A0005820616E64205A290A7832300A7A300ACD
:1093B00078300A67317832307932307A3230663537
:1093C000303020286665656420612032306D6D2064
:1093D000646961676F6E616C20696E20582C20593A
:1093E00020616E64205A290A783079307A300A7800
:1093F00034307934307A3430202874726176657272
:10940000736520612034306D6D206375626520695D
:109410006E20582C205920616E64205A290A783415
:109420003079307A300A78307934307A34300A78CA
:1094300034307934307A300A783079307A34300AFE
:1094400078307934307A300A78343079307A343080
:109450000A783079307A300A6738300A67307830E5
:1094600079300A673078310A673078300A6D3330E6
:1094700000284D53472A2A2A2A20486F6D696E67B3
:109480002054657374205B76315D202A2A2A2A29AC
:109490000A6732382E32783079307A300A6D3330BC
:1094A00000284D53472A2A2A2A20536D6F6B6520C6
:1094B00054657374205B76315D202A2A2A2A290A92
:1094C0004730302047313720473231204734302071
:1094D00047343920473830204739300A6D336734F4
:1094E00070310A6D35673470310A6D34673470310C
:1094F0000A6D33673470310A6D35673470310A6D27
:1095000037673470310A6D39673470310A6D3867E6
:109510003470310A6D390A6730783079307A300A20
:10952000673030207832300A78300A7932300A7960
:10953000300A7A32300A7A300A6132300A61300AEF
:109540004730302078323020793230207A32302063
:109550006132300A473030207830207930207A303C
:109560002061300A4730312066333020783220794C
:1095700032207A322061320A7830207930207A30F5
:109580002061300A673078310A673078300A6D32EE
:10959000002C000A00257300256C750025312E3043
:1095A00066002573002C000A0025733A25730025F8
:1095B000733A256C750025733A25312E30660025E7
:1095C000733A2573005B74765D202074657874208F
:1095D000766572626F7369747925313564205B300A
:1095E0003D73696C656E742C313D766572626F7384
:1095F000655D0A0025660A00256C750A0025640A67
:109600000025730A0074696E7967205B25735D20FD
:109610006572723A2025733A202573200074696EB2
:109620007967205B25735D206F6B3E2000456E647B
:10963000206F6620636F6D6D616E642066696C6576
:109640000A002DCC9ECA9ACCBBCC1ACDE3CAF2CF6D
:109650009ECA86D0F2D020CFE3CA00004006400662
:109660001040B800B8F2CF9ECA86D0F2D020CFE327
:10967000CA0000400620060840B800B868D29ECA5A
:1096800089D104D2B3D352D1A008400605060901FE
:109690000868D29ECA89D104D22CCDE3CAB0084052
:1096A000060540B030800000000000F0E0D0C0109F
:1096B0000100CF673322211F1B1301016E616E0071
:1096C000696E66004E414E494E495459494E46CD49
:1096D000CCCC3D0AD7233C17B7D13877CC2B329569
:1096E00095E6241FB14F0A000020410000C8420047
:1096F000401C4620BCBE4CCA1B0E5AAEC59D740011
:10970000407A10F35A00A0724E18090010A5D4E850
:109710000000E87648170000E40B54020000CA9AE3
:109720003B000000E1F50500008096980000004035
:10973000420F000000A0860100000010270000007A
:1097400000E803000000006400000000000A0000C0
:109750000000000100000000002C76D888DC674F74
:109760000823DFC1DFAE59E1B1B796E5E3E453C6A4
:109770003AE651997696E8E6C28426EB898C9B629C
:10978000ED407C6FFCEFBC9C9F40F2BAA56FA5F446
:1097900090055A2AF75C936B6CF9676DC11BFCE06E
:1097A000E40D47FEF520E6B500D0ED902E030094C1
:1097B0003577050080841E080000204E0A00000056
:1097C000C80C333333330F986E12831141EF8D2160
:1097D00014893BE65516CFFEE6DB18D1844B381BC7
:1097E000F77C1D901DA4BBE424203284725E22818C
:1097F00000C9F124ECA1E53D270011241FBECFEFE5
:10980000CDBFDFE5DEBF00E00CBF13E2A0E0B0E2B9
:10981000E0EFFDEC01E00BBF02C007900D92AA3A09
:10982000B107D9F72AE5AAEAB3E201C01D92A33530
:10983000B207E1F70E940B840C94F6E60C9400004A
:10984000FC0160817181828193810E94C7D86093FD
:10985000EC320895FC0160817181828193810E94C4
:10986000C7D86093EB320895AF92BF92CF92DF9248
:10987000EF92FF920F931F93CF93DF937B018C01A5
:1098800080E7C82E82E3D82EE601AA24A394BC2E3A
:10989000BC18F70161917191819191917F012CEA3E
:1098A00035EC47E257E30E9456DA18164CF4F801FB
:1098B00040815181628173818B2D0E947985A882BC
:1098C0000C5F1F4F2196F2E3C637DF0701F7DF91E8
:1098D000CF911F910F91FF90EF90DF90CF90BF90AD
:1098E000AF900C948485FC016081718182819381A9
:1098F0000E94C7D86093ED32613019F481E00E9474
:10990000807B81E00C94A17BCF93DF93CDB7DEB752
:109910006897CDBFDEBFFC01608171818281938138
:109920000E94C7D86093EE3281E0613019F40E9442
:10993000807B0CC00E94A17BCE01019628E1FC0136
:1099400011922A95E9F7BC010E94734C6896CDBF2D
:10995000DEBFDF91CF9108950F931F93CF93DF93D5
:10996000CDB7DEB72D97CDBFDEBF27E0EAEEF0E240
:109970008E010F5F1F4FD80101900D922A95E1F7DC
:10998000BC01660F771F680F791F660F771F660F80
:10999000771F660F771F61507A4E45E050E0CE0189
:1099A00008960E9466E4688570E0C8010E9494E40D
:1099B000009739F46B8570E0C8010E9494E4009729
:1099C00011F0801B01C08FEF2D96CDBFDEBFDF9160
:1099D000CF911F910F910895EF92FF920F931F93D4
:1099E000CF93DF938C01F62EE72EEC012D96FC0130
:1099F00061857285838594850E94C7D81F926F9375
:109A0000DF93CF930F5E1F4F1F930F93DF93CF937F
:109A1000EF92FF92EFE4FAE581818F9380818F933B
:109A20000E942DE5EDB7FEB73C96EDBFFEBFDF917E
:109A3000CF911F910F91FF90EF9008950F931F9377
:109A4000CF93DF93EC01162F072F8C819D810E940D
:109A5000AC4C83305CF58F3FA1F528C09E01235F9D
:109A60003F4F9F938F938C858F938B858F938A85A0
:109A70008F9389858F933F932F936196DF93CF9335
:109A80003F932F930F931F938091505A8F93809100
:109A90004F5A8F930E942DE58DB79EB740968DBF8C
:109AA0009EBFDF91CF911F910F910895E7E7F4E1F9
:109AB000659174914FE450E089E69DE30E9466E46D
:109AC000CDCFE091E632F0E0EE0FFF1FED58FB4EF8
:109AD000659174914FE450E089E69DE30E9466E44D
:109AE000BDCF0F931F93CF93DF93EC01162F072F5A
:109AF0008C819D810E94AC4C83307CF58F3FC1F5F9
:109B00002CC0AE014F5E5F4F9E01235F3F4F9F937E
:109B10008F938C858F938B858F938A858F9389857F
:109B20008F935F934F933F932F935F934F933F9305
:109B30002F930F931F938091505A8F9380914F5A78
:109B40008F930E942DE58DB79EB742968DBF9EBF25
:109B5000DF91CF911F910F910895E7E7F4E16591AF
:109B600074914FE450E089E69DE30E9466E4C9CF1A
:109B7000E091E632F0E0EE0FFF1FED58FB4E6591ED
:109B800074914FE450E089E69DE30E9466E4B9CF0A
:109B9000DF92EF92FF920F931F93CF93DF93CDB796
:109BA000DEB72897CDBFDEBF8B01E42ED52E37E080
:109BB000E1EFF0E2DE01119601900D923A95E1F7A6
:109BC00028870E94AC4CF82E288582E08F1518F06B
:109BD000E22FF0E002C0E2E0F0E0EE0FFF1FED58F0
:109BE000FB4E659174914FE450E089E69DE30E943D
:109BF00066E49F938F93F80183818F9382818F9383
:109C000081818F9380818F93E1E0F0E0EC0FFD1F65
:109C1000EF0DF11D80811F928F93DF92EF92809163
:109C2000505A8F9380914F5A8F930E942DE5CDBF4C
:109C3000DEBF2896CDBFDEBFDF91CF911F910F9180
:109C4000FF90EF90DF9008954F925F926F927F9216
:109C5000AF92BF92CF92DF92EF92FF920F931F933A
:109C6000CF93DF93C0E7D2E305E311E35C01899171
:109C7000813009F042C0F801C480D580E680F780C9
:109C80004080518062807380A3019201C701B601B8
:109C90000E94E4D69F772CEA35EC47E257E30E9416
:109CA00053D887FD2AC020E034E244E759ECC701CD
:109CB000B6010E9456DA18165CF4F5012081318154
:109CC00042815381C701B6010E9456DA181604F189
:109CD00020E034E244E759ECC301B2010E9456DAB5
:109CE00018165CF4F5012081318142815381C30152
:109CF000B2010E9453D887FD0BC00B5C1F4FF4E0EC
:109D0000AF0EB11C82E3C637D80709F0B0CF02C04E
:109D10008CED01C080E0DF91CF911F910F91FF90FA
:109D2000EF90DF90CF90BF90AF907F906F905F905B
:109D30004F90089580916C32811105C080916B32F3
:109D400080936A3229C0823031F487E080936A328E
:109D500080916B3221C0833031F489E080936A3284
:109D600080916B3219C0843031F48AE080936A327A
:109D700080916B3211C080916D32813031F485E079
:109D800080936A3280916B3207C0823019F486E08A
:109D900080936A3280916B32863019F080916A32FA
:109DA00008958BE080936A32089580916B32089514
:109DB00080936D32813059F018F0823041F008956F
:109DC0008BE992E38093993290939A32089588E9CF
:109DD00096E58093993290939A320895FC0184819C
:109DE0000895845B9F4FFC0180810895855B9F4FA0
:109DF000FC0180810895825B9F4FFC018081089562
:109E0000815B9F4FFC0180810895875B9F4FFC0120
:109E1000808108950C94589ACD96FC0160817181DF
:109E2000828193810895FC01648308958C5A9F4F29
:109E3000FC01608308958F5B9F4FFC014083518339
:109E400062837383089560939B3270939C328093F6
:109E50009D3290939E328FEF91E20C943366BF92C5
:109E6000CF92DF92EF92FF920F931F93CF93DF93E6
:109E7000D090E8327C010CE013E38091E73290E06F
:109E8000EC01CC0FDD1FC80FD91FCC0FDD1FCC0F8D
:109E9000DD1FCC0FDD1FCC57DF4C81E0D816A9F0B9
:109EA000B881A981CA80BB8040915F33413091F471
:109EB000F80120813181428153816B2F7A2F8C2DC3
:109EC0009B2D0E94E5D69B0109C020E030E080E098
:109ED00090E004C02B2F3A2F8C2D9B2DA901BC01A3
:109EE000F701458F568F678F70A3F4E0EF0EF11CDA
:109EF0000C5F1F4F249683E30432180771F6DF913D
:109F0000CF911F910F91FF90EF90DF90CF90BF9076
:109F10000895835B9F4FFC0160838BE992E30C946F
:109F20002F4F4F925F926F927F928F929F92AF923C
:109F3000BF92CF92DF92EF92FF920F931F93CF9336
:109F4000DF93CDB7DEB76897CDBFDEBF8C016091E0
:109F50005F3370E080E090E00E94F5D82B013C0177
:109F6000F80160817181828193810E94C7D870E07D
:109F70005B01AA0CBB1CA60EB71EAA0CBB1CAA0C2C
:109F8000BB1CAA0CBB1CC5018C579F4C5C010CE090
:109F900013E3FE0131964F01F501C190D190E1909C
:109FA000F1905F01F80161917191819191918F011F
:109FB000A30192010E94F8DA9B01AC01C701B6012E
:109FC0000E94E5D6F40161937193819391934F01BF
:109FD000F3E304321F0701F7CE0101960E943B9A7A
:109FE0008BE992E30E942F4F6896CDBFDEBFDF91D1
:109FF000CF911F910F91FF90EF90DF90CF90BF9086
:10A00000AF909F908F907F906F905F904F9008954A
:10A010008B59924369F4E62FF0E0EE0FFF1FEE0F2D
:10A02000FF1FEC50FD4C6081718182819381089506
:10A03000862F0C94309ACF92DF92EF92FF920F937B
:10A040001F93CF93DF93EC0182E3CB39D80709F05C
:10A050004AC070E0FB01EE0FFF1FEE0FFF1FEC5038
:10A06000FD4CC080D180E280F3808091E832813065
:10A0700059F18091E73290E0FC01EE0FFF1FE80FED
:10A08000F91FEE0FFF1FE60FF71FEE0FFF1FEE0F7A
:10A09000FF1FEC57FF4C00811181B281A3812091F9
:10A0A0005F332130B1F4FB01EE0FFF1FEE0FFF1FF6
:10A0B000E45FFC4C2081318142815381B8018B2FB8
:10A0C0009A2F0E94E5D608C060E070E080E090E042
:10A0D00003C0B8018B2F9A2F9B01AC01C701B601B9
:10A0E0000E94E4D603C0862F0E94449AC55BDF4FCE
:10A0F0002881211106C023E333E34BEC51E40E9495
:10A100005AD8DF91CF911F910F91FF90EF90DF9080
:10A11000CF90089588E1E0EAF2E3A4EFB2E3019082
:10A120000D928A95E1F78091E43281110CC0809103
:10A130009F32813041F41092D8321092D93210926D
:10A14000DA321092DB3208954F925F926F927F92D3
:10A150008F929F92AF92BF92CF92DF92EF92FF9237
:10A160000F931F93CF93DF93CDB7DEB76997CDBF22
:10A17000DEBF80916C32811155C080919132813067
:10A1800009F050C00E943DCA81114CC0109291321A
:10A190009CE9692E90E3792E26E3822E912C8E0184
:10A1A0000E5E1F4F38EFA32E30E2B32E33C0F701FF
:10A1B00081917F011F928F935F924F92BF92AF92D6
:10A1C0001F930F930E94F8E5B80188E693E20E947E
:10A1D00099638D839E83F60181919191A191B191B3
:10A1E0006F018A879B87AC87BD87CE0101960E944D
:10A1F000B060CDBFDEBF90EFE91690E2F906B9F688
:10A20000E8E16E0E711CFFEF8F1A9F0A8CE388162F
:10A21000910441F024018BEEE82E80E2F82E6301D8
:10A2200088E7C8CF80E06996CDBFDEBFDF91CF91D0
:10A230001F910F91FF90EF90DF90CF90BF90AF9064
:10A240009F908F907F906F905F904F9008952F9286
:10A250003F924F925F926F927F928F929F92AF92B6
:10A26000BF92CF92DF92EF92FF920F931F93CF9303
:10A27000DF93CDB7DEB72997CDBFDEBF4C015B01C1
:10A280004090EA325090E8322090E73260905F339D
:10A290007090E6326B0180EA92E3888799875CE2EE
:10A2A000E52E51E3F52E98E1299E10011124840139
:10A2B000D6016D917D918D919D916D012CEA35ECCA
:10A2C00047E257E30E9453D887FD80C0F7018081A1
:10A2D0008150823008F07AC041104CC0F1E05F1626
:10A2E00009F1E885F985E20DF31DEC51F24080811A
:10A2F000898391819D83B281A381E1E06E1217C0B1
:10A30000E885F985E459FF4F2081318142815381ED
:10A31000BC018B2F9A2F0E94E5D669837D838E83A3
:10A320009F8307C019821D821E821F8202C0BE83C6
:10A33000AF8371100CC023E333E34BEC51E4D8013D
:10A340006D917D918D919C910E94F8DA05C0F80184
:10A35000608171818281938129813D814E815F81FC
:10A360000E94E5D6A885B9856D937D938D939C93C6
:10A3700013972CC0A885B9858D919D910D90BC91A6
:10A38000A02D89839A83AB83BC8371100EC023E315
:10A3900033E34BEC51E4F801608171818281938158
:10A3A0000E94F8DA9B01AC0105C0D8012D913D91C6
:10A3B0004D915C9169817A818B819C810E94E5D667
:10A3C000E885F98560837183828393838885998585
:10A3D00004968887998795E3E90EF11C0C5F1F4F5F
:10A3E000A885B985AC5AB24309F062CF6090E632D5
:10A3F0007090EA32F091E832F983C090E732209110
:10A400005F332D838CE0A80EB11CABECB1E3A887C1
:10A41000B9874CEAE42E42E3F42EB8E1CB9E60010A
:10A4200011248401F50161917191819191915F01F4
:10A430002CEA35EC47E257E30E9453D887FD8CC0E5
:10A44000A885B9858C91882309F486C08150823013
:10A4500030F4F80124843584468457843BC061106D
:10A4600016C023E333E34BEC51E4D8011C966D9105
:10A470007D918D919C911F970E94F8DA20E030E049
:10A4800044EB53E40E94F8DA1B012C010DC020E0DC
:10A4900030E044EB53E4F801648575858685978543
:10A4A0000E94F8DA1B012C012BED3FE049EC50E44F
:10A4B000A885B98591966D917D918D919C91949788
:10A4C0000E94F8DA9B01AC01C201B1010E945AD886
:10A4D0001B012C01711031C0B981B130E1F0F701DD
:10A4E000EC0DFD1DEC51F240A081B1819280838082
:10A4F000ED81E130A1F4F701E459FF4F2081318172
:10A5000042815381BD01892D982D0E94E5D6DB0142
:10A51000982E892E04C0A0E0B0E0912C812CA201DD
:10A520009101BD01892D982D0E94E5D6D7016D932B
:10A530007D938D939C9313970FC0A2019101F70116
:10A5400060817181828193810E94E5D6D7016D93EC
:10A550007D938D939C931397E885F985F596E8870D
:10A56000F987F4E0EF0EF11C0C5F1F4F8885998589
:10A570008A56924309F056CF2996CDBFDEBFDF91B0
:10A58000CF911F910F91FF90EF90DF90CF90BF90F0
:10A59000AF909F908F907F906F905F904F903F9083
:10A5A0002F90089580916830909169308F3E92414C
:10A5B00011F08FE5089580911C3490911D348F3EE9
:10A5C0009241B9F78091F0329091F1328F3E9241F1
:10A5D00081F780916633909167338F3E924149F7BE
:10A5E0008091EF569091F0568F3E924111F78091F5
:10A5F000AB579091AC578F3E9241D9F680E00895C9
:10A6000080916C32811104C083E080936B3203C06F
:10A6100085E080936B3280E00895CF93C82F0E942D
:10A620003AB680E00E94DBB18C2F0E9429AB86E015
:10A6300080936B328C2FCF9108958093E53280E028
:10A6400008958093E63280E008958093EA3280E0B6
:10A650000895AF92BF92CF92DF92EF92FF920F9345
:10A660001F93CF93DF939FEF980F963008F041C070
:10A67000A090E6327A018B0198E1899F6001112454
:10A68000F601E859FF4C6F01C0E0D0E0BB24B39461
:10A69000F70161917191819191917F012CEA35ECE3
:10A6A00047E257E30E9456DA1816E4F4A1100CC0F2
:10A6B00023E333E34BEC51E4F80160817181828143
:10A6C00093810E94F8DA05C0F8016081718182816E
:10A6D0009381F601EC0FFD1F648F758F868F978F26
:10A6E000B092913224960C5F1F4FC831D10581F68C
:10A6F00002C08EE601C080E0DF91CF911F910F91E3
:10A70000FF90EF90DF90CF90BF90AF900895CF93E0
:10A71000DF93CDB7DEB76897CDBFDEBF8093E7325A
:10A72000682F70E080E090E00E94F3D869837A831C
:10A730008B839C831D821E821F82188619861A862F
:10A740001B861C861D861E861F86188A198A1A8AF1
:10A750001B8A1C8A1D8A1E8A1F8A188EAE014F5FB3
:10A760005F4FBA0181E99FE40E94BB8680E0689652
:10A77000CDBFDEBFDF91CF910895CF93DF93EBE99B
:10A78000F2E385E5DF011D928A95E9F78AE5A8E6FF
:10A79000B3E3ED01982F19929A95E9F7A2ECB3E390
:10A7A000ED0119928A95E9F78FEE92E18093683076
:10A7B0009093693080931C3490931D348093F032D1
:10A7C0009093F13280936633909367338093EF5682
:10A7D0009093F0568093AB579093AC57E093993297
:10A7E000F0939A32809181308093E63280917F306D
:10A7F0000E948753809180308093E532809182302F
:10A800008093E932809183308093EA3281E08093B3
:10A81000E4328093603394E090939F3210929232AE
:10A82000109293321092943280936B3280936A32FA
:10A830000E9479B0DF91CF910C94FD87CF92DF9287
:10A84000EF92FF92CF93C82F6A017B01E82FF0E0CF
:10A85000DF01AA0FBB1FAA0FBB1FAC50BD4CCD928E
:10A86000DD92ED92FC921397EE0FFF1FEE0FFF1F8C
:10A87000E056FD4CC082D182E282F382B701A6018C
:10A880000E946E85B701A6018C2F0E947985CF9119
:10A89000FF90EF90DF90CF900C9484853F924F9281
:10A8A0005F926F927F928F929F92AF92BF92CF9260
:10A8B000DF92EF92FF920F931F93CF93DF93CDB769
:10A8C000DEB76897CDBFDEBF362E872EA62EB72EF9
:10A8D0006C0100E010E0E12CF12C9E2CF50161915F
:10A8E0007191819191915F012CEA35EC47E257E338
:10A8F0000E9456DA18160CF050C08091E73290E0B2
:10A90000FC01EE0FFF1FE80FF91FEE0FFF1FEE0D0A
:10A91000FF1DEE0FFF1FEE0FFF1FEC57FF4C408097
:10A920005180628073808091E63281110EC023E3F2
:10A9300033E34BEC51E4F6016081718182819381B4
:10A940000E94F8DA9B01AC0105C0F601208131813B
:10A9500042815381C301B2010E94E5D6AB01BC0123
:10A96000E1E0F0E0EC0FFD1FE00FF11F40835183A9
:10A9700062837383980128593F4CF901E457FD4FD6
:10A980004083518362837383E455F109408351838B
:10A9900062837383892D0E946E85FFEFEF1AFF0A91
:10A9A0000C5F1F4F84E0C80ED11C0831110509F05F
:10A9B00094CF432D582DBE016F5F7F4F84E39CE4FD
:10A9C0000E94BB8680E06896CDBFDEBFDF91CF914D
:10A9D0001F910F91FF90EF90DF90CF90BF90AF90BD
:10A9E0009F908F907F906F905F904F903F900895D1
:10A9F0004F925F926F927F928F929F92AF92BF928F
:10AA0000CF92DF92EF92FF920F931F93CF93DF933A
:10AA1000CDB7DEB76897CDBFDEBF21E020935F33AF
:10AA20008090E7329090E6325B016C0104EF12E314
:10AA3000882D90E07C01EE0CFF1CE80EF91EEE0C58
:10AA4000FF1CEE0CFF1CEE0CFF1CC7018C579F4C2B
:10AA50007C01F50161917191819191915F012CEAE5
:10AA600035EC47E257E30E9456DA181664F5F70111
:10AA70002081318142815381F8016081718182811D
:10AA800093810E94E4D62B013C0191100EC023E378
:10AA900033E34BEC51E4F601608171818281938153
:10AAA0000E94F8DA9B01AC0105C0F60120813181DA
:10AAB00042815381C301B2010E94E4D6F801608F44
:10AAC000718F828F938FF4E0CF0ED11C0C5F1F4FDC
:10AAD00084E0E80EF11C93E30C30190709F0B9CFBC
:10AAE000682D70E080E090E00E94F3D869837A835B
:10AAF0008B839C831D821E821F82188619861A866C
:10AB00001B861C861D861E861F86188A198A1A8A2D
:10AB10001B8A1C8A1D8A1E8A1F8A188EAE014F5FEF
:10AB20005F4FBA0181E99FE40E94BB8680E068968E
:10AB3000CDBFDEBFDF91CF911F910F91FF90EF90BE
:10AB4000DF90CF90BF90AF909F908F907F906F904D
:10AB50005F904F900895CF93DF93CDB7DEB768979E
:10AB6000CDBFDEBF10925F3310920C3310920D33C5
:10AB700010920E3310920F33109210331092113343
:10AB80001092123310921333109214331092153323
:10AB90001092163310921733109218331092193303
:10ABA00010921A3310921B3310921C3310921D33E3
:10ABB00010921E3310921F331092203310922133C3
:10ABC00010922233109223336091E73270E080E0DC
:10ABD00090E00E94F3D869837A838B839C831D82E3
:10ABE0001E821F82188619861A861B861C861D8661
:10ABF0001E861F86188A198A1A8A1B8A1C8A1D8A31
:10AC00001E8A1F8A188EAE014F5F5F4FBA0181E91D
:10AC10009FE40E94BB8680E06896CDBFDEBFDF91D7
:10AC2000CF910895CF93DF93CDB7DEB76897CDBFAF
:10AC3000DEBF10925F336091E73270E080E090E019
:10AC40000E94F3D869837A838B839C831D821E8242
:10AC50001F82188619861A861B861C861D861E86EC
:10AC60001F86188A198A1A8A1B8A1C8A1D8A1E8ABC
:10AC70001F8A188EAE014F5F5F4FBA0181E99FE4D2
:10AC80000E94BB8680E06896CDBFDEBFDF91CF918A
:10AC90000895CF93DF93CDB7DEB76897CDBFDEBF02
:10ACA00081E080935F336091E73270E080E090E074
:10ACB0000E94F3D869837A838B839C831D821E82D2
:10ACC0001F82188619861A861B861C861D861E867C
:10ACD0001F86188A198A1A8A1B8A1C8A1D8A1E8A4C
:10ACE0001F8A188EAE014F5F5F4FBA0181E99FE462
:10ACF0000E94BB8680E06896CDBFDEBFDF91CF911A
:10AD00000895CF9310929F320E9427518091723004
:10AD1000813069F480EA92E30E94244EC82F882390
:10AD200031F00E9429AB82E080936B3217C08BE92F
:10AD300092E30E942F4F85E080936B3280916C32BA
:10AD4000811105C081E080936C320E94D1AE8BE905
:10AD500092E30E94659A0E948A50C0E08C2FCF91A6
:10AD6000089588E1E4EFF2E3A4E2B3E301900D92E9
:10AD70008A95E1F780E008950F931F93CF93DF93B7
:10AD8000CDB7DEB76A97CDBFDEBF8C0181E080937F
:10AD9000E8328BE992E3698F7A8F0E942F4F698D99
:10ADA0007A8DC8010E9481560E94F5858823E1F3BF
:10ADB00088E1E0E0F0E2DE01119601900D928A95C3
:10ADC000E1F7BE016F5F7F4F84E293E30E948156FB
:10ADD0006A96CDBFDEBFDF91CF911F910F9108958D
:10ADE00088E1E4EFF2E3ACE3B3E301900D928A95DE
:10ADF000E1F780E008950F931F93CF93DF93CDB7D2
:10AE0000DEB76A97CDBFDEBF8C0181E08093E83268
:10AE10008BE992E3698F7A8F0E942F4F698D7A8D2B
:10AE2000C8010E9481560E94F5858823E1F388E1DC
:10AE3000E0E0F0E2DE01119601900D928A95E1F7D3
:10AE4000BE016F5F7F4F8CE393E30E9481566A9649
:10AE5000CDBFDEBFDF91CF911F910F910895FB0110
:10AE6000DC018091E432811111C09B01AD0160E0F1
:10AE700070E080E89FE30E945AD86093D8327093C4
:10AE8000D9328093DA329093DB3218C08091E63267
:10AE9000811109C023E333E34BEC51E4CD010E945F
:10AEA000F8DAFB0101C0CD01AF01BC014093D832FB
:10AEB0005093D9326093DA327093DB3280E0089598
:10AEC0008093E43280E008958093E93280E0089531
:10AED0006093E0327093E1328093E2329093E332F8
:10AEE0000E94138780E008950F931F93CF93DF9301
:10AEF000EC018B018091E432882399F08091D83263
:10AF00009091D932A091DA32B091DB32BC01CD01FF
:10AF10009F772CEA35EC47E257E30E9453D887FD30
:10AF200030C081E080939F32B801CE010E9427514A
:10AF300080917230813069F480EA92E30E94244E5D
:10AF4000C82F882331F00E9429AB82E080936B32B6
:10AF500019C08BE992E30E942F4F85E080936B32FA
:10AF600080916C32811105C081E080936C320E9427
:10AF7000D1AE8BE992E30E94659AC82F0E948A5055
:10AF800001C0CEE88C2FDF91CF911F910F910895D2
:10AF9000CF93DF93CDB7DEB76897CDBFDEBF682F05
:10AFA00070E080E090E00E94F3D869837A838B831D
:10AFB0009C831D821E821F82188619861A861B8614
:10AFC0001C861D861E861F86188A198A1A8A1B8A65
:10AFD0001C8A1D8A1E8A1F8A188EAE014F5F5F4F22
:10AFE000BA0180E29CE40E94BB8680E06896CDBFF7
:10AFF000DEBFDF91CF910895CF93DF93CDB7DEB75A
:10B000006897CDBFDEBF6091EC3270E080E090E0E9
:10B010000E94F3D869837A838B839C831D821E826E
:10B020001F82188619861A861B861C861D861E8618
:10B030001F86188A198A1A8A1B8A1C8A1D8A1E8AE8
:10B040001F8A188EAE014F5F5F4FBA018AE29CE4FF
:10B050000E94BB8680E06896CDBFDEBFDF91CF91B6
:10B060000895CF93DF93CDB7DEB76897CDBFDEBF2E
:10B07000682F70E080E090E00E94F3D869837A83C3
:10B080008B839C831D821E821F82188619861A86D6
:10B090001B861C861D861E861F86188A198A1A8A98
:10B0A0001B8A1C8A1D8A1E8A1F8A188EAE014F5F5A
:10B0B0005F4FBA0183E79CE40E94BB8680E06896FC
:10B0C000CDBFDEBFDF91CF910895CF93DF93CDB792
:10B0D000DEB76897CDBFDEBF682F70E080E090E0FC
:10B0E0000E94F3D869837A838B839C831D821E829E
:10B0F0001F82188619861A861B861C861D861E8648
:10B100001F86188A198A1A8A1B8A1C8A1D8A1E8A17
:10B110001F8A188EAE014F5F5F4FBA0184E89CE42E
:10B120000E94BB8680E06896CDBFDEBFDF91CF91E5
:10B130000895CF93FC0160817181828193810E9487
:10B14000C7D860936B3210926D328BE992E3809393
:10B15000993290939A3280916C32813011F410922E
:10B160006C3210926E32109294320E941E9AC091EC
:10B170006B32C430C9F40E94AB5580917F300E947D
:10B180008753809180308093E53280918330809323
:10B19000EA3280E00E94DBB180E00E94655881E0E5
:10B1A0008093E432C0939F3281E0CF910C9495ADAF
:10B1B00080935C3380935D338093653380E00895A2
:10B1C0002CEA35EC47E257E360910834709109347A
:10B1D00080910A3490910B340E9456DA1816B4F418
:10B1E0008091AE339091AF33A091B033B091B13331
:10B1F000BC01CD019F772CEA35EC47E257E30E9472
:10B2000053D887FF03C010925C3303C081E0809362
:10B210005C3380E0089580935C338091AE339091ED
:10B22000AF33A091B033B091B13380935433909346
:10B230005533A0935633B093573380E008952CEAEA
:10B2400035EC47E257E360910834709109348091FE
:10B250000A3490910B340E9456DA1816B4F4809197
:10B26000AE339091AF33A091B033B091B133BC0104
:10B27000CD019F772CEA35EC47E257E30E9453D883
:10B2800087FF03C010925D3303C081E080935D337C
:10B2900080E0089580935D338091AE339091AF3319
:10B2A000A091B033B091B133809358339093593318
:10B2B000A0935A33B0935B3380E008952CEA35ECC9
:10B2C00047E257E3609108347091093480910A3461
:10B2D00090910B340E9456DA1816B4F48091AE3374
:10B2E0009091AF33A091B033B091B133BC01CD0197
:10B2F0009F772CEA35EC47E257E30E9453D887FF4B
:10B3000003C01092653303C081E08093653380E011
:10B310000895809365338091AE339091AF33A091BF
:10B32000B033B091B1338093613390936233A09383
:10B330006333B093643380E00895BC018FEF90E2F3
:10B340000C94566681E080939232089581E0809358
:10B350009332089581E08093943208951F93CF93A0
:10B36000DF93CDB7DEB76897CDBFDEBF0E94589A96
:10B370008130C9F10E942BD50E94788680E00E941E
:10B38000E6AE0E94EFAF10E0812F0E94309AAB0131
:10B39000BC01812F0E941E541F5F1630A9F780E068
:10B3A00090E0A0E4B0E489839A83AB83BC831D82E0
:10B3B0001E821F82188619861A861B861C861D8689
:10B3C0001E861F86188A198A1A8A1B8A1C8A1D8A59
:10B3D0001E8A1F8A188EBE016F5F7F4FCB010E94AD
:10B3E000995880E001C08AE66896CDBFDEBFDF9144
:10B3F000CF911F910895809192328130A9F42091CC
:10B400006D32213079F480916E3281110BC082E06F
:10B4100080936D3288E996E58093993290939A32C1
:10B4200020936E321092923280919332813091F457
:10B4300080916D32882331F0823061F490916E32C8
:10B44000943051F40E94589A811104C010929332A2
:10B450000E94AE5990916E32809194328130C1F445
:10B4600020919332211114C09150933088F01092A2
:10B47000943295E090936E3290936B3290916C324F
:10B48000911104C080936C320E94D1AE0E94CAA276
:10B4900080E0089585E080936B3280916C32811159
:10B4A00005C081E080936C320C94D1AE0895CF93A7
:10B4B000DF93CDB7DEB76897CDBFDEBF80916C322A
:10B4C000882311F180E090E0A0E4B0E489839A83BE
:10B4D000AB83BC831D821E821F82188619861A8642
:10B4E0001B861C861D861E861F86188A198A1A8A44
:10B4F0001B8A1C8A1D8A1E8A1F8A188EBE016F5FD6
:10B500007F4FCB010E9499586896CDBFDEBFDF9177
:10B51000CF910895CF93DF93CDB7DEB76897CDBFB6
:10B52000DEBF80E090E0A0E4B0E489839A83AB833F
:10B53000BC831D821E821F82188619861A861B866E
:10B540001C861D861E861F86188A198A1A8A1B8ADF
:10B550001C8A1D8A1E8A1F8A188EAE014F5F5F4F9C
:10B56000BA0189E998E50E94BB866896CDBFDEBF27
:10B57000DF91CF910895CF93DF93CDB7DEB7689772
:10B58000CDBFDEBF80E090E0A0E8B0E489839A837D
:10B59000AB83BC831D821E821F82188619861A8681
:10B5A0001B861C861D861E861F86188A198A1A8A83
:10B5B0001B8A1C8A1D8A1E8A1F8A188EAE014F5F45
:10B5C0005F4FBA0189E998E50E94BB866896CDBFB6
:10B5D000DEBFDF91CF910895CF93DF93CDB7DEB774
:10B5E0002797CDBFDEBF97E0E1EFF0E2DE011196D5
:10B5F00001900D929A95E1F7873050F4E1E0F0E088
:10B60000EC0FFD1FE80FF11D87FDFA95808101C049
:10B6100080E22796CDBFDEBFDF91CF910895EF92F4
:10B62000FF920F931F93CF93DF931F92CDB7DEB797
:10B630007C018B01642F70E080E090E049830E94E0
:10B64000F3D8F701618772878387948782E08783C5
:10B650004981E42FF0E0EE0FFF1FE00FF11F65912D
:10B6600074914FE450E089E69DE30E9466E4BC01DA
:10B67000C7010F90DF91CF911F910F91FF90EF9035
:10B680000C94F865CF93DF93EC010E949A4E482FFB
:10B6900061EB73E1CE01DF91CF910C940F5B409190
:10B6A0006B3262E773E10C940F5B40916C3269E49A
:10B6B00073E10C940F5B40916D3265E373E10C9480
:10B6C0000F5B40916E3267E073E10C940F5B409129
:10B6D0006F326AEE72E10C940F5BE0919932F09157
:10B6E0009A32E55BFF4F408164E174E10C940F5B9B
:10B6F000E0919932F0919A32E45BFF4F408160E231
:10B7000072E10C940F5BE0919932F0919A3244818E
:10B7100066E871E10C940F5BE0919932F0919A32F6
:10B72000E65BFF4F408163E571E10C940F5BE091B4
:10B730009932F0919A32E25BFF4F408169E071E10A
:10B740000C940F5BE0919932F0919A32E15BFF4FDC
:10B75000408168EC70E10C940F5BE0919932F091BC
:10B760009A32E75BFF4F408169E570E10C940F5B13
:10B77000CF93DF93EC01E0919932F0919A32E05B44
:10B78000FF4F608170E080E090E00E94F3D869870D
:10B790007A878B879C8782E08F8380E0DF91CF91CF
:10B7A0000895CF93DF93EC0160919B3270919C32AE
:10B7B00080919D3290919E320E94F3D869877A875A
:10B7C0008B879C8782E08F8380E0DF91CF91089503
:10B7D000CF93DF93EC01E0919932F0919A3260813E
:10B7E0007181828193810E94F3D869877A878B87E0
:10B7F0009C8782E08F8380E0DF91CF910895CF9383
:10B80000DF93EC0180916D32811105C019861A8693
:10B810001B861C8614C00E94279A69877A878B87AB
:10B820009C872091E35621110AC025E832E441E2C9
:10B830005DE30E94F8DA69877A878B879C878C8121
:10B840009D81FC01EE0FFF1FE80FF91FEE0FFF1F98
:10B85000EE0FFF1FEE0FFF1FEA5FF94E85919491E7
:10B86000888784E08F8380E0DF91CF910895CF9324
:10B87000DF93EC012091993230919A32F901FD96D3
:10B88000608171818281938169877A878B879C87A8
:10B890003E96208121110AC025E832E441E25DE3B1
:10B8A0000E94F8DA69877A878B879C878C819D81D3
:10B8B000FC01EE0FFF1FE80FF91FEE0FFF1FEE0F49
:10B8C000FF1FEE0FFF1FEA5FF94E85919491888765
:10B8D00084E08F8380E0DF91CF910895CF93DF9351
:10B8E000EC018C819D810E94AC4C682F8091993233
:10B8F00090919A320E941B5069877A878B879C8728
:10B900008C819D81FC01EE0FFF1FE80FF91FEE0FE8
:10B91000FF1FEE0FFF1FEE0FFF1FEA5FF94E85912D
:10B920009491888784E08F8380E0DF91CF910895A0
:10B93000CF93DF93EC018C819D810E94AC4C2091D0
:10B94000993230919A322B59324369F4E82FF0E062
:10B95000EE0FFF1FEE0FFF1FEC50FD4C6081718159
:10B960008281938102C00E94309A69877A878B878F
:10B970009C878C819D81FC01EE0FFF1FE80FF91F52
:10B98000EE0FFF1FEE0FFF1FEE0FFF1FEA5FF94ED6
:10B9900085919491888784E08F8380E0DF91CF91B7
:10B9A0000895CF93DF93EC018C819D810E94AC4C74
:10B9B000E0919932F0919A3294E0899FE00DF11D67
:10B9C0001124458D568D678D70A149875A876B87E5
:10B9D0007C878C819D81FC01EE0FFF1FE80FF91F12
:10B9E000EE0FFF1FEE0FFF1FEE0FFF1FEA5FF94E76
:10B9F00085919491888784E08F8380E0DF91CF9157
:10BA00000895CF93DF93EC010E94936169857A8555
:10BA10008B859C850E94C7D8462F60E474E1CE01D7
:10BA2000DF91CF910C940F5BCF93DF93EC018C816E
:10BA30009D810E94AC4C833054F48F3FA9F407C021
:10BA4000CE010E943D6280E01CC08DE61AC020E05D
:10BA500030E040E450E469857A858B859C850E94BE
:10BA600056DA181694F3ECCF20E030E040E050E4D2
:10BA700069857A858B859C850E9456DA18162CF389
:10BA8000DFCFDF91CF91089595E3899FF0011124D5
:10BA9000E35CFE4C60817181828193810895CF9235
:10BAA000DF92EF92FF92CF93DF936A017B0125E350
:10BAB000829FC001112488599F4CFC01EB52FF4F1B
:10BAC0004083518362837383EC01C352DF4F20E0D4
:10BAD00034E244E759E4C701B6010E94F8DA9B0159
:10BAE000AC0160E070E080E89FE30E945AD8688370
:10BAF00079838A839B83DF91CF91FF90EF90DF90D2
:10BB0000CF900895CF92DF92EF92FF92CF93DF9381
:10BB1000EC01C984DA84EB84FC8420E034E244E75D
:10BB200059E4C701B6010E9456DA181664F420E001
:10BB300034E244E759E4C701B6010E945AD8698744
:10BB40007A878B879C87CE010E941267C984DA842A
:10BB5000EB84FC848C819D810E94AC4C25E3829F08
:10BB6000C001112488599F4CFC01EB52FF4FC08249
:10BB7000D182E282F382EC01C352DF4F20E034E253
:10BB800044E759E4C701B6010E94F8DA9B01AC0111
:10BB900060E070E080E89FE30E945AD86883798370
:10BBA0008A839B8380E0DF91CF91FF90EF90DF90BD
:10BBB000CF900895CF92DF92EF92FF92CF93DF93D1
:10BBC000EC01C984DA84EB84FC8420E034E244E7AD
:10BBD00059E4C701B6010E9456DA181664F420E051
:10BBE00034E244E759E4C701B6010E945AD8698794
:10BBF0007A878B879C87CE010E94126780E0DF9155
:10BC0000CF91FF90EF90DF90CF90089581E08093E7
:10BC1000933280E008952CEA35EC47E257E3FC01CB
:10BC200061857285838594850E9456DA181614F40E
:10BC30000E94106F80E00895609195327091963265
:10BC4000809197329091983208950E94226380E00B
:10BC50000E94937180E008950E94226381E00E9417
:10BC6000937180E008950E94226382E00E949371A4
:10BC700080E008950E94226383E00E94937180E037
:10BC80000895CF93DF93EC01E0919932F0919A32CD
:10BC9000E55BFF4FE081F0E0EE0FFF1FED58FB4E3C
:10BCA000659174914FE450E089E69DE30E9466E45B
:10BCB000AC0162E470E1CE01DF91CF910C9494C5A8
:10BCC000CF93DF93EC01E0919932F0919A32E55BEA
:10BCD000FF4FE081F0E0EE0FFF1FED58FB4E659146
:10BCE00074914FE450E089E69DE30E9466E4AC0164
:10BCF0006AE270E1CE01DF91CF910C9494C5CF93AD
:10BD0000DF93EC0183E091E20E94CBE5CE010E943B
:10BD1000415ECE010E94605E66E170E1CE010E944C
:10BD20005BC56DEF7FE0CE010E9426C564EE7FE02B
:10BD3000CE010E9426C56BEC7FE0CE010E9426C595
:10BD400062EB7FE0CE010E9426C569E97FE0CE016B
:10BD50000E9426C560E87FE0CE010E9426C567E606
:10BD60007FE0CE010E9426C56EE47FE0CE010E94F6
:10BD700026C565E37FE0CE010E9426C56CE17FE029
:10BD8000CE010E9426C563E07FE0CE010E9426C559
:10BD90006AEE7EE0CE010E9426C561ED7EE0CE0116
:10BDA0000E9426C568EB7EE0CE010E945BC580E064
:10BDB000DF91CF91089566E170E10C945BC56DEF62
:10BDC0007FE00C9426C564EE7FE00C9426C56BECF6
:10BDD0007FE00C9426C562EB7FE00C9426C569E9F0
:10BDE0007FE00C9426C560E87FE00C9426C567E6EA
:10BDF0007FE00C9426C56EE47FE00C9426C565E3D5
:10BE00007FE00C9426C56CE17FE00C9426C563E0CE
:10BE10007FE00C9426C56AEE7EE00C9426C561EDA9
:10BE20007EE00C9426C568EB7EE00C945BC56CE369
:10BE30007EE00C945BC56BE07EE00C945BC566ED28
:10BE40007DE00C945BC56BE97DE00C945BC567E617
:10BE50007DE00C945BC5CF93DF93EC01E0919932C8
:10BE6000F0919A32E55BFF4FE081F0E0EE0FFF1FAB
:10BE7000ED58FB4E659174914FE450E089E69DE3E7
:10BE80000E9466E4AC0163E47DE0CE01DF91CF91D6
:10BE90000C9494C5CF93DF93EC01E0919932F0912B
:10BEA0009A32E55BFF4FE081F0E0EE0FFF1FED58A7
:10BEB000FB4E659174914FE450E089E69DE30E944A
:10BEC00066E4AC0162E27DE0CE01DF91CF910C949B
:10BED00094C565E07DE00C943CC5CF93DF93EC0105
:10BEE000E0919932F0919A32E55BFF4FE081F0E00A
:10BEF000EE0FFF1FED58FB4E659174914FE450E03B
:10BF000089E69DE30E9466E4AC0166EE7CE0CE012A
:10BF1000DF91CF910C9494C50F931F93CF93DF9330
:10BF20008C01FC0161857285838594850E94C7D848
:10BF3000E62FF0E0EE0FFF1FE05CFB4E6591749181
:10BF40004FE450E089E69DE30E9466E4E8012D9607
:10BF50009F938F93F80161857285838594850E94F4
:10BF6000C7D81F926F93DF93CF930F5E1F4F1F931E
:10BF70000F93DF93CF938AEC9CE09F938F93EFE432
:10BF8000FAE581818F9380818F930E942DE5EDB733
:10BF9000FEB73E96EDBFFEBFDF91CF911F910F918F
:10BFA000089562EA7CE00C941E4D6AE77CE00C94F4
:10BFB0001E4D68E57CE00C941E4D66E37CE00C941D
:10BFC0001E4D64E07CE00C941E4D63ED7BE00C9410
:10BFD0001E4D6AE97BE00C941E4D6AE77BE00C94F1
:10BFE0001E4D68E37BE00C94EC4C66EF7AE00C9419
:10BFF000EC4C6FEC7AE00C941E4D69EA7AE00C94FC
:10C000001E4D68E87AE00C941E4D68E67AE00C94C8
:10C010001E4D6BE47AE00C94714D6CE27AE00C9466
:10C02000714DBC01675F7F4F2091E63242EA5EE0CE
:10C03000FC01848195810C94C84DBC01675F7F4FE2
:10C0400021E048E85EE0FC01848195810C94C84DB4
:10C05000BC01675F7F4F21E04FE65EE0FC01848119
:10C0600095810C94C84D0F931F93CF93DF93EC01F0
:10C070000C811D810E94DD6808171907C0F48C81AE
:10C080009D81FC01EE0FFF1FE80FF91FEE0FFF1F50
:10C09000EE0FFF1FEE0FFF1FE55FF94E2591349164
:10C0A000CE01F901DF91CF911F910F91199485E194
:10C0B000DF91CF911F910F9108950F931F93CF930D
:10C0C000DF93EC010C811D810E94DD6808171907C0
:10C0D000C0F48C819D81FC01EE0FFF1FE80FF91F5A
:10C0E000EE0FFF1FEE0FFF1FEE0FFF1FE75FF94E72
:10C0F00025913491CE01F901DF91CF911F910F91DC
:10C10000199485E1DF91CF911F910F9108950F93BD
:10C110001F93CF93DF93EC010C811D810E94DD689A
:10C1200008171907C0F48C819D81FC01EE0FFF1FD9
:10C13000E80FF91FEE0FFF1FEE0FFF1FEE0FFF1F9F
:10C14000E95FF94E25913491CE01F901DF91CF914C
:10C150001F910F911994DF91CF911F910F91089525
:10C16000CF93DF93EC018C819D810E94F06888233E
:10C17000C9F08C819D81FC01EE0FFF1FE80FF91FB4
:10C18000EE0FFF1FEE0FFF1FEE0FFF1FEB5FF94ECD
:10C19000E491E1FF05C0CE01DF91CF910C9494842E
:10C1A00080E001C085E1DF91CF9108950F931F9347
:10C1B000CF93DF93EC0181E00E9421531C821D820A
:10C1C00080E090E08E010F5E1F4F47C08C819D8103
:10C1D0009C01220F331FF901E80FF91FEE0FFF1F1B
:10C1E000EE0FFF1FEE0FFF1FEB5FF94EE491E0FF34
:10C1F0002EC0280F391F220F331F220F331F220F8B
:10C20000331F215F394EF901459155916591749124
:10C2100049875A876B877C87BC01660F771F680F39
:10C22000791F660F771F660F771F660F771F6150A4
:10C230007A4E45E050E0C8010E9466E4CE010E94BB
:10C240003360CE010E94B0602C813D8101C09C0111
:10C250002F5F3F4F2C833D83C9010E94E06881110D
:10C26000B5CF0E94DFABDF91CF911F910F910C945E
:10C2700097ABCF93DF93EC012CEA35EC47E257E321
:10C2800069857A858B859C850E9453D887FF05C078
:10C29000CE01DF91CF910C948E7DCE010E94D660AD
:10C2A00082E08F8340E050E060E87FE349875A876F
:10C2B0006B877C8780E0DF91CF91089580915E3A13
:10C2C00090915F3A8F3E924111F08AE508958091F6
:10C2D000A03A9091A13A8F3E9241B9F780913435BE
:10C2E000909135358F3E924181F7809156389091EB
:10C2F00057388F3E924149F780915838909159387C
:10C300008F3E924111F780915C3A90915D3A8F3E59
:10C310009241D9F68091B83D8111D7CF0895FC01A3
:10C32000178289E60895CF93DF93EC018C819D817C
:10C33000FC01EE0FFF1FE80FF91FEE0FFF1FEE0FBE
:10C34000FF1FEE0FFF1FE35FF94EA591B4916C91B3
:10C3500070E080E090E00E94F3D869877A878B874D
:10C360009C8782E08F8380E0DF91CF910895CF9307
:10C37000DF93EC018C819D81FC01EE0FFF1FE80F24
:10C38000F91FEE0FFF1FEE0FFF1FEE0FFF1FE35F02
:10C39000F94EA591B4916D917D918D919C910E94E2
:10C3A000F3D869877A878B879C8782E08F8380E0C8
:10C3B000DF91CF910895CF93DF93DC0114968D9197
:10C3C0009C911597FC01EE0FFF1FE80FF91FEE0F70
:10C3D000FF1FEE0FFF1FEE0FFF1FE35FF94EC5912A
:10C3E000D491488159816A817B8119964D935D93DF
:10C3F0006D937C931C9783E017968C9380E0DF917C
:10C40000CF910895CF93DF93DC0114968D919C9189
:10C410001597FC01EE0FFF1FE80FF91FEE0FFF1F2E
:10C42000EE0FFF1FEE0FFF1FE35FF94EC591D49192
:10C43000488159816A817B8119964D935D936D93F3
:10C440007C931C97FC01EE0FFF1FE80FF91FEE0F06
:10C45000FF1FEE0FFF1FEE0FFF1FEA5FF94E8591E2
:10C46000949118968C93189784E017968C9380E09B
:10C47000DF91CF91089588E608950F931F93CF938E
:10C48000DF93EC018C819D81FC01EE0FFF1FE80F13
:10C49000F91FEE0FFF1FEE0FFF1FEE0FFF1FE35FF1
:10C4A000F94E0591149169857A858B859C850E944A
:10C4B000C7D8F801608382E08F8380E0DF91CF915D
:10C4C0001F910F910895CF93DF93EC0169857A85D1
:10C4D0008B859C850E94C7D86230B0F48C819D8189
:10C4E000FC01EE0FFF1FE80FF91FEE0FFF1FEE0F0D
:10C4F000FF1FEE0FFF1FE35FF94EA591B4916C9300
:10C5000082E08F8380E001C08EE6DF91CF910895B5
:10C51000CF93DF93EC0169857A858B859C850E949A
:10C52000C7D86330B0F48C819D81FC01EE0FFF1FF2
:10C53000E80FF91FEE0FFF1FEE0FFF1FEE0FFF1F9B
:10C54000E35FF94EA591B4916C9382E08F8380E014
:10C5500001C08EE6DF91CF910895CF93DF93EC0178
:10C5600069857A858B859C850E94C7D86430B0F434
:10C570008C819D81FC01EE0FFF1FE80FF91FEE0F6C
:10C58000FF1FEE0FFF1FEE0FFF1FE35FF94EA59198
:10C59000B4916C9382E08F8380E001C08EE6DF91DE
:10C5A000CF9108950F931F93CF93DF93EC018C816C
:10C5B0009D81FC01EE0FFF1FE80FF91FEE0FFF1F1B
:10C5C000EE0FFF1FEE0FFF1FE35FF94E0591149171
:10C5D00069857A858B859C850E94C7D8F801608320
:10C5E00071838283938382E08F8380E0DF91CF9198
:10C5F0001F910F910895CF93DF93DC0114968D91D5
:10C600009C911597FC01EE0FFF1FE80FF91FEE0F2D
:10C61000FF1FEE0FFF1FEE0FFF1FE35FF94EC591E7
:10C62000D49119964D915D916D917C911C974883A1
:10C6300059836A837B8383E017968C9380E0DF9134
:10C64000CF910895CF93DF93DC0114968D919C9147
:10C650001597FC01EE0FFF1FE80FF91FEE0FFF1FEC
:10C66000EE0FFF1FEE0FFF1FE35FF94EC591D49150
:10C6700019964D915D916D917C911C9748835983DA
:10C680006A837B83FC01EE0FFF1FE80FF91FEE0F9B
:10C69000FF1FEE0FFF1FEE0FFF1FEA5FF94E8591A0
:10C6A000949118968C93189784E017968C9380E059
:10C6B000DF91CF9108951F93CF93DF93EC01809189
:10C6C000BC3A8823D1F01DE10A80DB81C02D209780
:10C6D00011F480E013C08F818F3FD9F3811104C022
:10C6E000CE010E945D6006C0CE010E943360CE0183
:10C6F0000E94B060115041F7ECCF85E6DF91CF91F9
:10C700001F910895CF93DF93EC01BC0181E191E289
:10C710000E949FE4892B41F0BE0184E191E20E94D6
:10C720009FE421E0892B09F420E0822FDF91CF9153
:10C7300008950F931F93CF93DF93CDB7DEB729975B
:10C74000CDBFDEBF8B0144E050E0BC01CE010196BD
:10C750000E94BFE446E050E0B801CE0101960E947D
:10C76000AFE40E94DD68009709F43FC07981AA8197
:10C77000BB811C810D812FEF35E140E050E0F901D4
:10C780006491671327C03196E491E11103C0A111B0
:10C7900021C029C0EA131EC0F9013296E491E111CB
:10C7A00003C0B11117C01FC0EB1314C0F9013396B9
:10C7B000E491E11103C011110DC015C0E1130AC0CD
:10C7C000F9013496E491E11103C0011103C00BC0DB
:10C7D000E01749F04F5F5F4F285E3F4F48175907FA
:10C7E00009F0CDCF02C0CA0102C08FEF9FEF29969A
:10C7F000CDBFDEBFDF91CF911F910F910895CF93F1
:10C80000DF93FC012189222371F1EC016196BE01C5
:10C8100088E191E20E949FE4892B39F1BE0181E118
:10C8200091E20E949FE4892B11F1BE018BE191E21C
:10C830000E949FE4892BD9F0BE018FEF90E20E9405
:10C840009FE4892BB1F0BE018EE191E20E949FE44A
:10C85000892B79F0BE018FEF91E20E949FE4892B32
:10C8600051F485E009C080E007C082E005C083E0A4
:10C8700003C084E001C081E0DF91CF910895FC0105
:10C880008FEF878314821582118612861386148691
:10C890001086118A1586178A108EA081B181109793
:10C8A00011F416820DC017968C911797873029F4D2
:10C8B00016968C918F5F868303C016968C91868323
:10C8C000CF010895EF92FF920F931F93CF93DF93C1
:10C8D000EC010C811D810E94DD680817190708F022
:10C8E0006FC00C811D81CE010E943F640C831D83AB
:10C8F0007E0181E1E80EF11CB801660F771F600F21
:10C90000711F660F771F660F771F660F771F6150C5
:10C910007A4EC7010E9447E48E01035F1F4F2C81AE
:10C920003D81B901660F771F620F731F660F771F76
:10C93000660F771F660F771F65507A4EC8010E94F9
:10C9400047E48D85882311F18C819D81FC01EE0FD8
:10C95000FF1FE80FF91FEE0FFF1FEE0FFF1FEE0F77
:10C96000FF1FEB5FF94EE491E2FF02C01D8610C08D
:10C97000F80101900020E9F7BF01601B710B605FB7
:10C980007F4F6C0F7D1FC7010E94A8E48C819D81A1
:10C99000FC01EE0FFF1FE80FF91FEE0FFF1FEE0F58
:10C9A000FF1FEE0FFF1FE75FF94E25913491CE0177
:10C9B000F901DF91CF911F910F91FF90EF901994A2
:10C9C000DF91CF911F910F91FF90EF9008958F927B
:10C9D0009F92AF92BF92CF92DF92EF92FF920F930E
:10C9E0001F93CF93DF9300D01F92CDB7DEB76C01BA
:10C9F0005C0181E1A80EB11C87E0F6018783ABEFF3
:10CA0000EA2EA5E1FA2E00E010E01DC0B701CE012C
:10CA100001960E9447E4BE016F5F7F4FC5010E94EF
:10CA20009FE4892B59F44601F9E18F0E911CF60120
:10CA3000058F168FC4010E94626464010F5F1F4F4F
:10CA4000F8E1EF0EF11CC8010E94E0688111DECF11
:10CA50002496CDBFDEBFDF91CF911F910F91FF9044
:10CA6000EF90DF90CF90BF90AF909F908F90089500
:10CA7000CF93DF9310925A3810925B38ADE1B5E353
:10CA8000E6E3F5E391E08FEFA083B18379965B96BF
:10CA9000ED93FC935C975D961D921C925E97EF015F
:10CAA0006397988322961882219788832A96188202
:10CAB000599628E3E635F20739F710923F3810927D
:10CAC0004038109236351092373510923C3587E059
:10CAD00080933D3582E790E08093473590934835C9
:10CAE0008FE495E3DF91CF9108950F931F93CF9338
:10CAF000DF930E943865EC018FEE92E180935E3AFD
:10CB000090935F3A8093A03A9093A13A8093343502
:10CB10009093353580935638909357388093583892
:10CB20009093593880935C3A90935D3A81E00E94EB
:10CB300021531C821D82CE010E946B842091A83A51
:10CB40003091A93A4091AA3A5091AB3A69857A85D9
:10CB50008B859C850E9453D8882339F0CE01DF91C4
:10CB6000CF911F910F910C94D6600E949CAB1C82B8
:10CB70001D8280E090E08E010F5E1F4F2FC06C8100
:10CB80007D819B01220F331FF901E60FF71FEE0F86
:10CB9000FF1FEE0FFF1FEE0FFF1FEB5FF94EE4913B
:10CBA000E0FF17C0620F731F660F771F660F771FB6
:10CBB000660F771F61507A4E45E050E0C8010E9431
:10CBC00066E4CE010E946B84CE010E9433606C81CA
:10CBD0007D816F5F7F4F6C837D83CB010E94E06816
:10CBE0008111CDCFDF91CF911F910F910C94DFABCD
:10CBF000EF92FF920F931F93CF93DF938C012091BD
:10CC00005A3830915B38EB0109900020E9F7219701
:10CC1000C61BD70BAE01420F531F41305240D8F410
:10CC2000F901E45AF74C7F01AE014F5F5F4FCF012E
:10CC30000E9480E440915A3850915B384F5F5F4FBB
:10CC40004C0F5D1F40935A3850935B38F801E78AC8
:10CC5000F08E80E001C08DE0DF91CF911F910F91A8
:10CC6000FF90EF900895CF93DF932EE1CFE4D5E3CB
:10CC70003F813F3F59F00A80DB81C02D209719F496
:10CC800080E090E010C0215099F7FACFBC0188E60F
:10CC900093E20E9499638C839D83019689F3CE0170
:10CCA0000E946264CE01DF91CF910895EF92FF92CE
:10CCB0000F931F93CF93DF938B012EE1CFE4D5E346
:10CCC0003F813F3F59F00A80DB81C02D209719F446
:10CCD00080E090E01DC0215099F7FACF7E0121E15C
:10CCE000E20EF11C45E050E0BC01C7010E94BFE428
:10CCF000B801CE010E94F8658111EACFB70188E63C
:10CD000093E20E9499638C839D8385E08F83CE019B
:10CD1000DF91CF911F910F91FF90EF900895209197
:10CD2000BC3A213021F42091653D213029F4BC0129
:10CD30008FEF90E20C94566680E090E00895909119
:10CD4000BC3A913019F4642F0C94E7820C94A6C479
:10CD5000CF93DF93EC018091D529811103C00E940C
:10CD600023D502C00E941FCC682F70E080E090E0C5
:10CD70000E94F3D869877A878B879C8782E08F83AC
:10CD800080E0DF91CF9108950F931F93CF93DF93AE
:10CD9000CDB7DEB7C058D109CDBFDEBFFC0161857C
:10CDA0007285838594850E94C7D88FEF860F863061
:10CDB00030F082E591E20E948F668EE62AC0609391
:10CDC000D02981E08093D129E62FF0E0EE0FFF1FFC
:10CDD000EA53FA4E659174914FE450E089E69DE381
:10CDE0000E9466E49F938F9386E894E19F938F93CC
:10CDF0008E010F5F1F4F1F930F930E9421E6C80102
:10CE00000E948F660F900F900F900F900F900F90D1
:10CE100080E0C058DF4FCDBFDEBFDF91CF911F91C3
:10CE20000F9108950F931F93CF93DF93EC018BE93C
:10CE300092E30E94F64E882329F009851A858B8596
:10CE40009C8511C023E333E34BEC51E469857A857B
:10CE50008B859C850E94F8DA8B01AB01BC01498768
:10CE60005A876B877C872C813D81F901EE0FFF1F6C
:10CE7000E20FF31FEE0FFF1FEE0FFF1FEE0FFF1F5E
:10CE8000E35FF94EA591B491A801BC014D935D9368
:10CE90006D937C931397F901EE0FFF1FE20FF31FC1
:10CEA000EE0FFF1FEE0FFF1FEE0FFF1FEA5FF94EA1
:10CEB00085919491888784E08F8380E0DF91CF9182
:10CEC0001F910F91089567E975E10C943CC563E7E4
:10CED00075E10C943CC567E375E10C943CC56CEFBF
:10CEE00074E10C943CC56FEA74E10C943CC51F934B
:10CEF000CF93DF93EC0110E08881882301F10E9439
:10CF0000386545E050E0BE0180E695E30E94BFE44D
:10CF100060E675E388E693E20E9499638093533557
:10CF2000909354358FE495E30E94626442E063E09D
:10CF300080E00E949F661F5F26961D31E9F684E01F
:10CF4000DF91CF911F910895CF93DF93CDB7DEB7D7
:10CF5000EC97CDBFDEBF8CE3E8E1F0E2DE01119695
:10CF600001900D928A95E1F7CE0101960E947767B4
:10CF7000EC96CDBFDEBFDF91CF910895CF93DF93C5
:10CF8000CDB7DEB7AA97CDBFDEBF8AE2E4E5F0E217
:10CF9000DE01119601900D928A95E1F7CE0101967E
:10CFA0000E947767AA96CDBFDEBFDF91CF9108952B
:10CFB000CF93DF93CDB7DEB76E97CDBFDEBF8EE1E7
:10CFC000EEE7F0E2DE01119601900D928A95E1F70D
:10CFD000CE0101960E9477676E96CDBFDEBFDF91CE
:10CFE000CF910895CF93DF93EC0143E759E763E7CF
:10CFF00070E0498B5A8B6B8B7C8B0E94E76442E01C
:10D0000063E080E00E949F66CE010E94D867CE0157
:10D010000E94BE6720E731E340E0298B3A8B4B8BBF
:10D02000CE010E94E76442E063E080E00E949F66D8
:10D03000CE01DF91CF910C94A467CF92DF92EF9253
:10D04000FF92CF93DF93EC01C984DA84EB84FC84F4
:10D0500020E030E040E85FE3C701B6010E9456DA05
:10D0600018161CF1C701B6010E94C7D86093D229D7
:10D0700089859A85AB85BC85BC01CD019F772CEA5B
:10D0800035EC47E257E30E9456DA18163CF460E4A8
:10D0900070E080E00E94CCCA80E008C060E870E0E8
:10D0A00080E00E94CCCA80E001C08EE6DF91CF9183
:10D0B000FF90EF90DF90CF900895CF92DF92EF92A4
:10D0C000FF92CF93DF93EC01C984DA84EB84FC8474
:10D0D00020E030E040E050E4C701B6010E9456DA9B
:10D0E00018161CF1C701B6010E94C7D86093D42955
:10D0F00089859A85AB85BC85BC01CD019F772CEADB
:10D1000035EC47E257E30E9456DA18163CF464E027
:10D1100070E080E00E94CCCA80E008C068E070E067
:10D1200080E00E94CCCA80E001C08EE6DF91CF9102
:10D13000FF90EF90DF90CF900895CF92DF92EF9223
:10D14000FF92CF93DF93EC01C984DA84EB84FC84F3
:10D1500020E030E040E85FE3C701B6010E9456DA04
:10D1600018161CF1C701B6010E94C7D86093D329D5
:10D1700089859A85AB85BC85BC01CD019F772CEA5A
:10D1800035EC47E257E30E9456DA18163CF460E1AA
:10D1900070E080E00E94CCCA80E008C060E270E0ED
:10D1A00080E00E94CCCA80E001C08EE6DF91CF9182
:10D1B000FF90EF90DF90CF9008958CE891E0089574
:10D1C00021E08334914008F020E0822F08959C01F3
:10D1D0002F55314081E02932310508F080E0089573
:10D1E00021E08036914008F020E0822F0895CF9210
:10D1F000DF92EF92FF92CF93DF93EC01C984DA8440
:10D20000EB84FC84A7019601C701B6010E9419DCDA
:10D2100081113CC0E894F7F82FEF3FEF4FE75FE74D
:10D22000C701B6010E9419DC81110AC02FEF3FEF40
:10D230004FE75FE7C701B6010E9453D8181634F1D3
:10D240008C819D81FC01EE0FFF1FE80FF91FEE0F8F
:10D25000FF1FEE0FFF1FEE0FFF1FEB5FF94EE49174
:10D26000E3FF14C08BE992E30E94F64E81110EC0D9
:10D2700025E832E441E25DE369857A858B859C850A
:10D280000E94F8DA69877A878B879C87DF91CF9134
:10D29000FF90EF90DF90CF9008958091D12988235F
:10D2A00049F01092D1296091D02980E00E94D4CA1F
:10D2B00080E0089583E00895CF93DF93E091DB3A17
:10D2C000F091DC3A04C0E093DB3AF093DC3AEF01F2
:10D2D0008191982F9D7F9032B1F38930A1F34FE473
:10D2E00050E0BE018FED9CE30E94BFE468816111B4
:10D2F00005C08091BC3A81115DC028C0613221F423
:10D30000DF91CF910C94A259653221F4DF91CF9136
:10D310000C94A6596E3721F4DF91CF910C94AA5941
:10D320006B3741F481E08093BC3ACE01DF91CF911D
:10D330000C94E47D70E082E891E20E9494E4892BF1
:10D3400059F01092BC3ACE010E94FEC06FED7CE312
:10D35000DF91CF910C943EC28091BC3A811109C0FB
:10D36000CE010E945F746FED7CE3DF91CF910C944E
:10D370003EC247EF50E0BE018FED9AE30E94BFE44A
:10D380008FED9AE39F938F9387E891E29F938F931A
:10D39000DF93CF930E94F8E50F900F900F900F90BE
:10D3A0000F900F908091DB3A9091DC3ADF91CF9112
:10D3B0000C94E47DDF91CF910895FF920F931F931A
:10D3C000CF93DF931F921F92CDB7DEB7F82EE2EA1C
:10D3D000FAE32FE832E0DF01C9011D920197E9F776
:10D3E0002FEE32E12083318320932F3D3093303D67
:10D3F00006EF18E82CED33E40093A83A1093A93A0D
:10D400002093AA3A3093AB3A0CEE11E528E73FE3BC
:10D410000093AC3A1093AD3A2093AE3A3093AF3AC2
:10D4200000E010E020EA30E40093B03A1093B13A03
:10D430002093B23A3093B33A00E010E020E83FE3A3
:10D440000093B43A1093B53A2093B63A3093B73A72
:10D4500083E08093BE3A8F2D4A8369830E94E4CA99
:10D460006981862F0E94EFCA4A81842F0E94FACADE
:10D47000F092CF29F092CD290F900F90DF91CF91AC
:10D480001F910F91FF900895CF93DF931F921F92EA
:10D49000CDB7DEB780E6F82E01E010E00E944C7CAC
:10D4A0008230E1F30E94537C8230C1F30E94D54E5A
:10D4B000863009F0C6C00E94C8C88090C43A9090D7
:10D4C000C53AA090C63AB090C73A86169706A80605
:10D4D000B90620F70E94C8C86C597F4F8F4F9F4FE5
:10D4E0006093C43A7093C53A8093C63A9093C73A12
:10D4F0000E94C27BD3CF0E94D1BF882329F08CEC3D
:10D500000E940D53823051F20E94FB59823031F259
:10D510000E9424A1823011F20E945E618093B93D85
:10D5200081112EC08091A23A9091A33A8F3E9241F0
:10D5300009F08DC080912F3D9091303D8F3E9241FA
:10D5400009F085C08AC00E9440858093B93D811151
:10D5500017C00E94F5B58093B93D811111C00E949A
:10D560002A748093B93D81110BC00E94E6C9809353
:10D57000B93D811105C00E948EB6823031F48ECF44
:10D580000E940D538230B9F789CF0E94C7AD823017
:10D5900009F484CF0E9433AF823009F47FCF0E9418
:10D5A000FAAF823009F47ACF09831A836DED7AE3FA
:10D5B000CE0101960E9409CB8093DB3A9093DC3A2E
:10D5C000892B11F00E945C690E94838F823009F4DC
:10D5D00065CF0E945F6F823009F460CF0E941E7297
:10D5E000823009F45BCF0E940574823009F456CF73
:10D5F0000E94A450823009F44FCF0E94F5858430F8
:10D60000B0F54ACF8091BE3A843038F484E08093FC
:10D61000BE3A0E94A6590E94A1AB83E090E08983A4
:10D620009A836DED7AE3CE0101960E9409CB809337
:10D63000DB3A9093DC3A892B09F42ECF0E945C6987
:10D640002BCF0E94D54E823009F45ECF54CFF0929A
:10D65000B93D80E60E940D5395CF1092B93D0E94CE
:10D66000D2528093B93D882309F46DCF89CF809140
:10D67000E5289091E6280E9497D3682F70E080E01B
:10D6800090E00E94F5D823E333E34BE451E40E9499
:10D6900056DA87FF01CF0E944D69823009F0B2CF80
:10D6A000FBCE8091CF298093CD2908958093CD29F9
:10D6B00008958093CE290895CF93C82F8091B323E6
:10D6C000882379F040E050E0BA018C2F0E941E546C
:10D6D000EC2FFF27E7FDF095E059FD4C81E08083BA
:10D6E0000AC06C2F88E996E50E941B50AB01BC0173
:10D6F0008C2F0E941E544091DA235091DB236091BD
:10D70000DC237091DD238C2F0E944F5D85E29DE626
:10D710008093B4239093B52382E0CF910895CF9264
:10D72000DF92EF92FF920F931F93CF93DF93CDB7CA
:10D73000DEB7E097CDBFDEBF98E17E01A9E1EA0E3A
:10D74000F11CF701A92F1192AA95E9F7FE01319674
:10D750006F0111929A95E9F7F60194E08902E00DC4
:10D76000F11D1124408F518F628F738F80E090E004
:10D77000A0E8BFE380839183A283B3830093D83270
:10D780001093D9322093DA323093DB320E947886BC
:10D790000E94AA59B601C7010E9474578093B93DEF
:10D7A000811101C082E0E096CDBFDEBFDF91CF9155
:10D7B0001F910F91FF90EF90DF90CF9008950F93FE
:10D7C0001F93E091AD23FF27E7FDF095EB5BFF4C46
:10D7D0009381913099F40091BE231091BF23209141
:10D7E000C0233091C1234091C6235091C72360913B
:10D7F000C8237091C9230E948F6B1DC0E091AE2396
:10D80000FF27E7FDF095EB5BFF4C9381913099F496
:10D810000091BE231091BF232091C0233091C123DA
:10D820004091C6235091C7236091C8237091C923AA
:10D8300070580E948F6B85E29CE68093B42390938E
:10D84000B52382E01F910F9108950F931F93CF93FB
:10D85000C82F85E3C802F0011124EF5BFE4C408124
:10D860005181628173818C2F0E944F5D0091BE2394
:10D870001091BF232091C0233091C1234091BA233E
:10D880005091BB236091BC237091BD238C2F0E94CB
:10D890008F6B84EB9CE68093B4239093B52382E056
:10D8A000CF911F910F9108950F931F930091BE2365
:10D8B0001091BF232091C0233091C1234091CA23EE
:10D8C0005091CB236091CC237091CD230E948F6B1C
:10D8D0008CE59BE68093B4239093B52382E01F915F
:10D8E0000F9108950E9478868091D3230E948753D8
:10D8F0008091D2230E9421538091D4230E942553EA
:10D900008091D5230E9460578091D6239091D72390
:10D91000A091D823B091D9238093D8329093D93253
:10D92000A093DA32B093DB3264E08BE992E30E9499
:10D93000134F0E94575A10926C3280E00895CF9393
:10D94000C82F4091DA235091DB236091DC23709142
:10D95000DD230E944F5D8C2F0E94726C80E00E943C
:10D9600095AD80EFCF9108950F931F93E091AD2374
:10D97000FF27E7FDF095EB5BFF4C9381913039F089
:10D980008FE99CE68093B4239093B52318C000914F
:10D99000C2231091C3232091C4233091C523409109
:10D9A000C6235091C7236091C8237091C9230E9458
:10D9B0008F6B84E59CE68093B4239093B52382E03B
:10D9C0001F910F910895FF920F931F93CF93DF93B1
:10D9D000CDB7DEB7C058D109CDBFDEBFF82E0E944B
:10D9E00038658EEFF81205C084E991E20E948F66D7
:10D9F00019C08F2D0E94EC5A1F928F932BE13BE3AD
:10DA00003F932F938E010F5F1F4F1F930F930E9421
:10DA100021E6C8010E948F660F900F900F900F9023
:10DA20000F900F9042E062E080EF0E949F668F2D82
:10DA30000E94726C80EFC058DF4FCDBFDEBFDF9118
:10DA4000CF911F910F91FF9008954F925F926F9227
:10DA50007F929F92AF92BF92CF92DF92EF92FF920E
:10DA60000F931F93CF93DF938F3F09F045C02CEAAC
:10DA700035EC47E257E36091D1337091D233809116
:10DA8000D3339091D4330E9456DA18160CF469C13E
:10DA90002CEA35EC47E257E36091C9337091CA3301
:10DAA0008091CB339091CC330E9456DA18160CF447
:10DAB0005DC12CEA35EC47E257E36091CD337091BC
:10DAC000CE338091CF339091D0330E9456DA18161E
:10DAD0000CF455C12CEA35EC47E257E36091D5339D
:10DAE0007091D6338091D7339091D8330E9456DA13
:10DAF00018160CF43FC171C18230A1F52CEA35EC47
:10DB000047E257E36091C9337091CA338091CB33B8
:10DB10009091CC330E9456DA18160CF427C12CEAE7
:10DB200035EC47E257E36091CD337091CE3380916D
:10DB3000CF339091D0330E9456DA18160CF41FC1DF
:10DB40002CEA35EC47E257E36091D5337091D63338
:10DB50008091D7339091D8330E9456DA18160CF47E
:10DB600009C131C18823D9F2813051F32CC17E0122
:10DB70008DEEE80EF11CF70180819181A281B381C5
:10DB8000BC01CD019F772CEA35EC47E257E30E94B8
:10DB900053D887FD46C06E01F1EFCF0ED11CF601C0
:10DBA000408051806280738020E030E0A901C30191
:10DBB000B2010E9453D887FD34C0FE01EF52FF4FDF
:10DBC00020813181428153813497608171818281CA
:10DBD00093810E94E4D69B01AC015F77C301B2013F
:10DBE0000E94E5D62B013C019F772CEA35EC47E2F9
:10DBF00057E30E9453D887FD14C0AB2CAA0C8A2D82
:10DC00000E94CBBF8093AB23992493949A0C892DC7
:10DC10000E94CBBF8093AC232091AB23822780FD51
:10DC200002C08B2DDBC0B092AA23F80180819181C4
:10DC3000A281B381BF778093BE239093BF23A0932B
:10DC4000C023B093C123F701408151816281738168
:10DC50007F774093C2235093C3236093C423709370
:10DC6000C52320FF2DC0A092AD239092AE2377FA5A
:10DC7000709477F870944092BA235092BB236092CC
:10DC8000BC237092BD23F60180819181A281B38172
:10DC90008093C6239093C723A093C823B093C9232E
:10DCA000CB50DF4F88819981AA81BB818093CA23A1
:10DCB0009093CB23A093CC23B093CD238A2D2AC05D
:10DCC0009092AD23A092AE234092BA235092BB23F0
:10DCD0006092BC237092BD23F60180819181A28164
:10DCE000B381B0588093C6239093C723A093C823D1
:10DCF000B093C923CB50DF4F88819981AA81BB8122
:10DD0000B0588093CA239093CB23A093CC23B09395
:10DD1000CD23892D0E94CBBF8D7F813039F085E2E4
:10DD20009DE68093B4239093B52369C08091AE2380
:10DD30000E94CBBF811103C08FEF8093AE238B2D48
:10DD40000E94445D6093DA237093DB238093DC238D
:10DD50009093DD238FED9BE68093B4239093B523BE
:10DD60004EC082E090E032E0B32E0DC080E090E043
:10DD7000B12C09C083E090E023E0B22E04C081E022
:10DD800090E0BB24B394FC01E059FD4C108225E3E4
:10DD9000289FE001299FD00D1124C859DF4C8E0126
:10DDA00007511F4FF80180819181A281B381BC018D
:10DDB000CD019F772CEA35EC47E257E30E9453D818
:10DDC00087FFD5CE2ECF81E080936F3282E79CE62D
:10DDD0008093B4239093B52312C08EEFDF91CF913F
:10DDE0001F910F91FF90EF90DF90CF90BF90AF9079
:10DDF0009F907F906F905F904F900C94E36C82E0C7
:10DE0000DF91CF911F910F91FF90EF90DF90CF9016
:10DE1000BF90AF909F907F906F905F904F900895CC
:10DE2000CF93DF93C9E9D2E3888199810E94F64EAE
:10DE30008093D223888199810E94F14E8093D323CD
:10DE4000888199810E94004F8093D4238881998191
:10DE50000E94054F8093D523888199810E940C4FA1
:10DE60006093D6237093D7238093D8239093D9239C
:10DE700081E00E94215381E00E94255380E00E94AE
:10DE8000875381E00E94605781E08093B3238FEF36
:10DE90008093AA2385E29DE68093B4239093B523D3
:10DEA00083E080936C3210926F3280E0DF91CF91EB
:10DEB00008950E94106F1092B32380E0089580911E
:10DEC0006C32833059F40E940A4F813049F0E0915E
:10DED000B423F091B5238091AA23199483E0089587
:10DEE00082E008958AE79FE68093EF239093F023E2
:10DEF00082E008952F923F924F925F926F927F92AD
:10DF00008F929F92AF92BF92CF92DF92EF92FF9249
:10DF10000F931F93CF93DF93CDB7DEB7CA54D109C8
:10DF2000CDBFDEBF98E19E01275E3F4F29AB3AABE4
:10DF3000D901E92F1D92EA95E9F728513109190114
:10DF4000D9011D929A95E9F724E08202F00111248B
:10DF50002B96EEAFFFAF2B97E20DF31D80E090E024
:10DF6000A0E8BFE380839183A283B383C090E723BB
:10DF7000D090E823E090E923F090EA234090E32357
:10DF80005090E4236090E5237090E6238090DF2397
:10DF90009090E023A090E123B090E223A5019401AA
:10DFA000C301B2010E9453D818165CF080E090E0E3
:10DFB000A0E8BFE329968CAF9DAFAEAFBFAF299766
:10DFC0000AC080E090E0A0E8BFEB29968CAF9DAF3F
:10DFD000AEAFBFAF2997A3019201C501B4010E9462
:10DFE000E4D60E94C2D89B0177FF04C022273327C2
:10DFF000261B370BB901882777FD8095982F0E9443
:10E00000F5D825966CAF7DAF8EAF9FAF2597C092A8
:10E01000D832D092D932E092DA32F092DB320E94DA
:10E0200078860E94AA5920E030E040E050E425962E
:10E030006CAD7DAD8EAD9FAD25970E9456DA18165A
:10E040006CF08091EB239091EC23A091ED23B091A3
:10E05000EE238BAF9CAFADAFBEAFDBC02AE037ED98
:10E0600043E25CE325966CAD7DAD8EAD9FAD25970B
:10E070000E9456DA18162CF709E110E08AE0882E83
:10E0800087ED982E83E2A82E8CE3B82E412C512CDC
:10E0900032012B96AEADBFAD2B97A20DB31D589696
:10E0A0002196AEAFBFAF21974BAA5CAA6DAA7EAAFC
:10E0B0008FAA98AEA9AEBAAE29962CAD3DAD4EADA5
:10E0C0005FAD29976FA978AD89AD9AAD0E94F8DA56
:10E0D0009B01AC016091E3237091E4238091E523DF
:10E0E0009091E6230E94E5D62196EEADFFAD2197F3
:10E0F0006083718382839383C092D832D092D93265
:10E10000E092DA32F092DB32B101CE0149960E9400
:10E1100074578093B93D8111AAC020E030E040E8F7
:10E120005FE36BA97CA98DA99EA90E94E5D66BAB84
:10E130007CAB8DAB9EAB20E030E048EC51E40E941C
:10E140005AD89B01AC0160E070E080E291E40E944B
:10E150005BDB2B013C018091EB239091EC23A091A0
:10E16000ED23B091EE238BAF9CAFADAFBEAFC090AF
:10E17000E723D090E823E090E923F090EA23A70179
:10E180009601BC01CD010E94E4D64B015C0120E068
:10E1900030E040E251E4C301B2010E945AD89B0131
:10E1A000AC01C501B4010E94F8DA9B01AC01C701C2
:10E1B000B6010E94E5D66B017C012BA93CA94DA9B3
:10E1C0005EA9CA01B9010E94E5D620E030E048EC22
:10E1D00051E40E945AD89B01AC016FA978AD89AD7A
:10E1E0009AAD0E94E5D66FAB78AF89AF9AAF9B012D
:10E1F000AC0125966CAD7DAD8EAD9FAD25970E948F
:10E2000056DA181634F4015011090115110509F0F8
:10E2100053CF8BAD9CADADADBEAD8093D832909356
:10E22000D932A093DA32B093DB322B96EEADFFAD4C
:10E230002B97E20DF31D8091DF239091E023A091B5
:10E24000E123B091E223808F918FA28FB38FB10130
:10E25000CE0149960E9474578093B93D811107C041
:10E260008EE491E78093EF239093F02382E0C65BE6
:10E27000DF4FCDBFDEBFDF91CF911F910F91FF9098
:10E28000EF90DF90CF90BF90AF909F908F907F9056
:10E290006F905F904F903F902F900895CF93DF93B2
:10E2A0001F92CDB7DEB789830E9478864091F9230B
:10E2B0005091FA236091FB237091FC2389810E9485
:10E2C0004F5D8091F6230E9487538091F5230E9431
:10E2D00021538091F7230E9425538091F8230E94B7
:10E2E00060578091F1239091F223A091F323B09194
:10E2F000F4238093D8329093D932A093DA32B0933A
:10E30000DB3264E08BE992E30E94134F0E94575A7C
:10E3100010926C3280EC91E20E94CBE580E00F908D
:10E32000DF91CF9108950F931F93CF93C82F09E9E1
:10E3300012E3F801808191810E94F64E8093F523CB
:10E34000F801808191810E94F14E8093F623F801BB
:10E35000808191810E94004F8093F723F801808192
:10E3600091810E94054F8093F823F801808191816B
:10E370000E940C4F6093F1237093F2238093F32358
:10E380009093F4238C2F0E94445D6093F923709343
:10E39000FA238093FB239093FC2381E00E94215376
:10E3A00080E00E94255380E00E94875381E00E9414
:10E3B000605740E050E060E271E44093E7235093FF
:10E3C000E8236093E9237093EA2385E3C89FF00173
:10E3D0001124EF5CFE4C4081518162817381409336
:10E3E000EB235093EC236093ED237093EE236C2F7B
:10E3F00088E996E50E9408506093E3237093E42334
:10E400008093E5239093E6230E941C5E6093DF23B4
:10E410007093E0238093E1239093E223C093DE2363
:10E4200082E79FE68093EF239093F02384E080932C
:10E430006C3280E0CF911F910F91089580916C32E2
:10E44000843059F40E940A4F813049F0E091EF2363
:10E45000F091F0238091DE23199483E0089582E007
:10E460000895E091FF23F0E0EB5BFF4C838188236C
:10E4700041F08CE492E78093FD239093FE2382E0A9
:10E4800008956CE474E284E394E20E9474578093EC
:10E49000B93D882371F308951F93CF93DF93E091E3
:10E4A000FF23F0E0EB5BFF4C81E09381913009F0BA
:10E4B00080E080937632C7E7D2E310E0612F88E9ED
:10E4C00096E50E941B50AB01BC01812F0E941E5497
:10E4D000612F8091993290919A320E9408506993ED
:10E4E0007993899399931F5F163041F78AEC91E2F3
:10E4F0000E94E47D8AEB92E78093FD239093FE23B4
:10E5000082E0DF91CF911F9108951F93CF93DF9306
:10E510000E9478868091002480934530E091FF230B
:10E52000F0E080910124EB5BFF4C83870E94E8BF01
:10E53000C4E0D4E210E04991599169917991812F19
:10E540000E944F5D1F5F1630B1F7809103240E9437
:10E550008753809102240E94255364E08BE992E363
:10E560000E94134F0E94575A10926C32DF91CF9144
:10E570001F9108950E94857280E008950F931F9364
:10E58000CF93DF93CDB7DEB7C058D109CDBFDEBF83
:10E59000182F0E9438651E3F29F487ED91E20E94F2
:10E5A0008F6619C0812F0E94EC5A1F928F9389E4C5
:10E5B0009BE39F938F938E010F5F1F4F1F930F93CA
:10E5C0000E9421E6C8010E948F660F900F900F9065
:10E5D0000F900F900F9042E062E08AEF0E949F66DA
:10E5E0000E9485728AEFC058DF4FCDBFDEBFDF913A
:10E5F000CF911F910F910895FF920F931F93CF9387
:10E60000DF931092763282E080936C3204E014E261
:10E61000C1E4D1E3F12C8F2D0E94445DF801619398
:10E620007193819391938F01488159816A817B8194
:10E630008F2D0E944F5D6F2D8091993290919A326B
:10E640000E940850F801648B758B868B978BF3942E
:10E65000E596F6E0FF12DFCF64E374E28CE194E22A
:10E660000E94CBC52AE43CE042E85EE30E9453D816
:10E6700087FF03C08EEF0E94BE72C8E2D4E213E0AF
:10E6800069917991899199912C893D894E895F8908
:10E690000E94E4D69F772CEA35EC47E257E30E94CC
:10E6A00056DA18161CF4812F0E94BE721F5F1630B6
:10E6B00039F784E08093FF238091543080930124C4
:10E6C00081E08093543080914530809300241092F3
:10E6D00045300E94E8BF8091993290919A320E9411
:10E6E000F14E809303248091993290919A320E9446
:10E6F000004F8093022480E00E94255380E00E9416
:10E70000875380E00E94DBB181E392E78093FD2391
:10E710009093FE2382E0DF91CF911F910F91FF90A4
:10E7200008950F931F93CF93DF938C01EB0180919A
:10E73000E432882399F08091D8329091D932A09117
:10E74000DA32B091DB32BC01CD019F772CEA35EC97
:10E7500047E257E30E9453D887FD4FC088819981D3
:10E76000AA81BB81BC01CD019F772CEA35EC47E241
:10E7700057E30E9456DA1816F4F48C819D81AE811D
:10E78000BF81BC01CD019F772CEA35EC47E257E30E
:10E790000E9456DA18167CF488859985AA85BB856F
:10E7A000BC01CD019F772CEA35EC47E257E30E948C
:10E7B00056DA181624F188E1F801A4E3B4E20190D6
:10E7C0000D928A95E1F788E1FE01ACE4B4E2019094
:10E7D0000D928A95E1F788E1E7E7F2E3DF011D9208
:10E7E0008A95E9F782E0809376328CEF92E7809306
:10E7F000FD239093FE2380E003C08EE801C086E8ED
:10E80000DF91CF911F910F91089580916C328230EA
:10E8100021F080917632823049F40E940A4F813093
:10E8200039F0E091FD23F091FE23199483E00895DF
:10E8300082E00895E1E3FDE380E2DF011D928A9525
:10E84000E9F78FEE92E180934F3D9093503D8083A6
:10E850009183089580914F3D9091503D8F3E92411C
:10E8600011F08CE508958091313D9091323D8F3EBD
:10E870009241B9F780E00895CF93DF93C82FCB0181
:10E88000BA010E94A7DB27E0C29FE0011124CF5C00
:10E89000D24C0E94C2D86D837E838F839887DF918C
:10E8A000CF91089597E0899FF0011124EF5CF24C1D
:10E8B00065817681878190850E94F5D808952F9291
:10E8C0003F924F925F926F927F928F929F92AF9200
:10E8D000BF92CF92DF92EF92FF920F931F93CF934D
:10E8E000DF93CDB7DEB72797CDBFDEBF8C011B828C
:10E8F00080916B32823009F4A6C6D801BC90B11069
:10E90000CFC680E06E01B3E0CB0ED11C3DC0F60156
:10E910008081811108C0B72CD7011C926E01B3E031
:10E92000CB0ED11CBAC6883239F4B72CF70110824D
:10E93000FFEFCF1ADF0AB1C68B33B9F3A82EB12C83
:10E94000C5010E941BE4892B39F4B50181E092E2F4
:10E950000E9494E4892B51F047018FEF881A980A9E
:10E96000C5010E943FE4D7018C937401BFEFCB1A1D
:10E97000DB0AF70180818111CACFB72CD8018C91B5
:10E980006E01B3E0CB0ED11CF8011CC08E32E1F059
:10E9900090E0C0970A9790F08181803391F4828152
:10E9A00090E0C0970A9760F4DF01119611968C9160
:10E9B00011978D938111FACF808104C0818101C0AC
:10E9C00080E331968111E2CFF601A080A11007C04B
:10E9D00036C0D6011196AC90BFEFCB1ADB0A760198
:10E9E0008A2C912CC4010E942FE4892B91F7C40139
:10E9F0000E9437E48D369105A1F4F601818190E003
:10EA00000E9437E48337910561F4D60112968C9108
:10EA100090E00E9437E48736910519F4F6013396A9
:10EA200002C0FE013396AA2061F08A2DD7018932F7
:10EA300009F41C9211968C918111F9CF02C0FE014C
:10EA40003396BFE2BB1609F400C68081882319F013
:10EA5000CF010E949D5980E1E1E5FDE3DF011D92B8
:10EA60008A95E9F78AE5E2ECF3E3DF01982F1D923E
:10EA70009A95E9F7E8E6F3E3DF011D928A95E9F755
:10EA80008BE992E30E94EE4E80936933812C912CA6
:10EA900080E8A82E8FE3B82E5524539492E0492E97
:10EAA00024E0322EBDC3C701B6010E94C7D8862F0D
:10EAB00090E08F35910508F0CCC5FC01EC50FF4F7C
:10EAC0000C949EE0109269335092C3338091523D72
:10EAD0008F5F8093523DA4C3509269335092C333E9
:10EAE0008091523D8F5F8093523D9AC3409269332B
:10EAF0005092C3338091523D8F5F8093523D90C3BB
:10EB000083E0809369335092C3338091523D8F5F8D
:10EB10008093523D85C38DE0809368335092C23319
:10EB20007FC388E0B2C0109298335092F233809144
:10EB3000533D8F5F8093533D73C3509298335092EF
:10EB4000F2338091533D8F5F8093533D69C3409270
:10EB500098335092F2338091533D8F5F8093533DB1
:10EB60005FC3109299335092F3338091563D8F5F7B
:10EB70008093563D55C3509299335092F333809110
:10EB8000563D8F5F8093563D4BC3C701B6010E942F
:10EB900012DC6C837D838E839F8320E030E040E233
:10EBA00051E4C701B6010E94F8DA6B017C0120E054
:10EBB00030E040E251E46C817D818E819F810E9432
:10EBC000F8DA9B01AC01C701B6010E94E4D60E94AD
:10EBD000C7D8623001F128F4662341F0613089F032
:10EBE00038C56330E9F0643001F133C5B5E0B09366
:10EBF00068335092C2338091513D8F5F8093513D75
:10EC00000FC3309268336093C2338091513D8F5F60
:10EC10008093513D05C3509268335092C23300C374
:10EC2000409268335092C233FBC283E080936833D2
:10EC30005092C233F5C2C701B6010E9412DC6C8348
:10EC40007D838E839F8320E030E040E251E4C70162
:10EC5000B6010E94F8DA6B017C0120E030E040E26E
:10EC600051E46C817D818E819F810E94F8DA9B0145
:10EC7000AC01C701B6010E94E4D60E94C7D8662342
:10EC800019F0613061F0E5C487E0809368335092F9
:10EC9000C2338091513D8F5F8093513DC1C2E6E008
:10ECA000E09368336093C2338091513D8F5F8093CE
:10ECB000513DB6C2C701B6010E9412DC6C837D8350
:10ECC0008E839F8320E030E040E251E4C701B6012B
:10ECD0000E94F8DA6B017C0120E030E040E251E470
:10ECE0006C817D818E819F810E94F8DA9B01AC014D
:10ECF000C701B6010E94E4D60E94C7D8623009F06D
:10ED0000A8C48EE0809368335092C23389C2509277
:10ED10009B335092F53384C250929A335092F4331D
:10ED200080915A3D8F5F80935A3D7AC240929A33C8
:10ED30005092F43380915A3D8F5F80935A3D70C258
:10ED400083E016C030929A335092F43380915A3D4A
:10ED50008F5F80935A3D64C2F5E0F0939A335092EE
:10ED6000F43380915A3D8F5F80935A3D59C286E0BB
:10ED700080939A335092F43380915A3D8F5F809301
:10ED80005A3D4EC2C701B6010E9412DC6C837D83DE
:10ED90008E839F8320E030E040E251E4C701B6015A
:10EDA0000E94F8DA6B017C0120E030E040E251E49F
:10EDB0006C817D818E819F810E94F8DA9B01AC017C
:10EDC000C701B6010E94E4D60E94C7D8662319F095
:10EDD000613059F03EC410929D335092F7338091C8
:10EDE0005B3D8F5F80935B3D1BC260939D3360935F
:10EDF000F73380915B3D8F5F80935B3D11C2409202
:10EE00009D335092F73380915B3D8F5F80935B3DE4
:10EE100007C2309269335092C3338091523D8F5F65
:10EE20008093523DFDC110929E335092F8338091F1
:10EE3000543D8F5F8093543DF3C150929E33509266
:10EE4000F8338091543D8F5F8093543DE9C1C701F1
:10EE5000B6010E9412DC6C837D838E839F8320E049
:10EE600030E040E251E4C701B6010E94F8DA6B01DC
:10EE70007C0120E030E040E251E46C817D818E81B4
:10EE80009F810E94F8DA9B01AC01C701B6010E9484
:10EE9000E4D60E94C7D8613089F028F06230A1F032
:10EEA0006330C1F0D6C399E0909368335092C23377
:10EEB0008091513D8F5F8093513DB2C1AAE0A093F4
:10EEC00068336093C233ACC1BBE0B09368335092F7
:10EED000C233A6C1ECE0E09368335092C233A0C1C4
:10EEE000109293335092ED338091553D8F5F809314
:10EEF000553D96C1509293335092ED338091553DDC
:10EF00008F5F8093553D8CC1C701B6010E94C7D861
:10EF1000862F90E08D33910508F099C3FC01ED5ADE
:10EF2000FE4F0C949EE010926A335092C43380914D
:10EF30005C3D8F5F80935C3D73C150926A33509209
:10EF4000C43380915C3D8F5F80935C3D69C150927A
:10EF5000A4335092FE3380915E3D8F5F80935E3D7F
:10EF60005FC14092A4335092FE3380915E3D8F5F2B
:10EF700080935E3D55C11092A4335092FE33809130
:10EF80005E3D8F5F80935E3D4BC15092A1335092A6
:10EF9000FB3346C15092A2335092FC3380915F3DC7
:10EFA0008F5F80935F3D3CC15092A3335092FD33FD
:10EFB00080915F3D8F5F80935F3D32C11092A3339C
:10EFC0005092FD3380915F3D8F5F80935F3D28C1FC
:10EFD000509296335092F0338091603D8F5F8093D2
:10EFE000603D1EC1109296335092F0338091603D87
:10EFF0008F5F8093603D14C1509294335092EE33F2
:10F000008091603D8F5F8093603D0AC15092AD3327
:10F01000509207348091603D8F5F8093603D00C1C6
:10F02000C701B6010E9412DC0E94C7D86093A033CA
:10F030005092FA33F5C0C0928733D0928833E09271
:10F040008933F0928A338092E1339092E233A09236
:10F05000E333B092E433E4C0C092AE33D092AF3326
:10F06000E092B033F092B133809208349092093438
:10F07000A0920A34B0920B34D3C0C092A533D09280
:10F08000A633E092A733F092A8338092FF33909298
:10F090000034A0920134B0920234C2C0C0926F33E7
:10F0A000D0927033E0927133F09272338092C93310
:10F0B0009092CA33A092CB33B092CC33B1C0C092FD
:10F0C0007333D0927433E0927533F092763380923A
:10F0D000CD339092CE33A092CF33B092D033A0C034
:10F0E000C0927733D0927833E0927933F0927A33CA
:10F0F0008092D1339092D233A092D333B092D43352
:10F100008FC0C0927B33D0927C33E0927D33F092FB
:10F110007E338092D5339092D633A092D733B0927B
:10F12000D8337EC0C0927F33D0928033E092813357
:10F13000F09282338092D9339092DA33A092DB330B
:10F14000B092DC336DC0C0928333D0928433E092AE
:10F150008533F09286338092DD339092DE33A09235
:10F16000DF33B092E0335CC0C092B633D092B73395
:10F17000E092B833F092B933809210349092113407
:10F18000A0921234B09213344BC0C092BA33D092D2
:10F19000BB33E092BC33F092BD3380921434909232
:10F1A0001534A0921634B09217343AC0C092BE33D0
:10F1B000D092BF33E092C033F092C13380921834C2
:10F1C00090921934A0921A34B0921B3429C0C09284
:10F1D000B233D092B333E092B433F092B53380922D
:10F1E0000C3490920D34A0920E34B0920F3418C0AB
:10F1F000C701B6010E94C7D860936B3370936C331C
:10F2000080936D3390936E3381E090E0A0E0B0E0A6
:10F210008093C5339093C633A093C733B093C8335C
:10F22000D8012C90222009F416C2822D90E00E9471
:10F2300026E4892B09F421C23801BFEF6B1A7B0A3F
:10F24000F8018181803349F48281883531F40E5F81
:10F250001F4FC12CD12C760114C2BE016F5F7F4FAE
:10F26000C3010E94BEE06B017C0109811A81601616
:10F27000710609F006C203C2809193330E94605761
:10F28000182F01C010E06091E1337091E23380915A
:10F29000E3339091E4330E94C7D8662359F060911C
:10F2A0008733709188338091893390918A330E949B
:10F2B0002F57182F6091E5337091E6338091E73333
:10F2C0009091E8330E94C7D8662371F060918B3328
:10F2D00070918C3380918D3390918E330E94C7D87A
:10F2E000862F0E940B59182F6091E9337091EA33F1
:10F2F0008091EB339091EC330E94C7D8662371F074
:10F3000060918F33709190338091913390919233CB
:10F310000E94C7D8862F0E944A59182F6091FF3348
:10F320007091003480910134909102340E94C7D8CA
:10F33000662359F06091A5337091A6338091A7336D
:10F340009091A8330E940FB2182F609103347091EE
:10F35000043480910534909106340E94C7D8662306
:10F3600071F06091A9337091AA338091AB33909181
:10F37000AC330E94C7D8862F0E948959182F8091DC
:10F38000FA33882329F08091A0330E94C857182FA0
:10F390008091FB33882329F08091A1330E94FC5790
:10F3A000182F8091FE33882329F08091A4330E9486
:10F3B000DBB1182F8091FC33882329F08091A23390
:10F3C0000E943158182F8091FD33882329F08091B5
:10F3D000A3330E946558182F8091EE33882329F0BB
:10F3E000809194330E94E058182F8091EF33882346
:10F3F00029F0809195330E941F59182F809107346E
:10F40000882329F08091AD330E945E59182F809196
:10F41000F033882329F0809196330E94D858182F12
:10F42000809168338D3029F08091F2338823A9F0E0
:10F430000FC06091AE337091AF338091B033909133
:10F44000B1330E9468578093B93D882369F32DC179
:10F45000809198330E941D53182F8091F333882395
:10F4600029F0809199330E942153182F8091F43311
:10F47000882329F080919A330E948753182F809116
:10F48000F733882329F080919D330E946457182F09
:10F490008091F833882329F080919E330E94255370
:10F4A000182F4091683350E04F30510508F0B4C038
:10F4B000FA01E057FE4F0C949EE00E94B156182FBF
:10F4C000ABC069EC73E38FE693E30E94BC56182F40
:10F4D000A3C00E94F056182F9FC069EC73E38FE61B
:10F4E00093E30E94FB56182F97C00E94106F182FAD
:10F4F00093C069EC73E38FE693E30E944E54182F98
:10F500008BC00E94596F182F87C069EC73E38FE698
:10F5100093E30E949173182F7FC06091AE33709176
:10F52000AF338091B0339091B1330E94C7D8862F0A
:10F5300049EC53E36FE673E30E942953182F6CC024
:10F5400069EC73E38FE693E30E94F854182F64C0CC
:10F550000E94AB55182F60C00E941256182F5CC035
:10F560000E944956182F58C060919B338BE992E353
:10F570000E94894F80916933843038F48230D8F406
:10F58000882349F0813079F047C0843009F044C0C5
:10F5900080939F3241C069EC73E38FE693E30E944E
:10F5A0008156182F39C069EC73E38FE693E30E940C
:10F5B0007457182F31C0A090BE33B090BF33C090A5
:10F5C000C033D090C133E090BA33F090BB33009198
:10F5D000BC331091BD332091B6333091B733409195
:10F5E000B8335091B9338F938091B5338F93809115
:10F5F000B4338F938091B3338F938091B2338F93D1
:10F6000069EC73E38FE693E30E940888182F0F904C
:10F610000F900F900F900F9060E08BE992E30E94A3
:10F62000894F8091C433813061F480916A338111B4
:10F6300004C00E948A5A812F38C00E94BB5A812F71
:10F6400034C0812F32C08BEC30C083E02EC084E800
:10F650002CC083E82AC01092B93D60916B33709141
:10F660006C3380916D3390916E330E94234F809163
:10F67000ED33882309F406CEFFCD85E616C086E675
:10F6800014C0822D90E0FC01E154F109EA31F1054A
:10F6900000F7E156FE4F0C949EE0D8018C9174C99E
:10F6A00068018B2D78017B2C3EC92796CDBFDEBF2C
:10F6B000DF91CF911F910F91FF90EF90DF90CF904E
:10F6C000BF90AF909F908F907F906F905F904F9082
:10F6D0003F902F900895CF93DF93EC016FED7CE383
:10F6E0000E94F8658093B93D811102C095E09F8327
:10F6F000DF91CF910895FC018789908D0C945F7400
:10F7000083FF06C0E0913D30F0913E3090E295835A
:10F7100082FF06C0E0913F30F091403090E2958347
:10F7200081FF06C0E0914130F091423090E2958334
:10F7300080FF06C0E0914330F091443080E2858341
:10F74000089583FF06C0E0913D30F0913E3090E295
:10F75000968382FF06C0E0913F30F091403090E206
:10F76000968381FF06C0E0914130F091423090E2F3
:10F77000968380FF06C0E0914330F091443080E2F0
:10F78000868308958091BF3A811107C084E00E946A
:10F79000807B81E08093BF3A089584E00E94A17B42
:10F7A0001092BF3A0895CF92DF92EF92FF920F939B
:10F7B0001F93CF93DF93C12C26E0D22EC0922D3021
:10F7C000D0922E3030EAE32E36E0F32EE0922F3046
:10F7D000F092303000E816E0009331301093323070
:10F7E000C0E6D6E0C0933330D0933430C092353089
:10F7F000D0923630C0933730D093383000933930C0
:10F8000010933A30E0923B30F0923C302DEC3CECDF
:10F810004CED50E40E9456DAC0923D30D0923E301A
:10F82000E0923F30F092403018164CF4C0934130D3
:10F83000D0934230009343301093443008C000937B
:10F84000413010934230C0934330D0934430DF9125
:10F85000CF911F910F91FF90EF90DF90CF9008957F
:10F860000E9437D660E070E080E091E40E94D37B94
:10F870000C9456D681E08093C83A089520E093E036
:10F8800088ED08B618BE84BF909380002091820056
:10F8900021FDFCCF08BEFFCF8091C83A81110E94A4
:10F8A0003E7C83E008958091C93A882341F0F89422
:10F8B00061E089E790E00E9439D682E0089583E014
:10F8C0000895CF93DF93CDB7DEB7AD97CDBFDEBF41
:10F8D00021E2E4E0F2E2DE01119601900D922A9518
:10F8E000E1F722E02093CA01DE019296E8E0F0E021
:10F8F00024912D933196EE30F105D1F72DE228A712
:10F90000E0E1F0E0E491EF7121E030E02C0F3D1FE9
:10F910002E0F311DF901208129A7E2E1F0E0E491E9
:10F92000EF719E012E0F311DF90121812AA7E4E11B
:10F93000F0E0E491EF719E012E0F311DF90121815C
:10F940002BA71CA61092CA0125E0FC012783BE014B
:10F950006E5D7F4F0E94F8658093B93DAD96CDBF37
:10F96000DEBFDF91CF91089581E08093C93A80E0B6
:10F970000895CF93DF93EC0120E030E040E051E4C4
:10F9800069857A858B859C850E9456DA18166CF0FD
:10F99000CE010E94226369857A858B859C850E94B1
:10F9A000D37B0E94E8BF80E001C08DE6DF91CF915C
:10F9B00008956BEE7BE30C947BC56DEC7BE30C94BC
:10F9C0007BC56EEA7BE30C947BC560E97BE30C941A
:10F9D0007BC56CE77BE30C9426C5CF93DF9381E373
:10F9E00097E49F938F93CFE4DAE589818F938881A1
:10F9F0008F930E942DE58BEF94E49F938F938981E1
:10FA00008F9388818F930E942DE583E794E49F93E1
:10FA10008F9389818F9388818F930E942DE589EA46
:10FA200093E49F938F9389818F9388818F930E9412
:10FA30002DE50E94A1AB8DB79EB740968DBF9EBFAE
:10FA400080E0DF91CF910895CF93DF9384E893E432
:10FA50009F938F93CFE4DAE589818F9388818F9389
:10FA60000E942DE586E192E49F938F9389818F9385
:10FA700088818F930E942DE58BE890E49F938F936C
:10FA800089818F9388818F930E942DE583E794E489
:10FA90009F938F9389818F9388818F930E942DE507
:10FAA00089EA93E49F938F9389818F9388818F93C1
:10FAB0000E942DE58DB79EB744968DBF9EBF80E016
:10FAC000DF91CF910895CF93DF938AE690E49F93DF
:10FAD0008F93CFE4DAE589818F9388818F930E9499
:10FAE0002DE58CEE9CE39F938F9389818F93888182
:10FAF0008F930E942DE589EA93E49F938F938981E8
:10FB00008F9388818F930E942DE58DB79EB70C96B9
:10FB10008DBF9EBF80E0DF91CF910895CF93DF939B
:10FB200084EC9CE39F938F93CFE4DAE589818F93F4
:10FB300088818F930E942DE583E59CE39F938F93AB
:10FB400089818F9388818F930E942DE589EA93E4C0
:10FB50009F938F9389818F9388818F930E942DE546
:10FB60008DB79EB70C968DBF9EBF80E0DF91CF9181
:10FB70000895CF93DF9380E39CE39F938F93CFE42B
:10FB8000DAE589818F9388818F930E942DE587E044
:10FB90009CE39F938F9389818F9388818F930E9499
:10FBA0002DE589EA93E49F938F9389818F938881D0
:10FBB0008F930E942DE58DB79EB70C968DBF9EBF8B
:10FBC00080E0DF91CF9108952F923F924F925F9204
:10FBD0006F927F928F929F92AF92BF92CF92DF925D
:10FBE000EF92FF920F931F93CF93DF93CDB7DEB7C2
:10FBF0006A97CDBFDEBF5C010E9438652C011F866D
:10FC0000188A198A1A8AF50101900020E9F73197BC
:10FC1000EA19FB09E130F24008F002C2D5018C91EB
:10FC2000882359F17501BFEFEB1AFB0A850120E02B
:10FC3000211115C0883229F08132C8F08F37B9F010
:10FC400001C021E06801EFEFCE1ADE0A90E02A8FB2
:10FC50000E9437E4D8018C9386012A8D08C021E0E8
:10FC6000893209F420E0F80180830F5F1F4FD7012C
:10FC70008D917D018111DCCF01C08501F8011082D9
:10FC80001092B93DFDE19F2EAAE36A2EA2E27A2EE0
:10FC9000812CB6E02B2E03C09A9409F49CC18BE70B
:10FCA0009CE2A2E2B0E08B879C87AD87BE876B8A1F
:10FCB0007C8A8D8A8DE79CE2A2E2B0E08F839887F0
:10FCC000A987BA87E5E2F2E2DE011196822D019062
:10FCD0000D928A95E1F7C2010E943F648501075F9A
:10FCE0001F4F75019FEFA91AB90AD7016C9170E0F7
:10FCF000CE010B960E9494E4892B21F487010E5DBE
:10FD00001F4F04C0A016B10661F793C16501BFEF94
:10FD1000AB1ABB0AF601608170E0CE0143960E94E7
:10FD200094E4892B91F0D6011D928D0192012F5EF2
:10FD30003F4F288F398F46E050E0B701C9010E943C
:10FD4000BFE43AE0C30ED11C04C0A016B106F1F620
:10FD500070C15801D8013D908D01E32CF12CC701F1
:10FD60000E941BE4892B59F4B701CE0101960E9431
:10FD700094E4892B21F40C151D0559F75AC185010E
:10FD8000BEE63B1641F0E2E23E120CC0D5011196F0
:10FD90008C918232A9F5F2011782118612861386A0
:10FDA0001486A3C0B0E3EB1AF108EAE0EE16F10402
:10FDB00018F0FDE23F1217C0BE016A5E7F4FC50119
:10FDC0000E94BEE0D20119966D937D938D939C9312
:10FDD0001C978E899F898A159B0509F42DC1E4E043
:10FDE0001796EC9382C0FBE73F124FC0E7E0D201C9
:10FDF0001796EC93FFEFAF1ABF0AE2E0FE2E95C014
:10FE00002FEFA21AB20AE5E0D2011796EC9362E254
:10FE100070E0C5010E9494E48E8B9F8B009709F4DB
:10FE200008C1DC011C92F50101900020E9F731972F
:10FE3000EA19FB093397C8F0F80181818033A9F4EE
:10FE40008281883791F440E050E060E070E0C501C5
:10FE50000E942FE2D20119966D937D938D939C930E
:10FE60001C9783E017968C9308C0B501C2010E94CD
:10FE7000F8658093B93D811153C0AE88BF88BFEF4C
:10FE8000AB1ABB0AAE8ABF8A30C0E4E73E120EC08E
:10FE9000E1E0D2011796EC9380E090E0A0E8BFE3A8
:10FEA000F20181879287A387B4871FC0F6E63F12CD
:10FEB0000CC0E1E0D2011796EC93179719961D92AA
:10FEC0001D921D921C921C9710C0BBE53B12B1C045
:10FED000F2012782B501C2010E94F8658093B93D05
:10FEE00081111EC077E6F72E7DC0BE01695F7F4F8E
:10FEF000C5010E94D9E45C01009709F49AC0DC01B5
:10FF00008C918D3729F411968C91F50131965F0112
:10FF10008C3209F48BC0FFEFAF1ABF0AF12C05C079
:10FF2000F82E22E0281708F45DC08F858201035F58
:10FF30001F4F882341F043E050E0BE01615F7F4FD7
:10FF4000C8010E94BFE4688D798DC8010E94996341
:10FF5000D20114968D939C9315978F3FBFEF9B070B
:10FF6000B9F10E94E768882371F0888D998D0E940D
:10FF70008263882341F043E050E0688D798DCE01A3
:10FF80000F960E94BFE4F201428053804114510455
:10FF900011F1F11081CE80915635811108C08FE4A6
:10FFA00095E30E945D608093B93DF82E1BC080915F
:10FFB0006B32823099F08FE495E30E943360809336
:10FFC000B93D81110EC08FE495E30E94B0600AC074
:10FFD00064E6F62E07C050E7F52E04C04BECF42E75
:10FFE00001C0F82E42E060E08F2D0E949F6681E004
:10FFF0000E9495AD6A96CDBFDEBFDF91CF911F9174
:020000021000EC
:100000000F91FF90EF90DF90CF90BF90AF909F90B7
:100010008F907F906F905F904F903F902F900895BA
:100020008BE68093B93D3BE6F32EDCCF22E0F22E47
:100030007CCF9FE6F92ED6CF86E6F82ED3CF2F922F
:100040003F924F925F926F927F928F929F92AF9268
:10005000BF92CF92DF92EF92FF920F931F93CF93B5
:10006000DF9300D000D0CDB7DEB78C0169837A83EF
:100070004B835C835A0128E0A21AB108A60EB71E72
:10008000DC0116967C907B01BFEFEB1AFB0A8BE735
:10009000FB01808380E0912C95E0692E2FE2422EB7
:1000A00022E2522E3BE2232E32E2332E4DE7842E03
:1000B000ED82FE82D80117969C919F3F09F429C1D9
:1000C000882339F02CE2ED81FE8120833196ED8387
:1000D000FE838091633D811119C0C80141969F93B1
:1000E0008F933F922F923E813F938D818F930E94F9
:1000F000F8E5AD81BE81A80FB91FAD83BE830F9017
:100100000F900F900F900F900F9018C0C80141965C
:100110009F938F935F924F92BE81BF93ED81EF9338
:100120000E94F8E52D813E81280F391F2D833E83E3
:100130000F900F900F900F900F900F90D80117967F
:100140008C911797843059F51996CD90DD90ED90EC
:10015000FC901C97A7019601C701B6010E9419DC0B
:10016000811117C0E894F7F82FEF3FEF4FE75FE7F3
:10017000C701B6010E9419DC811121C12FEF3FEFA9
:100180004FE75FE7C701B6010E9453D818160CF07D
:1001900016C1F801118612861386148610C18111CA
:1001A00013C0E5E3F2E2AD81BE81862D01900D9290
:1001B0008A95E1F72D813E812C5F3F4F2D833E8351
:1001C000D80117968C9199C0823061F4F80184852A
:1001D0008F9383858F9382858F9381858F93AAE3F5
:1001E000B2E214C0833029F5D8011C968C911C977B
:1001F0008F931B968C911B978F931A968C911A97BD
:100200008F9319968C918F93A0E4B2E2BF93AF9332
:10021000FE81FF932D812F930E94F8E5AD81BE8171
:10022000A80FB11DAD83BE83F8018781CDBFDEBFAE
:1002300064C0853059F4D80158968C9158978F93A3
:1002400057968C918F93A8E4B2E20CC0863009F5E2
:10025000D80158968C9158978F9357968C918F937D
:10026000ADE4B2E2BF93AF93FE81FF932D812F9354
:100270000E94F8E5AD81BE81A80FB11DAD83BE839C
:10028000F80187810F900F900F900F900F900F90B3
:1002900034C0813091F52CEA35EC47E257E3D801C0
:1002A00019966D917D918D919C911C970E9453D8C8
:1002B00087FF12C0E2E5F2E2AD81BE8186E00190E7
:1002C0000D928A95E1F7ED81FE813596ED83FE83EF
:1002D000D80117968C9111C0E8E5F2E2AD81BE819C
:1002E000862D01900D928A95E1F7ED81FE8134967D
:1002F000ED83FE83D80117968C91873049F42BE764
:10030000ED81FE8120833196ED83FE8380E001C084
:1003100081E0AD81BE81AA15BB0518F08FEF9FEF7C
:1003200065C0F801028113810115110549F0D8015A
:1003300016969C912FEF290D99153CF0992EBACE67
:10034000ED80FE807914B4F020C0ED81FE81D801EB
:10035000CF010196808216969C9016973FEF320F40
:1003600092161CF4232FFC01F3CF8D839E838D0105
:1003700081E0A0CEF7012DE7CF01019620839A946A
:10038000791414F4FC01F8CF7C018DE79AE0A0E029
:10039000F70180839183A283F2E0EF0EF11C898143
:1003A0009A812B813C81820F931F8E159F0508F443
:1003B000B5CFC701A981BA818A1B9B0B17C0C801A1
:1003C0000E94F768F8014185528563857485208510
:1003D0008D819E810E94BFC72D813E81280F311DD6
:1003E0002D833E83D80117968C9187CF2696CDBF5B
:1003F000DEBFDF91CF911F910F91FF90EF90DF90C3
:10040000CF90BF90AF909F908F907F906F905F90B4
:100410004F903F902F90089540E052E06FED7AE3C7
:100420000E941F8060914F5A7091505A8FED9AE34D
:100430000C947CE5EF92FF920F931F93CF93DF9381
:10044000CDB7DEB76297CDBFDEBFF82E9091613D8C
:10045000992309F4B2C08FE6F81212C00E943865E1
:100460006FED7CE38091DB3A9091DC3A0E949FC76C
:10047000BC018EE191E20E9456660FE415E34AC08A
:1004800080916B320FE415E3882309F443C0EE2416
:10049000EA94C8010E94FF638823E1F1823029F4C5
:1004A0008091683D811120C01DC0843029F4809165
:1004B000653D811119C016C08530B1F48091673D4A
:1004C000882381F0F80181859285A385B485BC01DC
:1004D000CD019F772CEA35EC47E257E30E9453D8D1
:1004E00087FF02C0F801E782F8010281138101153C
:1004F000110579F60FC0F80102811381011511056C
:1005000049F440E052E06FED7AE386E395E30E9420
:100510001F8053C0F80197819F3F69F78091D529CB
:1005200081111AC08091DE3A8F938091DD3A8F93CA
:100530001F92FF928DE592E29F938F93CE010196D9
:100540007C01FF928F930E94F8E51092DD3A1092A1
:10055000DE3ACDBFDEBF13C00E941FCC1F928F9327
:100560001F92FF9285E692E29F938F93CE010196B0
:100570007C01FF928F930E94F8E5CDBFDEBFB701EB
:10058000C8010E94F865F801168286E0878386E636
:1005900090E0818B928B1282138240E052E06FEDEB
:1005A0007AE386E395E30E941F8060914F5A709131
:1005B000505A8FED9AE30E947CE56296CDBFDEBF74
:1005C000DF91CF911F910F91FF90EF9008956130CF
:1005D00019F0623029F008958FE495E30C940C82B1
:1005E0000C941A82CF92DF92EF92FF92FC01C184A9
:1005F000D284E384F48420E030E040EA50E4C70190
:10060000B6010E9456DA18160CF453C0C701B601A1
:100610000E94C7D86093613D1092643D1092653D81
:100620001092663D1092673D1092683D20E030E0E8
:1006300040E85FE3C701B6010E9456DA87FD03C0B8
:1006400081E08093643D20E030E040E050E4C70169
:10065000B6010E9456DA87FD03C081E08093653DB4
:1006600020E030E040E450E4C701B6010E9456DAD1
:1006700087FD03C081E08093663D20E030E040E8E4
:1006800050E4C701B6010E9456DA87FD03C081E03D
:100690008093673D20E030E040EA50E4C701B601B6
:1006A0000E9456DA87FD07C081E08093683D80E0B4
:1006B00003C08EE601C080E0FF90EF90DF90CF9006
:1006C000089563ED77E40C943CC56CE777E40C94F3
:1006D0003CC568E477E40C943CC5BF92CF92DF92AE
:1006E000EF92FF920F931F93CF93DF93CDB7DEB7B7
:1006F0006897CDBFDEBF6B0128E1FC01DE011196DA
:1007000001900D922A95E1F78CE2E82E81E3F82E14
:100710008E010F5F1F4FB12CF7018081823029F4C9
:10072000F80110821182128213828091D1588B11AC
:1007300014C02091E4583091E5584091E65850910A
:10074000E758F80160817181828193810E94F8DA13
:10075000F60160837183828393838091F0588B11BB
:1007600014C020910359309104594091055950917A
:100770000659F80160817181828193810E94F8DAC3
:10078000F601648375838683978380910F598B115B
:1007900014C02091225930912359409124595091ED
:1007A0002559F80160817181828193810E94F8DA74
:1007B000F601608771878287938780912E598B110C
:1007C00014C0209141593091425940914359509160
:1007D0004459F80160817181828193810E94F8DA25
:1007E000F6016487758786879787B394F5E3EF0EE4
:1007F000F11C0C5F1F4F86E0B8128ECF6896CDBFFC
:10080000DEBFDF91CF911F910F91FF90EF90DF90AE
:10081000CF90BF900895F8940E94307C0E9462842B
:100820000E9456D60E949BC90E943AB60E941A7432
:100830000E94E8BF0E9428A940E060E080E00E949A
:10084000DD690E9475650E9450840E9454860E9452
:10085000BD530E944ED68091A20084608093A20076
:100860008091A20082608093A2008091A2008160AA
:100870008093A20078940E94A1AB0E94FDC00E94C8
:10088000446AFDCFE82FF0E0EE0FFF1FE150F84B78
:10089000659174914FE450E089E69DE30C9466E421
:1008A0008091BD3A823041F440E060E081E00E94F6
:1008B000DD6980E00E94596B0C941DCD682F81E0AA
:1008C0000C948ECA1092BA3D1092BB3D1092BC3D62
:1008D0001092BD3D0895CF93DF93EC018C819D81F3
:1008E000880F991F880F991F2091BC3D3091BD3D05
:1008F000820F931F8093BE3D9093BF3D44E050E034
:1009000064EC7DE30E944ED54091C43D5091C53DBD
:100910006091C63D7091C73D49875A876B877C8738
:1009200080E0DF91CF9108958F929F92AF92BF9216
:10093000CF92DF92EF92FF92CF93DF93EC01809101
:100940006C32882369F089E0DF91CF91FF90EF90BE
:10095000DF90CF90BF90AF909F908F900C9429AB79
:1009600089859A85AB85BC858093C03D9093C13DB8
:10097000A093C23DB093C33DCE010E946B8480938F
:10098000B93D81116EC0C984DA84EB84FC84A7016F
:100990009601C701B6010E9419DC81112FC04601E2
:1009A0005701E894B7F82FEF3FEF4FE75FE7C50136
:1009B000B4010E9419DC81110AC02FEF3FEF4FE70D
:1009C0005FE7C501B4010E9453D81816BCF08090AF
:1009D000C03D9090C13DA090C23DB090C33DA501E7
:1009E0009401C701B6010E94E4D69F772CEA35EC4A
:1009F00047E257E30E9456DA181674F58091C03D1D
:100A00009091C13DA091C23DB091C33D8093C43D42
:100A10009093C53DA093C63DB093C73D8C819D8109
:100A2000880F991F880F991F2091BC3D3091BD3DC3
:100A3000820F931F8093BE3D9093BF3D44E050E0F2
:100A400064EC7DE30E94DFD58090C03D9090C13D75
:100A5000A090C23DB090C33D89869A86AB86BC8685
:100A600080E0DF91CF91FF90EF90DF90CF90BF902B
:100A7000AF909F908F9008950E945ABB80E0089598
:100A80008091C83D9091C93D8F3E924111F08EE515
:100A900008958091EE3D9091EF3D8F3E9241B9F7E0
:100AA0008091F03D9091F13D8F3E924181F7809190
:100AB000595590915A558F3E924149F780915B5517
:100AC00090915C558F3E924111F78091ED56909137
:100AD000EE568F3E9241D9F680E0089594E0899FCA
:100AE000F0011124E853F24C4283538364837583ED
:100AF000089594E0899FF0011124E55AFA4A45AB24
:100B000056AB67AB70AF08955F926F927F928F92F2
:100B10009F92AF92BF92CF92DF92EF92FF920F938C
:100B20001F93CF93DF93CDB7DEB76097CDBFDEBF06
:100B3000BE016F5F7F4F80E995E50E946D83CE0116
:100B400001964C0188E0A82E86E5B82E98E1C92EC2
:100B500096E5D92E28E2E22E26E5F22E08E416E5E7
:100B600038E6632E39E5732E512CF40141915191F1
:100B7000619171914F01F50141935193619371938B
:100B80005F01F60141935193619371936F01F701F6
:100B900041935193619371937F01852D0E943C7421
:100BA000F80111921192119211928F01F3011082AA
:100BB0001182128213825394F8E16F0E711C84E04B
:100BC0005812D3CF6096CDBFDEBFDF91CF911F917A
:100BD0000F91FF90EF90DF90CF90BF90AF909F90DC
:100BE0008F907F906F905F9008958091F23D08956F
:100BF0001F93CF93DF938BE697E1E0EFFDE3DF01F7
:100C00009C011D9221503040E1F78FEE92E18093DC
:100C1000F03D9093F13D8093595590935A55C9EF0B
:100C2000DDE3C093F33DD093F43DC093F53DD09305
:100C3000F63DC093F73DD093F83D81E090E06EE93A
:100C400074E520E030E01BEB129FA001139F500DD4
:100C50001124FA01E051F24CD90111961A9F90012A
:100C60001B9F300D11242750324C23873487618716
:100C70007287BA016750724C9C01019680329105CF
:100C800019F78BEB829FF001839FF00D1124E05147
:100C9000F24CC387D4876187728780E28093F23DEC
:100CA000DF91CF911F910895CF93DF93EBE5F5E5A9
:100CB00084E991E0DF01EC011D922197E9F7A8ECAE
:100CC000BDE388E2ED0119928A95E9F78FEE92E192
:100CD0008D939C938093EE3D9093EF3D8083918321
:100CE0008093ED569093EE56DF91CF910C94F8855A
:100CF0000E944F900E94F88580E00C94D84EE091BD
:100D0000F33DF091F43D848581111BC02281338134
:100D1000808191814BEBDF011D924A95E9F7228397
:100D200033838083918381E084878091F23D815079
:100D30008093F23D828193818093F33D9093F43DC3
:100D400005C08CE10E9429ABE0E0F0E0CF010895FE
:100D5000A5EFBDE3ED91FC911197858781E0878731
:100D600082E08487828193818D939C9381E00E94AD
:100D7000E6AE0C94A0B8EF92FF920F931F93CF931F
:100D8000DF9300D01F92CDB7DEB78C014B835C831D
:100D900069837A830E947F86FC014B815C81698133
:100DA0007A81009761F48EE02496CDBFDEBFDF919B
:100DB000CF911F910F91FF90EF900C940D5383E012
:100DC00085878CE395E884839583068317838B015D
:100DD0007A0126E0D8014D915D916D917D918D0153
:100DE000CF0185599F4FDC014D935D936D937C93AB
:100DF0001397D7014D915D916D917D917D01418B4F
:100E0000528B638B748B215034962111E3CF83E096
:100E10002496CDBFDEBFDF91CF911F910F91FF9040
:100E2000EF900C94A886CF92DF92EF92FF926B0125
:100E30007C010E947F86009739F48EE0FF90EF904E
:100E4000DF90CF900C940D5326E937E8FC01248302
:100E50003583E556FF4FC082D182E282F38221E0E2
:100E6000FC01278782E00E94A88680E0FF90EF9037
:100E7000DF90CF9008958091F73D9091F83DFC016F
:100E800024853EEF320F323018F424E02487089591
:100E9000243011F080E090E00895E091F73DF0916A
:100EA000F83D22813381808191814BEBDF011D92DE
:100EB0004A95E9F72283338380839183E091F73D5C
:100EC000F091F83D0280F381E02DE093F73DF0933F
:100ED000F83D8485823011F483E084878091F23D6F
:100EE0008F5F8093F23D8FEF0E94E6AE81E04091EC
:100EF000F33D5091F43D2091F73D3091F83D42177C
:100F0000530709F080E00895BC016F5E7F4FDC015C
:100F10001696ED91FC91179785599F4F19950E9450
:100F20004D8781110E94575A80E0089585569F4F42
:100F300020E034E244E759E4FC0160817181828160
:100F400093810E94F8DA0E94C7D80E94F3D80E94C9
:100F500064BB0E944D8781110E94575A80E008951A
:100F60008091F73D9091F83DFC0124853EEF320FD2
:100F7000323018F424E024870895243011F080E002
:100F800090E00895CF93DF93C091F73DD091F83D65
:100F90008C859EEF980F923018F484E08C8705C002
:100FA000843019F080E090E010C02097D9F3DE0182
:100FB0001296ED91FC9113978785882329F0EC1701
:100FC000FD0711F0DF01F4CFCD01DF91CF9108953E
:100FD000CF93DF93EC012A813B81888199814BEB90
:100FE000FB01DE0101900D924A95E1F72A833B83D4
:100FF00088839983DF91CF9108958FEE92E180935A
:10100000EF569093F0568093AB579093AC5708955A
:101010002F923F924F925F926F927F928F929F9208
:10102000AF92BF92CF92DF92EF92FF920F931F93F6
:10103000CF93DF93CDB7DEB76B97CDBFDEBF4C014B
:101040001B0129013A01EB86FC860D871E871A2DAC
:101050000B2DE9A8BAA8ABA82CA929838091E4326A
:10106000882399F08091D8329091D932A091DA32C8
:10107000B091DB32BC01CD019F772CEA35EC47E221
:1010800057E30E9453D887FDEFC680910C349091AE
:101090000D34A0910E34B0910F34BC01CD019F7777
:1010A00031E039872CEA35EC47E257E30E9456DA03
:1010B000181614F0198610C02DEC3CEC4CEC5DE3D6
:1010C0006091B2337091B3338091B4339091B53362
:1010D0000E9453D887FDCAC6F10180819181A28107
:1010E000B381BC01CD019F77F1E0FD832CEA35ECA3
:1010F00047E257E30E9456DA18160CF01D82F10100
:1011000084819581A681B781BC01CD019F77F1E0F3
:10111000FF872CEA35EC47E257E30E9456DA1816AF
:101120000CF01F86F10180859185A285B385209101
:1011300010343091113440911234509113342F8B6C
:10114000388F498F5A8F2091143430911534409143
:101150001634509117342B8B3C8B4D8B5E8B40910A
:1011600018345091193460911A3470911B34F090F6
:10117000E532F11021C010923B5781E080933C573B
:1011800082E080933D573985332341F04D814111F1
:1011900071C65F8551116EC68CE99FC6CB01BA013D
:1011A0009F772CEA35EC47E257E30E9456DA18168F
:1011B0000CF065C68BE991C6BC01CD019F77A1E01B
:1011C000AB8F2CEA35EC47E257E30E9456DA18164B
:1011D0000CF01B8EB1E0FB1216C010923B5782E060
:1011E00080933C57F0923D57E985EE2339F0FD811D
:1011F000F11140C62B8D222379F23CC66B897C8984
:101200008D899E89CDCF32E0F31217C081E08093A3
:101210003B57F0923C5710923D574985442341F08B
:101220005F85511127C68B8D882309F4B5CF22C65F
:101230006F89788D898D9A8DB3CFB101C4010E94D9
:1012400027519985992309F451C02091A0323091FA
:10125000A1324091A2325091A3326091F432709148
:10126000F5328091F6329091F7320E94E4D69F7762
:101270002CEA35EC47E257E30E9453D887FF36C08B
:101280002091A4323091A5324091A6325091A732DC
:101290006091F8327091F9328091FA329091FB327C
:1012A0000E94E4D69F772CEA35EC47E257E30E9490
:1012B00053D887FF1BC02091A8323091A9324091AA
:1012C000AA325091AB326091FC327091FD32809124
:1012D000FE329091FF320E94E4D69F772CEA35ECE3
:1012E00047E257E30E9453D887FDC2C58DA980937A
:1012F0009F328BE992E30E942F4F85E5EBE9F2E301
:10130000A6E5B7E501900D928A95E1F788E1E4EF53
:10131000F2E3A2EFB6E501900D928A95E1F7809194
:10132000E6328111B1C523E333E34BEC51E46E2D7A
:101330007B2D8A2D99810E94F8DA4B015C01609324
:10134000265770932757809328579093295723E364
:1013500033E34BEC51E4C301B2010E94F8DA60932D
:101360000A5770930B5780930C5790930D5723E3B4
:1013700033E34BEC51E46B857C858D859E850E9423
:10138000F8DA60930E5770930F578093105790932D
:10139000115723E333E34BEC51E4612F702FC60167
:1013A0000E94F8DA162F072F412F502FBC014093CF
:1013B0001257509313576093145770931557809199
:1013C000AE339091AF33A091B033B091B133BC0143
:1013D000CD019F770E9430D90E94C7D82B013C01D4
:1013E00060933757709338578093395790933A5793
:1013F00010913B5780913C57A82FB0E0AB87BC873A
:101400007D01EE0CFF1CEE0CFF1CF101EE0DFF1D2B
:1014100080819181A281B381BC01CD019F772CEAAB
:1014200035EC47E257E30E9453D8881F8827881F6E
:101430008983E12FF0E0E987FA878F01000F111F00
:10144000000F111FF101E00FF11F80819181A28136
:10145000B381BC01CD019F772CEA35EC47E257E31D
:101460000E9453D8881F8827881FF981F823F983A1
:10147000F09336572CEA35EC47E257E3C501B40147
:101480009F770E9456DA181624F00D831E83870179
:1014900005C1E985FA85EE0FFF1FEE0FFF1FE0562D
:1014A000FD4CA985BA85AA0FBB1FAA0FBB1FAC5064
:1014B000BD4C2D913D914D915C91608171818281F6
:1014C00093810E94E4D66F87788B898B9A8BEB850A
:1014D000FC85EE0FFF1FEE0FFF1FE056FD4CAB85A6
:1014E000BC85AA0FBB1FAA0FBB1FAC50BD4C2D91D2
:1014F0003D914D915C9160817181828193810E94C7
:10150000E4D66B8B7C8B8D8B9E8BA5019401C501E2
:10151000B4010E94F8DA20E030E040E850E40E9494
:10152000F8DA6D837E838F8398872F853889498980
:101530005A89CA01B9010E94F8DA6B017C012B8932
:101540003C894D895E89CA01B9010E94F8DA9B0184
:10155000AC01C701B6010E94E5D69B01AC016D81CB
:101560007E818F8198850E94E4D66B017C0120E00A
:1015700030E0A9010E9456DA1816D4F4C701B6016A
:101580000E94D1DB6B017C012B893C894D895E89EE
:101590006F85788989899A890E9463DA9B01AC01F9
:1015A000C701B60190580E945AD86B017C0103C054
:1015B000C12CD12C760180919F32833021F4F7FA2F
:1015C000F094F7F8F09420E030E0A901C501B401EF
:1015D0000E9453D887FF04C0F7FAF094F7F8F0940C
:1015E00029853A85220F331F220F331F2D833E8317
:1015F00089010151194AA70196016B897C898D895E
:101600009E890E94F8DA9B01AC016F8578898989EF
:101610009A890E94E4D620E030E040E05FE30E9437
:10162000F8DAD8015B966D937D938D939C935E97CA
:101630000B851C85000F111F000F111FF801E151D0
:10164000F94A5F01A70196016F85788989899A898E
:101650000E94F8DA9B01AC016B897C898D899E8997
:101660000E94E5D620E030E040E05FE30E94F8DA37
:10167000D5015B966D937D938D939C935E97E091DE
:101680003D57F0E0EE0FFF1FEE0FFF1FE151F94A4B
:10169000138E148E158E168E1092B93DF801E151FD
:1016A000F94AC38CD48CE58CF68CF7FAF094F7F8F1
:1016B000F094ED81FE81E151F94A838D948DA58DE1
:1016C000B68DBC01CD019058A70196015F770E94AD
:1016D0005AD80E9449D74B015C0120E030E0A901B3
:1016E000C701B6010E9456DA1816C4F020E030E0B7
:1016F000A901B401C5010E9456DA9401A50118168A
:101700002CF46BED7FE089E490E404C06BED7FE0A6
:1017100089E490EC0E94E4D64B015C01C401D50140
:1017200080931E5790931F57A0932057B093215733
:101730009401A501B401C5010E9419DC8111C8C33F
:10174000B981BB23B1F1C301B2010E94F3D86B018F
:101750007C012CEA35EC47E257E30E9453D887FD21
:1017600011C0B0909F322BED3FE049EC50E4C7012F
:10177000B6010E94F8DA9B01AC01C12CD12CE12CFE
:10178000F12CEFC081E090E0A0E0B0E0809337570B
:1017900090933857A0933957B0933A57B0909F32EF
:1017A0002BED3FE049EC50E4C12CD12CE12CF12C85
:1017B000D8C0EB85FC85EE0FFF1FEE0FFF1FE55A2B
:1017C000F84A98012151394A7901D9015B962D9146
:1017D0003D914D915C915E97608171818281938191
:1017E0000E94E4D6F70123813481458156810E940D
:1017F000E4D66B017C01E985FA85EE0FFF1FEE0F41
:10180000FF1FE55AF84A2D813E812151394A1901BD
:10181000D9015B962D913D914D915C915E976081D0
:101820007181828193810E94E4D6F1012381348108
:10183000458156810E94E4D6A70196015F770E94F8
:101840005AD80E9449D71B0189839F8720E030E046
:10185000A901C701B6010E9456DA1816E4F020E08B
:1018600030E0A901B10189819F850E9456DA91017A
:1018700049815F8518162CF46BED7FE089E490E4D4
:1018800004C06BED7FE089E490EC0E94E4D61B017C
:10189000F82EE92E02C0F980EF84C101AF2DBE2DD4
:1018A0008093225790932357A0932457B0932557A2
:1018B00091014F2D5E2DB1018F2D9E2D0E9419DCBF
:1018C000811106C391014F2D5E2DB401C5010E9407
:1018D00056DA1816B4F42BED3FE049EC50E4B101B0
:1018E0008F2D9E2D0E94E5D61B01AB01BC014093BC
:1018F0002257509323576093245770932557F82EFF
:10190000E92E9401A501B1018F2D9E2D0E94E4D6F0
:101910006B017C01B0909F32F3E0BF1669F0C30108
:10192000B2010E94F3D82BED3FE049EC50E40E9455
:10193000F8DA9B01AC0115C02BED3FE049EC50E417
:101940000E94E4D66B017C01C301B2010E94F3D86E
:101950002BED3FE049EC50E40E94F8DA9B01AC012A
:1019600008C082E0B81205C0B601C7010E94E5D6E2
:1019700004C0B601C7010E94E4D66B01AB01BC01F3
:1019800040932A5750932B5760932C5770932D57A1
:101990007C01F801E151F94A238D348D458D568D36
:1019A000ED81FE81E151F94A638D748D858D968DAF
:1019B0000E9463DA2B013C016093265770932757EE
:1019C000809328579093295710913D57A12FB0E04D
:1019D000FD01EE0FFF1FEE0FFF1FE55AF84AAA0F99
:1019E000BB1FAA0FBB1FA151B94A13962D913D9160
:1019F0004D915C91169760817181828193810E94E3
:101A0000E4D64B015C0160932E5770932F5780935F
:101A10003057909331579601A701C301B2010E943C
:101A2000F8DA6B017C0160933257709333578093DF
:101A3000345790933557A50194010E9463DA698366
:101A40007A838B839C836093165770931757809388
:101A500018579093195720917730309178304091F2
:101A6000793050917A302D833E834F8358870E947E
:101A700053D887FD2FC28091E432811118C0309174
:101A8000D8323B8F4091D9324F875091DA325B8BFD
:101A90008091DB328F8B1092D8321092D932109213
:101AA000DA321092DB3281E08093E43212C020916E
:101AB000D8323091D9324091DA325091DB3269819B
:101AC0007A818B819C810E945AD86B8F7F878B8B08
:101AD0009F8B85E3A985BA858A9FF0018B9FF00DC6
:101AE0001124E35DFE4C2081318142815381C70185
:101AF000B6010E945AD86987072F382E292E2B8DC0
:101B00003F854B895F89832D922D0E9453D887FF93
:101B100003C0BB8DB98703C00F873B8A2F8A85E33B
:101B20002B853C85829FF001839FF00D1124E35D9E
:101B3000FE4C2081318142815381C701B6010E9450
:101B40005AD8F62E072F382E292E262F372F482F1A
:101B5000592F69857F858B899F890E9456DA1816CF
:101B600024F40F853B882F8801C0F9868985902F42
:101B7000A32DB22D80931A5790931B57A0931C57F7
:101B8000B0931D5720E030E0A901C501B4019F7753
:101B90000E9456DA18167CF535E3139FF0011124E4
:101BA000E35DFE4C2081318142815381C501B40146
:101BB0000E945AD86B017C01E894F7F8A7019601BE
:101BC0006985702F832D922D0E9456DA181614F411
:101BD000198504C01C2D0D2D3E2C2F2C812F902FEC
:101BE000A32DB22D80931A5790931B57A0931C5787
:101BF000B0931D5701C01985C0906E30D0906F30E2
:101C0000E0907030F090713020E030E040E850E437
